:10000000A0480020151201003FBA0100691201004A
:10001000691201006912010069120100000000006C
:10002000000000000000000000000000351001008A
:100030006912010000000000ED0F010099A8010005
:10004000D51101009DF40100D5110100D511010069
:10005000D5110100D5110100D5110100D511010004
:1000600065F40100D5110100D511010083F40100F0
:10007000D5110100D5110100D5110100D5110100E4
:10008000D5110100D5110100D5110100D5110100D4
:10009000D5110100D5110100D5110100D5110100C4
:1000A000D5110100D5110100D5110100D5110100B4
:0800B000D5110100D51101007A
:1000B80053B94AB9002908BF00281CBF4FF0FF31C7
:1000C8004FF0FF3000F06CB9ADF1080C6DE904CECB
:1000D80000F006F8DDF804E0DDE9022304B070471B
:1000E8002DE9F047089E0D4604468E46002B40F049
:1000F80082808A42174646D9B2FA82F24AB1C2F1E0
:10010800200105FA02F320FA01F1974041EA030EB3
:1001180094404FEA1748230CBEFBF8FCB9B208FB21
:100128001CEE43EA0E430CFB01F098420AD9FB1877
:100138000CF1FF3580F01681984240F21381ACF142
:10014800020C3B441B1AA4B2B3FBF8F008FB1033B3
:1001580044EA034400FB01F1A14209D93C1900F12A
:10016800FF3380F00181A14240F2FE8002383C4416
:10017800641A40EA0C4000211EB1D4400023C6E9AD
:100188000043BDE8F08702B9FFDEB2FA82F2002A26
:100198004FD1CB1B4FEA174E1FFA87F80121B3FB4B
:1001A800FEFC250C0EFB1C3345EA034508FB0CF34B
:1001B800AB4207D97D190CF1FF3002D2AB4200F2F5
:1001C800E7808446ED1AA3B2B5FBFEF00EFB10558E
:1001D80043EA054408FB00F8A04507D93C1900F19B
:1001E800FF3302D2A04500F2D7801846A4EB0804DA
:1001F80040EA0C40C0E78B4208D9002E00F0AF80DF
:100208000021C6E900050846BDE8F087B3FA83F186
:1002180000294BD1AB4202D3824200F2B780841A44
:1002280065EB030301209E46002EAAD0C6E9004EC6
:10023800A7E7C2F1200C01FA02F3974020FA0CF06C
:100248004FEA174E21FA0CFC1843BCFBFEF1050CD3
:100258000EFB11CC1FFA87F845EA0C4501FB08F3A1
:10026800AB4204FA02F409D97D1901F1FF3C80F090
:100278008B80AB4240F2888002393D44EB1A85B24C
:10028800B3FBFEF00EFB103345EA034500FB08F311
:10029800AB4207D97D1900F1FF3C71D2AB426FD94F
:1002A80002383D44EB1A40EA014178E7C1F1200CDD
:1002B8008B4022FA0CF71F4320FA0CF405FA01F3DD
:1002C8004FEA174E25FA0CF51C43230CB5FBFEF933
:1002D8001FFA87F80EFB195543EA054509FB08FA8A
:1002E800AA4502FA01F200FA01F308D97D1909F1C9
:1002F800FF3047D2AA4545D9A9F102093D44A5EBEB
:100308000A05A4B2B5FBFEF00EFB105544EA0544FD
:1003180000FB08F8A04507D93C1900F1FF352DD29C
:10032800A0452BD902383C4440EA0940A4EB080414
:10033800A0FB02894C45C6464D4619D316D05EB17E
:10034800B3EB0E0264EB050404FA0CFCCA404CEA59
:100358000202CC40C6E900240021BDE8F0873146FE
:1003680030460EE7AC46EDE6184601E74345E6D2CF
:10037800B8EB020E69EB07050138E0E72846D3E73A
:1003880060468FE78146BAE7614677E708464BE75C
:10039800ACF1020C3D4415E702383C4426E700BFA7
:1003A800704700BFF8B515460A4A1C4656682EB174
:1003B80001B02A46B446BDE8F040604700208DF8F9
:1003C800000068460AF048FC9DF80000281A2070D2
:1003D8000020F8BD00000020002819D00378134938
:1003E800134A13B1012B0ED011E00379012B00D071
:1003F8006BB943790BB1012B09D18368643B8B42FC
:1004080005D2C0680EE00379012B02D00BB10020A1
:10041800704743790BB1012BF9D1C368643B8B4218
:10042800F5D280689042F2D8012070473D860100DD
:10043800FF1FA10710B5054C206810B180470020A8
:100448002060BDE8104001F091BF000008000020C6
:100458002DE9F0410E46050004D000F045F80746A6
:1004680000240AE06FF01500BDE8F081204600F096
:1004780041F8807838B1641CE4B2BC42F6D300BFBE
:100488006FF00B00F0E72746FF2CF9D0204600F06C
:1004980031F804460AF083FD27712146074801F028
:1004A8003DFFE070202805D00120A560A0703770BE
:1004B8000020D9E76FF02200D6E7000007AD000062
:1004C80010B5820702D06FF00D0010BD054A1170FB
:1004D800506028B101EBC1018A0000210AF0F0FF49
:1004E800002010BD0C000020014800787047000073
:1004F8000C00002005490A78904201D3002070477B
:10050800496800EBC00001EB800070470C00002038
:1005180070B50546202A27D019481A4C00EB831CD1
:100528000CEB420004EB8303202922D00CEB4101A1
:1005380040784C784870204601460CEB41009142C7
:1005480005704078F8D193F82220202A1ABF0CEBC6
:100558004202547083F8214020220CEB410C8CF8A5
:10056800012083F8221070BD40F29121702003F021
:1005780013F993F82040407883F82000DBE7000067
:10058800CC0C00204C0D00202DE9FF4F0C4649896A
:1005980087B001F5E1611546814200F2DA8005AACB
:1005A80002A902F0B3F802980A9F284420F07F407D
:1005B8000490A948A94E00EB8700039090F82050BA
:1005C8002020E9460DF104088DF8000006F5407A70
:1005D800202D18BF0AEB871B26D000BF05EB45006E
:1005E80006EBC0002168C268891A0902CA1701EB24
:1005F80012610830091217D4618971B1418961B952
:1006080000F0B4FD02F066F82168081A0002C1176C
:1006180000EB11600012332806DB0BEB450089F86C
:1006280000504578202DD9D199F8000088F80000AD
:10063800A146202D1CBF8A4800EB871B00F00881CB
:1006480005EB450106EBC10AD9F80410DAF80820D1
:100658004846511A0902CA1701EB12610AF1080744
:10066800091215D47989002900F0F28041890029FE
:1006780040F0EE8000F07AFD02F02CF83968081A94
:100688000002C11700EB11600012332880F2E080ED
:1006980088F800509AF8141099F80C00814206D98D
:1006A8000BEB45004578202DCAD100F0D1B89DF854
:1006B800040000EB400006EBC005688AEF680028DC
:1006C8003FD16089E8B3A8680AF012FD698A2A7CDC
:1006D8001144491C634A4318904204D940F21661F8
:1006E800702003F059F86048814204DD40F2176138
:1006F800702003F051F85D48814204DA4FF4C36179
:10070800702003F049F85A489842DCBF03F5F70314
:10071800A3F1F85305DD002BBCBFA3F5F70303F1E4
:10072800F853184601F0D6FF20F07F40391A090225
:10073800CA1701EB126109123329BCBF333020F00C
:100748007F470498381A0002C11700EB11600012A5
:1007580003D40BB00020BDE8F08FD4E90010401A94
:10076800384427F07F4120F07F40C4E90010039807
:10077800DDF828806F4690F8205020200DF1040AFB
:100788008DF80000202D1CBF354800EB881924D0B7
:1007980005EB450006EBC0002268C168511A090242
:1007A800CA1701EB12610830091216D4618971B1B8
:1007B800418961B900F0DAFC01F08CFF2168081A60
:1007C8000002C11700EB11600012332805DB09EBAA
:1007D80045003D704578202DDAD138788AF8000038
:1007E8002746202D1CBF1E4800EB881B30D005EB88
:1007F800450106EBC1097968D9F808203846511A2D
:100808000902CA1701EB126109F10808091212D48A
:10081800B8F80A10E1B14189D1B900F0A7FC01F09C
:1008280059FFD8F80010081A0002C11700EB116030
:10083800001233280CDA8AF8005099F81400397B32
:1008480088427FF634AF0BEB45004578202DCED19A
:100858000BB00120BDE8F08F4C0D0020CC09002022
:10086800CC0C0020FF7F841E0020A10700E05EF86A
:100878000080841E2DE9F05F04463C480E4600EBDC
:1008880086003B4F90F820502020984692461070E2
:1008980007F54079202D18BF09EB861B28D000BF2B
:1008A80005EB450007EBC00000F10801C0682268AD
:1008B800101A0002C21700EB1260001218D46089E7
:1008C80078B1488968B9084600F050FC01F002FF89
:1008D8002168081A0002C11700EB116000123328C2
:1008E80006DB0BEB45008AF800504578202DD7D160
:1008F8009AF8000088F80000202D18BF09EB861A26
:1009080030D005EB450107EBC1096168D9F808202B
:100918002046511A0902CA1701EB126109F10806AB
:10092800091210D47189E9B14189D9B900F01EFCC6
:1009380001F0D0FE3168081A0002C11700EB1160FF
:10094800001233280EDA88F8005099F81400217B39
:10095800884202D80020BDE8F09F0AEB45004578A0
:10096800202DCED10120BDE8F09F00004C0D0020C5
:10097800CC0900202DE9F74F4FF0000898B0164633
:100988000D46C34602F01EF90446012D18BF022D7C
:1009980005D040F693114FF0700002F0FDFEFD49BE
:1009A80001200860FC498968086000200C90401EFE
:1009B8000E90FA4906EB460001EBC00308330FAF6F
:1009C8000FCB87E80F000FA800F0D0FB0D90F3487D
:1009D800BDF84690B0F89C03ADF84C00B9F1000F93
:1009E80014BF4FF0010A4FF0000A0F981490BAF1A3
:1009F800000F09D0EA4890F82C0028B902F068FEE8
:100A0800002808BF012700D00027E64800221592D9
:100A180000781646012818BF032840D1E148B0F8ED
:100A28000280A8EB09001590C84538D90D9B6FEADC
:100A38000801DFF874E358180DF10C0C17AA734578
:100A480004D940F21661702002F0A6FED74B9942F5
:100A580004DD40F21761702002F09EFED44B9942EB
:100A680004DA4FF4C361702002F096FED149814246
:100A7800DCBF00F5F700A0F1F85005DD0028BCBF89
:100A8800A0F5F70000F1F850614601F03FFE039829
:100A98000F9920F07F400390081A20F07F42002F22
:100AA80018BF322604D19DF84C00002818BF022632
:100AB800B4F1807F08D00F98001B0002C11700EB2B
:100AC80011600012012802DA042118980BE047B1DE
:100AD800B34890F82D0020B19DF84C00061C18BFB3
:100AE800022620460121B9F1000F02D0159B1E2BCA
:100AF80002DA9DF84C3013B14FF0010B491E8B19E7
:100B0800A8499DF84DE0097815910F99891A21F0A7
:100B18007F4CACEB00010902CE1701EB16610912FC
:100B2800994218DB002A18BFCDF83CC00F9E0597E4
:100B3800002701F041FF301A0002C11700EB1160D5
:100B480000123E283FDA012D20D0701E059920F0B2
:100B58007F4019B32DE082B1BEF1000F04BF159993
:100B680003290AD027B99DF84C10002918BF9B1EED
:100B780000228DF84C209046C7E707BB9DF84C1023
:100B8800E9B100218DF84C109B1EBEE7B4F1807FBF
:100B980020D140F60C11702002F0FEFDB4F1807FE8
:100BA80007D0211A0902CA1701EB12610912042998
:100BB80003DD044601F006FF0CE000290ADD1BB046
:100BC8000020BDE8F08F701E20F07F44204601F021
:100BD800F9FE5746B4F1807F28D00F98DDF840C061
:100BE800001B8BF00103744A20F07F40ACEB040C2F
:100BF8002CF07F4C834298BFB0F5800FDFD262455E
:100C0800DDD320460AF074FA67490D9A4B1C161A70
:100C1800B6EB930F24BFA0EB020CBCEB930F10D3E1
:100C2800B14208D2081A1044461C0AE040F62B21AB
:100C3800702002F0B1FD61452CD2891A0844401C8D
:100C480046425748807F50B3284645464FF0000B30
:100C5800D846012805D0022002F0FCF8012002F055
:100C6800F9F8A9452CD2A6EB05014FF001034FF086
:100C780003024FF0020002F025F8002808BF4FF0E9
:100C88000108B9F1000F35D00123A6EB09010322B1
:100C9800184623E040F60B31702002F07DFDC14577
:100CA80034BF40464846BBF1000F14BF00211E2147
:100CB8000844B042C8DB40F63E21702002F06CFDCB
:100CC80010D90123A6EB09010322184601F0FAFF07
:100CD80028B37DB1711B01230322022001F0F2FF2A
:100CE800E8B107E055EA090004D040F67611702013
:100CF80002F052FD012303223146002001F0E2FFF9
:100D080068B10125B8F1000F03D014980F908DF841
:100D18004CB0DFF8A880BAF1000F0ED109E002202C
:100D280002F098F8012002F095F81BB00020BDE809
:100D3800F08F1B4890F82D0000B14FB3DFF860A08A
:100D48009AF82C0018B102F06DFB8AF82CB007B3A2
:100D5800A4F1320020F07F414FF40020C8F80000D1
:100D680000230322052001F0ADFF68B34FF0804453
:100D7800052002F04FF91249C1F81005C1F81445D1
:100D88001049E0120860064C94F82D00F0B35BE0BF
:100D98001BE01FE00805004014000020CC090020DB
:100DA8004C0D002016000020FF7F841E0020A107A4
:100DB80000E05EF80080841EFFFF3F0008F5014058
:100DC80098F0014004F5014035E0DFF8B8A09AF842
:100DD8002C0058B32B4C94F82D0050B14FF4002040
:100DE800C8F80000052002F035F802F083FB84F80B
:100DF8002DB00CAC244894E80E10C0F88013C0F84D
:100E08008423C0F88833C0F88CC300E018E010AC25
:100E180094E80E10C0F89013C0F89423C0F89833E3
:100E2800C0F89CC31BB00120BDE8F08F02F016FB90
:100E38008AF82C508BE740F25131702002F0ACFC5C
:100E480002F04AFB84F82D50A6EB0900A0F1190125
:100E5800002904DC40F66821702002F09DFC032282
:100E68000123104601F02EFF38B108488068C0F809
:100E780000B00748C0F800B0BBE740F67321702007
:100E880002F08AFC4C0D0020CC0900201400002040
:100E9800080500402DE9F043064683B008789073B2
:100EA800CF7A5773887A10730889144650810D4693
:100EB8000A785F4999464FEA810C4B42ACF1010828
:100EC8005AB1C043D5F8048004F1080288423DDDD8
:100ED80040F21761702002F05FFCEE686D686FEAFF
:100EE800000904F1080206EB0900464504D940F25E
:100EF8001661702002F050FC8945E9DC994528DB31
:100F08008445DCBF00F5F700A0F1F85005DD0028A6
:100F1800BCBFA0F5F70000F1F850214601F0F6FB40
:100F2800206820F07F417019401C2160002F08BF05
:100F38007A3003D0012F08BF44302DD101F0CAFB0D
:100F480020F07F40606003B0BDE8F083014698421E
:100F580004DA4FF4C361702002F01EFC8445DCBF44
:100F6800A1F1F450A0F5902005DD0028BCBF01F1E7
:100F7800F45000F59020214601F0C8FB2068002FAE
:100F880020F07F4108F10100216008BF7A3008D0C5
:100F9800012F08BF443004D040F2BE61702002F037
:100FA800FBFB01F097FB20F07F416160608901AA9B
:100FB800694601F0ABFB1F4890F82F10202923D079
:100FC8000069401D20F07F40D4E90021891A206083
:100FD800084420F07F4060604B4632462146E8686E
:100FE800FFF7D2FA00281CBF03B0BDE8F083D4E9AC
:100FF8000010401A304426F07F4120F07F40C4E9B9
:10100800001003B0BDE8F083608906F1090720B13C
:1010180002F05EFB002808BF323707484178009885
:10102800814284BF081A074427F07F40CCE70000BC
:101038000020A1074C0D00201600002010B5154C0B
:1010480094F82F00202818BF10BD94F82E2004EB28
:10105800820090F82010202917D0DFF83CC00CEB54
:10106800821303EB41035B7880F82030012380F87A
:10107800233084F82B3084F82F10022000F0B0F8C9
:10108800002084F82A00A07710BD40F29E3170201D
:1010980002F082FB4C0D0020CC0C00202DE9F05F03
:1010A800DFF8B88098F82E5008EB850090F82140BA
:1010B800202C08BFBDE8F09FDFF8A4B0DFF8A4A09B
:1010C800AAF540790AEB8517072617F814000128B6
:1010D8000ED0042808BF02260AD005280CBF032614
:1010E800062805D040F6D8014FF0700002F054FBF6
:1010F800BBF1000F18BFAFF30080EFF3108072B69A
:1011080007EB44014A7808EB850181F8212091F822
:101118002220A24204BF202281F82220B8B12A4608
:101128002146012000F05CF804EB440109EBC10002
:1011380059F8312040683146904798F82E5008EB0E
:10114800850090F82140202CBCD1BDE8F09F0648CE
:10115800002818BFAFF3008062B6E0E74C0D00200E
:1011680000000000CC0C00200000000010B5044670
:10117800006809F0BDFF02466089217A144B0844D3
:10118800411C50189A4204D940F21661702002F0AE
:1011980003FB104A914204DD40F21761702002F00F
:1011A800FBFA0D4A914204DA4FF4C361702002F051
:1011B800F3FA0A498142DEBF00F5F700A0F1F850C2
:1011C80010BD0028BCBFA0F5F70000F1F85010BD15
:1011D800FF7F841E0020A10700E05EF80080841EC7
:1011E800DFF854C010B500230CEB821C07281ED270
:1011F800DFE800F0050505050404040001230CF8E8
:101208001100002B08BF10BD0C4800EB820292F8B9
:10121800220020280EBF82F821100CEB40004170FC
:1012280020200CEB4103587082F8221010BD40F2C8
:101238006721702002F0B0FACC0C00204C0D002081
:101248002DE9F34F83B05C48049900EB81000190CD
:1012580090F8204003982546012818BF022805D099
:1012680040F6AF214FF0700002F096FA0027202DCB
:101278004AD0514800910026807F002808BF0226E6
:1012880001F09AFBDFF838A104EB44010AEBC10135
:10129800DFF828918A68C968121A091A22F07F4271
:1012A80021F07F41964298BFB2F5800F01D289455F
:1012B80028D2444A009902EB811B22460BEB4201DB
:1012C8004C78202C16D004EB44010AEBC10CDCF856
:1012D8000880DCF80CC0A8EB000828F07F48ACEBCD
:1012E800000121F07F41464598BFB8F5800FE4D250
:1012F8008945E2D3202A05D020210420009BFFF74E
:1013080007F90446AC4215D12F48002818BFAFF39F
:10131800008001F051FB284C94F8301020290DD0A2
:10132800E168821C511A0902CA1701EB12610912FD
:10133800002903DD05B00020BDE8F08F202D0DD079
:101348002A460399FFF716FB58B3019880F82370D3
:1013580084F8305005B00120BDE8F08F94F82C00D7
:1013680018B102F05FF884F82C7094F82D0050B191
:1013780016494FF400200860052001F06BFD02F0CB
:10138800B9F884F82D70042001F064FD01F0CAFD5D
:10139800202084F830000E48806807600D480760F8
:1013A800D8E72A4620210420049BFFF7B1F805B0AE
:1013B8000020BDE8F08F00004C0D0020FFFF3F002B
:1013C800CC090020CC0C00200000000008F50140EA
:1013D8001400002008050040064910B591F82F2098
:1013E800202A1CBF887710BD40F2FD31702002F022
:1013F800D3F900004C0D00202DE9F04F5B4E8146DB
:1014080085B096F82F008A4620284DD096F82F00F0
:1014180006F10C0400EB4000A6F5607808EBC00765
:1014280020208DF8000096F82E0003AA06EB800015
:1014380001A990F82050306902903068484401F0C2
:1014480065F9F86801994A4A0844A9F1640191428A
:101458002FD8B968411A21F07F41B1F5800F28D201
:1014680020F07F406060304684F80CA090F82E0091
:10147800EA46202D1CBF3F4901EB801B3CD005EB01
:10148800450008EBC0076068BA682146101A0002D8
:10149800C21700EB126007F1080600121BD470890E
:1014A80050B3488948B127E040F67331702002F004
:1014B80073F905B00120BDE8F08F2046FFF756FE0E
:1014C80001F008F93168081A0002C11700EB116031
:1014D8000012332810DA8AF80050397D207B8142C7
:1014E80005D80298606005B00220BDE8F08F0BEBCC
:1014F80045004578202DC2D1052001F0ABFC1B4CDE
:101508004FF0FF30A06094F82E309DF80020202185
:10151800202A13BF052004EB830090F82000FEF773
:10152800F7FF94F82E20134901EB821194F82F202D
:1015380001EB42014870206848442060012084F88B
:101548002B00607E012805D12069401E20F07F40D5
:1015580001F0D2FA9DF80000202803D00648407810
:1015680002F0EAF905B00020BDE8F08F4C0D00202C
:101578009C1FA107CC0C0020140000200246144B2D
:1015880010B508449A4204D940F21661702002F05E
:1015980003F9104A914204DD40F21761702002F00D
:1015A800FBF80D4A914204DA4FF4C361702002F04F
:1015B800F3F80A498142DEBF00F5F700A0F1F850C0
:1015C80010BD0028BCBFA0F5F70000F1F85010BD11
:1015D800FF7F841E0020A10700E05EF80080841EC3
:1015E800104A0B1A02F1010CB3EB9C0F3CBF1846D2
:1015F800704710B5441AB4EB9C0F3CBF184610BD99
:101608009A4203D2101A0844401C10BDA24204D2C8
:10161800511A0844401C404210BD40F60B3170205E
:1016280002F0BAF8FF7F841E074991F83020824201
:1016380004BF4868704700EB4000044901EBC00054
:101648000830FFF793BD00004C0D0020CC090020A6
:101658000E4910B591F82F00202812D091F82F00CC
:10166800A1F5607200EB400002EBC00091F82F106A
:10167800406801EB410152F83120BDE810400421D7
:10168800104740F6BB01702002F086F84C0D002090
:1016980070B56A4D6A49012605F5607408287DD23F
:1016A800DFE800F0046197A9C643AEB394F82C00B4
:1016B80018B901F0D3FE84F82C60E08A10B102F06A
:1016C80007F888B1FFF7BAFC84F82960A168B1F17E
:1016D800FF3F05D001230322052001F0F3FA40B1B2
:1016E800607E012810D109E040F66F01702002F0F9
:1016F80053F840F67401702002F04EF82069401E3D
:1017080020F07F4001F0F8F994F82F0094F82F109A
:1017180000EB400005EBC000406801EB410155F8C3
:101728003120BDE8704001211047FFF787FC4FF0DA
:10173800FF30A06094F8290080B194F82F0094F845
:101748002F1000EB400005EBC000406801EB4101A1
:1017580055F83120BDE870400621104740F6850154
:10176800702002F019F8FFF769FC84F8286001F08E
:10177800AFFF18B194F82C0028B108E040F69501A5
:10178800702002F009F801F069FE84F82C6094F8E2
:101798002D0068B14FF400202A4900E048E00860B5
:1017A800052001F057FB01F0A5FE002084F82D006C
:1017B80094F82F0094F82F1000EB400005EBC000C0
:1017C800406801EB410155F83120BDE87040002127
:1017D800104701F0F1FBE08A10B101F079FF28B160
:1017E80019480078032808BF667770BD4FF40A616E
:1017F800702001F0D1FF154806608868066070BD4A
:101808000878BDE8704002F097B8FFF717FC94F825
:101818002F0094F82F1000EB400005EBC000406843
:1018280001EB410155F83120BDE870400521104712
:1018380040F6B301702001F0AFFF0000CC09002092
:101848001400002008F5014016000020080500409B
:10185800034810B5407809F04BFC80B210BD000079
:10186800160000202DE9F34F8246D1488BB000685E
:10187800D04DC005C00D0ED0103840B20028B8BFFA
:1018880000F00F0000F1E020ACBF90F8000490F8E1
:10189800140D40090DD00C984FF0000B007800286B
:1018A80018BF012818D040F25C714FF0700001F0A9
:1018B80073FF95F82F004FF0010B202807D00C98E4
:1018C800007848B14FF4EB61702001F065FF40F2F9
:1018D8005571702001F060FFB74C24B1002140F22F
:1018E8005F70AFF30080B5490AEB4A0001EBC00016
:1018F8004FF00108009024B1002140F26770AFF367
:101908000080B8F1000F09D095F82E604FF000095B
:1019180085F82B90BBF1000F07D02EE0A8480028CF
:1019280018BFAFF3008062B6EEE73746012020EA21
:101938000706A448402200EB871100EB861009F047
:1019480045FD24B1002140F2DA50AFF3008005EBE9
:10195800870105EB8600096A016224B1002140F283
:10196800DE50AFF3008024B1002140F27170AFF374
:10197800008095F82B000028BDD124B1002140F249
:101988007B70AFF3008001F017F88046334606AA53
:101998000C99FFF77FFA24B1002140F28270AFF36F
:1019A8000080884906A801EB861717F81A10012944
:1019B80018BF02293ED10699079BA1EB0801824A6C
:1019C80021F07F41A3EB080323F07F4302296AD368
:1019D800B1F5800F67D29A4265D34FF0010901AB88
:1019E80005AA3146FEF746FF002864D09DF814107A
:1019F8009DF8042033468A4261D00520FEF788FD11
:101A08004FEA000107EB4A0041709DF814002028B6
:101A180003BF05EB860080F820A080F8239007EB31
:101A2800400018BF80F801A0324651465FF003001D
:101A3800FFF7D6FB05EB860090F8237024B1002150
:101A480040F28970AFF300806048002818BFAFF3F8
:101A58000080EFF3108872B624B1002140F28F7035
:101A6800AFF3008095F82B0000287FF444AF24B131
:101A7800002140F29770AFF300800DF1180E009826
:101A88009EE80E1000F10800B9F1000F80E80E1072
:101A980042D024B1002140F2A470AFF30080BBF122
:101AA800000F2BD115E0324651460420FFF798FB72
:101AB8004FF00109BEE7324651460420B8E7202915
:101AC80019BF07EB4100417805EB860090F820101C
:101AD80098E79FB195F82F0020280FD124B1002155
:101AE80040F2A970AFF3008031460220FFF7A8FB4F
:101AF80020B90C980078E8B3012849D024B1002116
:101B080040F2C670AFF3008085F82E60012085F89A
:101B18002B0000BF4FF0010924B1002140F2CF7023
:101B2800AFF30080B8F1000F3BD024B1002140F2A0
:101B3800D370AFF30080B9F1000F11D095F82E00E3
:101B480005EB800090F82100202809D024B100215D
:101B580040F2DA70AFF300801D48407801F0ECFEE7
:101B680024B1002140F2DF70AFF300800DB0484689
:101B7800BDE8F08FFFE724B1002140F2B170AFF368
:101B8800008095F82E2051460420FFF729FBC1E775
:101B9800002C3FF4B0AE002140F2BC70AFF30080DF
:101BA800A9E60748002818BFAFF3008062B6BCE773
:101BB80004ED00E04C0D002000000000CC090020DE
:101BC80000000000CC0C0020FFFF3F0000000000D8
:101BD800140000202DE9F14FA34886B00068C00525
:101BE800C00D11D0103840B20028B8BF00F00F0067
:101BF80000F1E020ACBF90F8000490F8140D400903
:101C080008BF4FF0010901D04FF00009069800788D
:101C180000284FF000001CBF07B0BDE8F08FDFF8C8
:101C28004CA2934D934C4FF0000B049025B100212A
:101C380040F26560AFF3008094F82E6084F82BB012
:101C48004FF0000825B1002140F26A60AFF3008030
:101C5800B9F1000F1DD13746012020EA0706864852
:101C6800402200EB871100EB861009F0AFFB25B18D
:101C7800002140F2DA50AFF3008004EB870104EB57
:101C88008600096A016225B1002140F2DE50AFF3F7
:101C9800008025B1002140F27260AFF3008000F0AF
:101CA8008BFE074633466A460699FFF7F3F825B1D7
:101CB80000214FF4CF60AFF3008094F82F00202864
:101CC80014D020690099091A0902CA1701EB126198
:101CD80009120BD5DDE90021891A20F07F4208445A
:101CE80020F07F40CDE900204FF001084DB10021E0
:101CF80040F28260AFF3008000214FF4D160AFF36F
:101D0800008000980199C01BC91B20F07F4021F07A
:101D18007F41B0F5800F05D28A4503D3B9F1000F92
:101D28000CD103E0B9F1000F38D094E033463A46BD
:101D380069465248FEF728FC48EA0008B8F1000F47
:101D480022D0009809F0D4F9BDF80A109DF80820AF
:101D58004B4B1144491C4218984241D8474881428C
:101D68005ADC404281425FDB581C9042DCBF02F5DE
:101D7800F702A2F1F85205DD002ABCBFA2F5F7026E
:101D880002F1F8520698C26001200490002D62D03A
:101D9800002140F29B60AFF300805CE0BDF80A00D0
:101DA80005AA04A900F0B2FC94F82F0020281CD042
:101DB8002069401D20F07F40DDE90021891A014497
:101DC80021F07F41CDE9000109F092F9BDF80A1030
:101DD8009DF808202A4B1144491C4218984218D9EA
:101DE80040F21661702001F0D7FCBDF80A0007F137
:101DF800090620B101F06CFC002808BF32362148E2
:101E080041780498814284BF081A064426F07F402E
:101E1800D2E71A48814204DD40F21761702001F0D0
:101E2800BBFC1948814204DA4FF4C361702001F009
:101E3800B3FC16489042DCBF02F5F702A2F1F85253
:101E480005DD002ABCBFA2F5F70202F1F852069898
:101E5800C2600120049094F82B0000287FF4E6AEBD
:101E6800049807B0BDE8F08F04ED00E0FFFF3F00E5
:101E7800000000004C0D0020CC0C00200020A10721
:101E8800FF7F841E1600002000E05EF80080841E9C
:101E98002DE9F14F804D8CB095F82E000020099067
:101EA80001207E4C4FF00008A5F18007834608907A
:101EB80024B1002140F2EE70AFF30080089890B38F
:101EC80085F82B8024B1002140F2F370AFF3008035
:101ED80095F82E9040222BEA090607EB861007EBAF
:101EE8008911824609F072FA24B1002140F2DA50D1
:101EF800AFF3008005EB860005EB89010090096AC5
:101F0800016224B1002140F2DE50AFF3008095F861
:101F18002B0080B1002C1CBF002140F2F970C7D003
:101F2800AFF30080C4E7FFE75D48002818BFAFF3B0
:101F3800008062B6C4E724B1002140F2FD70AFF31F
:101F480000800C981AF81000032878D1DDF800906A
:101F5800CDF818900C9999F82000884214BF4FF0DA
:101F6800000A4FF0010A09F1200C8646202207EBEF
:101F7800861303E0024603EB42004078884202D011
:101F880020280AD0F6E7202807D0864507D103EB9A
:101F98004E0040788CF8000007E040460CE003EB68
:101FA800400003EB42014078487024B1002140F220
:101FB8004450AFF30080584610EA0A0F18BF89F85A
:101FC80023B0E0B324B1002140F60200AFF3008053
:101FD800324601200C99FFF703F9069890F82390F0
:101FE80024B1002140F60D00AFF300802D480028F1
:101FF80018BFAFF30080EFF3108072B6089024B1D9
:10200800002140F61200AFF3008095F82B0038B19C
:10201800002C1CBF002140F616003FF449AF7FE7B3
:10202800B9F1000F08D095F82F00202804D13146C7
:102038000220FFF705F9F8B134B1002100E009E00A
:1020480040F62A00AFF3008085F82E6085F82BB0A3
:102058000120099024B1002140F63300AFF300803D
:10206800089888B124B1002140F63700AFF300800A
:1020780009980DB0BDE8F08F002CF1D0002140F692
:102088002500AFF30080E6E70548002818BFAFF346
:10209800008062B6E6E700004C0D0020000000005A
:1020A8000000000000000000202824BF0020704726
:1020B80000EB4000034B43F8301003EBC0004260D4
:1020C80001207047CC09002010B5202811D20E49F4
:1020D80091F82E30A1F1800202EB831C1CF810301D
:1020E8003BB191F82E3002EB831212F81020012A2E
:1020F80001D0002010BD91F82E2001460020FFF7E6
:102108006FF8012010BD00004C0D00202DE9F05F94
:102118007E4E804696F82E00A6F1800707EB8010C9
:1021280010F81800002865D096F82E90784D25B143
:10213800002140F6B930AFF3008007EB891414F89A
:102148001800012818D0C0B204281CBF052806288A
:1021580055D02DB14FF0000140F6C530AFF30080E7
:1021680001F040FC25B1002140F6C930AFF30080F2
:1021780014F818000128E6D1012425B100214FF4F4
:102188003D60AFF30080A4B3002086F82B0025B192
:10219800002140F6D530AFF3008096F82EB001202C
:1021A80020EA0B0907EB8B1107EB8910402209F095
:1021B8000DF925B1002140F2DA50AFF3008006EBAB
:1021C8008B0006EB890A006ACAF8200025B10021B5
:1021D80040F2DE50AFF3008096F82B00E0B1002DFE
:1021E8001CBF002140F6DB30C7D000BFAFF3008032
:1021F800C3E70AE04FF43B61702001F0CDFA4A468C
:1022080041460120FEF7ECFFACE74248002818BF22
:10221800AFF3008062B6B7E725B1002140F6DF30A2
:10222800AFF300809AF821300AF1210140461C469C
:102238004FF0200B07EB89120AF1220A04E0A346AB
:1022480002EB4B0C9CF80140844202D0202C2BD08E
:10225800F5E7202C28D0A34204D102EB43004078B4
:10226800087005E002EB440002EB4B01407848702F
:10227800BAF1000F11D025B1002140F23C50AFF364
:1022880000809AF80000A04207D125B1002140F251
:102298003F50AFF300808AF800B05DB1002140F2F2
:1022A8004450AFF3008000E025B1002140F6E33050
:1022B800AFF300801848002818BFAFF30080EFF391
:1022C800108472B696F82B0038B1002D1CBF00217F
:1022D80040F6E9303FF451AF88E786F82E900120A8
:1022E80086F82B0054B1002D08BFBDE8F09F0021EF
:1022F80040F6F630AFF30080BDE8F09F05480028AF
:1023080018BFAFF3008062B6EDE700004C0D002067
:1023180000000000000000000000000070B50D463D
:10232800064601F0C3F90F4890F82E2000248038A3
:1023380000EB821010F8141029B1611CCCB2202CCB
:10234800F8D3202070BD084804EB440140F8316000
:1023580000EBC100214645600120FEF741FF204601
:1023680070BD00004C0D0020CC0900202DE9F04F75
:1023780083B000F021FB054600F0D4FD634CA06853
:10238800B0F1FF3F1CBF4FF0FF30A060A07FDFF827
:1023980080B1A8B9D4E90301081A0002C11700EBFB
:1023A800116000124FF40C7108F0CFFE2169084447
:1023B800281A0002C11700EB11600012C00F0BD0E1
:1023C800607EE8B100F004FC94F82A00F0B140F215
:1023D8005441702001F0E0F994F82F0094F82F1080
:1023E80000EB40000BEBC000406801EB41015BF8DB
:1023F80031200821904740F24341702001F0CCF988
:10240800E81C20F07F4000F0DDFADDE74FF0010A1C
:1024180084F82AA094F82F00202824D094F82F803C
:10242800202084F82F0084F83000002684F82860E3
:1024380084F82960374826600078022816BF0328E8
:1024480001200020207794F82E7004EB870999F872
:102458002000202831D000EB40000BEBC000817D2C
:10246800012905D029E040F25741702001F094F984
:10247800AB4600F10805408A01AA694600F046F912
:1024880094F82F00202804D02069401D20F07F40B8
:102498000BE068890BF1090B28B101F019F9002844
:1024A80008BF0BF1320B2BF07F40D5E90021891AC8
:1024B8002860084420F07F40686039460120FEF714
:1024C800BFFE0028F9D0144800EB871010F8180058
:1024D800022804D13A4641460620FEF781FE84F8D8
:1024E8002BA099F82100202803D00C48407801F04F
:1024F80023FA207F002804BF03B0BDE8F08F00F066
:102508005BFD2677667703B0BDE8F08F4C0D0020A1
:10251800CC09002016000020CC0C0020140000205C
:1025280010B5304C82B094F82F10202908D0A1683B
:10253800B1F1FF3F09D040F6E821702001F02CF9F5
:1025480040F6E721702001F027F962680146264B22
:1025580050189A4204D940F21661702001F01CF913
:10256800224A914204DD40F21761702001F014F90B
:102578001F4A914204DA4FF4C361702001F00CF94C
:102588001C498142DCBF00F5F700A0F1F85005DDD9
:102598000028BCBFA0F5F70000F1F85001AA694671
:1025A80000F0B4F89DF804000F288CBF012000202B
:1025B8000099084420F07F41A16094F82900002880
:1025C80004BF02B010BD01230322052000F07AFBEE
:1025D80000281CBF02B010BD4FF42F61702001F01D
:1025E800DBF800004C0D0020FF7F841E0020A107AF
:1025F80000E05EF80080841E70B51E4C202184F82F
:10260800201084F8211084F82210002084F8230078
:1026180084F82E0084F82F10421EA2602060A07754
:1026280084F8280084F829002077607784F830102F
:10263800114984F82C0084F82D00087048704880EF
:10264800A4F182011022887001F8040F521EFAD1F9
:102658000A4D012684F82A60FF202870084801F0F6
:102668004DF9687001F0A8F9A86000F0EDFC84F855
:10267800316070BD4C0D00201600002014000020B1
:10268800A510000070B504461546084608F025FD5B
:102698000F4A011B02F1010CB1EB9C0F24BF231A56
:1026A800B3EB9C0F0BD38A4203D2111B0844411C85
:1026B80005E09A4207D2101A2044401C414201F119
:1026C8000F00281A70BD40F60B31702001F064F835
:1026D800FF7F841E410B48F2376251430A0C094BB5
:1026E800510202FB03020848504300F586306E3061
:1026F800400D5B4210FB03F3B2EB532F88BF491C1C
:1027080008447047F7C2FFFF6F0C0100430B48F203
:10271800376C03FB0CF330B41B0CDFF844C05C02CD
:1027280003FB0C030F4858434FEA505C04EB0C00C2
:1027380043F609541CFB04F404F5807C43F6085561
:10274800A3EB5C2C2C440CF0FF0CB3EB542F84BF90
:102758004FF0000C401C086082F800C030BC704785
:10276800F7C2FFFF6F0C01002DE9F041384CD4F897
:102778000403DFF8E08010F4803F4FF400664FF068
:10278800E0274FF000051CBFD4F84001002817D0FF
:10279800C4F84051C7F880622F480068D8F8001084
:1027A800A0EB010020F07F40022802D3B0F5800F93
:1027B80006D34FF48030C4F808030420FEF768FFFE
:1027C800D4F8040310F4003F1CBFD4F844010028D7
:1027D80017D0C4F84451C7F8806220480068D8F878
:1027E8000010A0EB010020F07F40022802D3B0F5D2
:1027F800800F06D34FF40030C4F808030520FEF715
:1028080047FFD4F8040310F4802F1ABFD4F8480106
:102818000028BDE8F081C4F84851C7F88062104824
:102828000068D8F80010A0EB010020F07F400228D3
:1028380004D3B0F5800F38BFBDE8F0814FF4802095
:10284800C4F80803BDE8F0410620FEF721BF0000E8
:1028580000B0004004B5004040B5004044B5004019
:1028680048B500402DE9F0413A4D287804286CD04D
:10287800E81C0122017859B1012908BF6A7002D009
:10288800697800295CD002210170407800F0E2FAF2
:10289800314CD4F804034FF0000810F4002F4FF423
:1028A80080764FF0E0271CBFD4F84C01002808D0F0
:1028B8004FF0030000F0CEFAC7F880620320FEF75D
:1028C800E7FED4F8040310F4802F1CBFD4F84801A5
:1028D800002808D04FF0020000F0BCFAC7F8806268
:1028E8000220FEF7D5FED4F8040310F4003F1CBF05
:1028F800D4F84401002808D04FF0010000F0AAFAEB
:10290800C7F880620120FEF7C3FED4F8040310F470
:10291800803F1ABFD4F840010028BDE8F0814FF08D
:10292800000000F097FAC7F8806204202870C5F804
:102938000880C4F80082BDE8F0410020FEF7A8BE78
:1029480040F266316C2000F027FFBDE8F041072017
:10295800FEF79EBE200000200080004001221302E6
:102968004FF0E0210020C1F8803101F5C071BFF3BC
:102978004F8FBFF36F8FC1F800310C494A60431E77
:10298800C1F808330A4B1860C1F840011B1D1860D4
:10299800C1F844011B1D1860C1F848011B1D1860CF
:1029A800C1F84C010A610349487070470080004033
:1029B8004085004020000020014800687047000062
:1029C80004B500402DE9F05F414E0446F71E96F825
:1029D80000C0F868BCF1010F04BFA042BDE8F09F39
:1029E8004FF040413B4A11603B496FF48023C1F8E6
:1029F80008333A4A4FF00005BCF1000F57D06FF486
:102A0800A023C1F848331560C1F84451D1F84821D2
:102A18004FF0E0294FF00108002A04BF4FF400628C
:102A2800C9F880224FF48033C1F80833C1F848331D
:102A3800C1F840512A4AD2F800A0A4EB0A0A2AF0A9
:102A48007F4BBBF1020F3CD34FF0020ABBF5800F5E
:102A580037D2C1F84045C1F84433BCF1000F05D066
:102A68001168411A21F07F410229F9D3C7F808807B
:102A78003D70FFF773FF1B480560001DC0F800A0FC
:102A88001949042008601949C1F80C80BA68C1F8CE
:102A980000228101C9F88012C9F80011144A4107BF
:102AA8001160FC60707086F80080BDE8F09FC1F886
:102AB8004833104B1D60C1F840511560C1F84451AE
:102AC800A4E7C1F8405540F2EF116C2000F064FE15
:102AD8002300002008F5014000B0004044B5004044
:102AE80004B5004004850040108500400080004087
:102AF80004F5014040B500402DE9F0412B4CE16858
:102B0800814214BF01220022DFF8A4C09CF80070A3
:102B1800022F02D0002A38D003E0002A08BFBDE8FF
:102B2800F081627882B3234B4FF080421A60224BC7
:102B38009513C3F80853C3F848530026C3F84061F7
:102B48001E4AD2F80080A0EB080828F07F48B8F1A8
:102B5800020F24D3B8F5800F21D2C3F84005C3F87B
:102B680044532FB11368CB1A23F07F43022BF9D3B8
:102B7800134B02214A071A60E06004208CF8010018
:102B88008CF80010BDE8F08104E040F2FD116C20E3
:102B980000F002FE40F201216C2000F0FDFDC3F8B8
:102BA800406540F20D216C2000F0F6FD2000002069
:102BB8002300002008F5014000B0004004B50040A3
:102BC80004F501400148C06870470000200000205B
:102BD8002DE9F04133486FF48024C0F80843DFF84A
:102BE800C8C0324A00219CF8003063B16FF4A024B9
:102BF800C0F848431160C0F8441100BFD0F848013C
:102C0800012280B909E0C0F84843294C2160C0F886
:102C180040111160C0F84411F0E74FF0E0244FF480
:102C28000060C4F88002022B04D040F219216C2005
:102C380000F0B2FD1F4E30681F4CC01C20F07F40D2
:102C4800E3681E4D98420BD03768DF1B27F07F479B
:102C5800042F05D3B7F5800F02D2FFF7B3FE1BE0B0
:102C68003068181A20F07F40022813D3B0F5800F7F
:102C780010D2134B4FF080401860A26021706A6038
:102C8800EA604000191F086004208CF801008CF8E5
:102C9800002001E0A2602170A068C5F80002BDE82C
:102CA800F081000000B000402300002044B500403F
:102CB80040B5004004B500402000002000800040DE
:102CC80008F501402DE9F047DFF874C101274FF0FE
:102CD80000089CF800509CF801C007287ED2DFE865
:102CE80000F0040404046A6A6A00564CE668B6F107
:102CF800807F04BF6478002C02D0022D05D03CE010
:102D08004FF413716C2000F047FD4FEA8C0404F176
:102D18008046ACF104042406A40D04F1804906F5AC
:102D2800004609F530490024012D02D0022D11D0AA
:102D380020E0BCF1040F05D2D6F840A1BAF1000F8B
:102D480018D104E0D9F840A1BAF1000F12D14FF020
:102D580000440FE0BCF1040F05D2D6F840A1BAF147
:102D6800000F07D104E0D9F840A1BAF1000F01D152
:102D780044F0804414F0804FD5D1334C00F1100C4E
:102D880007FA0CFCC4F808C38000204452B1076459
:102D9800D0F840658D1B25F07F45AA4298BFB5F550
:102DA800800F43D2C0F84015012B08BFC4F804C3F4
:102DB8000120BDE8F08735B1844504D140F26F2188
:102DC8006C2000F0E9FC001FC0B2012B0CBF0124ED
:102DD8000024032806D340F2491100E02BE06C20C0
:102DE80000F0DAFCDFF864C000F1100307FA03F31F
:102DF800CCF80833CCF8483380006044C0F84081F0
:102E08004AB1134D2E688D1B25F07F45AA4298BF05
:102E1800B5F5800F0AD2C0F84015002C18BFCCF8C1
:102E28000433CCF844330120BDE8F087C0F840856E
:102E38000020BDE8F0874FF41D716C2000F0ACFC59
:102E480023000020200000200080004000B0004047
:102E580004B50040F8B50127002407284CD2DFE864
:102E680000F00404040416161600264A00F11001A6
:102E780007FA01F1C2F8081381001144C1F840456E
:102E8800C1F84041204951F820000090F8BD1F4D7D
:102E9800011FCEB2297879B16A7882420CD11C4AD6
:102EA8004FF040401060012908BFFFF757FD2C7014
:102EB80018494FF08070C86006F1100007FA00F159
:102EC8001548C0F80813C0F84813B00000F1804056
:102ED80000F53040D0F84015104A1268891A21F0E0
:102EE8007F41022924BFC0F84045C0F840410C4842
:102EF80050F826000090F8BD40F2ED216C2000F05B
:102F08004BFC00000080004040810040230000206E
:102F180008F501402000002000B0004004B5004042
:102F280040B100401E496FF48023C1F808331D48A2
:102F38001D4A90F800C00020BCF1000F0AD06FF4C1
:102F4800A023C1F848331060C1F84401D1F84811F2
:102F580081B909E0C1F84833144B1860C1F8400141
:102F68001060C1F84401F1E74FF0E0224FF400612E
:102F7800C2F880120E494FF0FF32C1F808230D4AFB
:102F88001060C1F84001121D1060C1F84401121D03
:102F98001060C1F84801121D1060C1F84C0170475B
:102FA80000B000402300002044B5004040B5004078
:102FB8000080004040850040084890F90200002841
:102FC800B8BF704700F01F01012202FA01F1400961
:102FD800800000F1E020C0F80012704720000020B7
:102FE80010B507280DD2DFE800F004040404060633
:102FF8000600064902E0001F0549C0B201EB800047
:1030080010BD4FF426716C2000F0C6FB40810040D3
:1030180040B1004010B507280DD2DFE800F00404E5
:10302800040406060600064902E0001F0549C0B26E
:1030380001EB800010BD4FF426716C2000F0ACFB52
:103048004081004040B1004070B519480024042177
:103058000470C01E01708905C160FFF77FFC01255F
:103068004FF0E02CEB02CCF88031BFF34F8FBFF369
:103078006F8FCCF880320F4A556095600E48016812
:103088000029FCD1481EC2F80803C2F848030B48BF
:103098000460C2F84041001D0460C2F84441001DAC
:1030A8000460C2F84841CCF80031156070BD0000DA
:1030B8002300002000B0004004B5004040B50040A7
:1030C8002DE9F041164C607A002827D04FF4807122
:1030D8008D05284608F05DF880464FF48271284631
:1030E80008F057F800260746B8F1000F09D001206C
:1030F800C5F80803207920B12671E06908B1804736
:10310800E66137B1C5F804610220C5F8080300F08C
:103118008BFA4046BDE8F04100F05AB8BDE8F081AE
:103128003000002010B508F0DEF830B908F0FCF8DF
:1031380018B908F02FF9002802D0024902200860C7
:1031480010BD0000340C004070B500F087F900F0A5
:10315800BFFA094C4FF0804530B1FFF7E3FF01207B
:1031680028610420A07204E00320A0720120C5F8A1
:1031780004030020E07170BD3000002070B5134CCE
:10318800A079F0B1012803D0E179401E814218DA14
:1031980000F09EFA054600F06FFBA179012902D9DB
:1031A800E179491CE1710DB1616900E02169411AB9
:1031B800022902DA11F1020F07DC0DB1606100E0AB
:1031C8002061BDE87040FFF7BFBF70BD3000002030
:1031D8002DE9F04706464FF080454FF486712846A2
:1031E80007F0D7FF80464FF48871284607F0D1FFD3
:1031F800274C8246277804F1080008F03EF810B101
:103208004FF4D57116E04FF0010946B1A07A0328B2
:1032180005D10420A072FFF785FFC5F8109000269D
:10322800B8F1000F18D0C5F80C61A07A042804D0B2
:103238004FF4DE716D2000F0AFFA08F054F828B9A9
:1032480008F072F810B908F0A5F808B1114806603E
:103258000220A07200F0E6F8BAF1000F08D0C5F815
:103268001061A07A022801D1FFF788FFC5F81490F1
:103278003FB12670A07A022801D1FFF765FF00F060
:10328800D1F8BDE8F0470248083008F00DB8000052
:1032980030000020340C00402DE9F0475C4C4FF022
:1032A80000080646C4F81880437882780078E072EF
:1032B80063710127A271BD0784F80780052824D20D
:1032C800DFE800F00F03051F2100A76109E000F007
:1032D800C5F80121284607F061FF0028F9D002202F
:1032E800A06107F087FFB0B100F00CFA217E01F071
:1032F800030188420FD1B07950B10220C5F8040308
:103308006AE04448ECE74448EAE74FF44C7149E086
:1033180000F0CCF960E0EF604FF4827AC5F80481E0
:10332800A069C5F8180507F0CAFF40B907F0D1FF32
:1033380028B907F0E5FF10B907F0F6FF38B14FF0EC
:1033480080513648D1F84412C1F34231016007F088
:10335800B6FF40B907F0BDFF28B907F0D1FF10B993
:1033680007F0E2FF10B12D4810300760AF6002206F
:10337800C5F80403B07978BBD5F8040310F0020F40
:103388000ED0DFF89C90D9F80010C94341F300171C
:10339800D9F8001041F01001C9F800107F1C07E0AF
:1033A80040F2F1216D2000F0F7F900BF00F01AFBA0
:1033B8005146284607F0EDFE0028F7D000F076F9D0
:1033C8002FB9D9F8001021F01001C9F80010022017
:1033D800C5F80803C5F80481A07970B1307860B9E0
:1033E80000F076F9064600F047FA6FF0004216B191
:1033F800C4E9042001E0C4E904020121284607F0D9
:10340800CDFE08B100F05EF984F80A80BDE8F087C7
:103418003000002001000200010003003C050040CC
:1034280010ED00E010B5EFF3108472B60A48417849
:1034380029B14178491E4170417829B108E040F22C
:103448000D116D2000F0A8F9807808B900F04EF948
:10345800002C00D162B610BD3000002010B5EFF38B
:10346800108472B606484178491C4170407801289A
:1034780001D107F0AAFE002C00D162B610BD0000F1
:1034880030000020054810B5C17821B10021017134
:10349800C170FFF7C7FF002010BD000030000020FA
:1034A80070B50C4CE17861B90125E570E061FFF772
:1034B800D5FF00F00DF930B1E06910B18047002068
:1034C800E061002070BD4FF080402571C0F80453C2
:1034D800F7E7000030000020EFF3108072B60449CF
:1034E8008A78521C8A70002800D162B670470000A2
:1034F8003000002010B5EFF3108472B60A488178C6
:1035080029B18178491E8170417829B108E040F2DB
:1035180025116D2000F040F9807808B900F0E6F830
:10352800002C00D162B610BD300000202DE9F0411A
:1035380004006FF015003CD02178042939D80029FF
:10354800617838D0002934D1A178002931D1002000
:1035580007F0EAFD002007F0DAFD4FF080484FF051
:10356800FF31C8F808130026C8F80061C8F80461DC
:10357800C8F80C61C8F81061144F7E70A088B88133
:1035880007F01AFE012508B1FD707D700121404643
:1035980007F004FE08B100F095F82046FFF77CFE1E
:1035A8007D72002007F0B3FD4FF0E0213046C1F8EE
:1035B8000051BDE8F0810029FBD02029F9D8A17875
:1035C8002129F6D80129C2D1F3E7000030000020F4
:1035D80001488089704700003000002010B50D4870
:1035E80007F04BFE0B49083948B1012008704FF02D
:1035F800E021C1F80002BDE81040FFF72FBF887A2C
:10360800022801D1FFF7A0FDBDE81040014807F0EE
:103618004BBE0000380000200248807A002800D005
:103628000120704730000020F8B51F4DE87A0028C7
:103638000FD1287E00F0030007F0CCFD002808D049
:10364800EFF3108172B6FFF7E7FF18B1002900D138
:1036580062B6F8BD0126AE7201B962B618204FF005
:103668008044C4F80803A6614FF42070ADF8000048
:10367800BDF80000411EADF80010F9D20027C4F8CB
:103688000C71C4F810710848083007F009FE2F7053
:10369800FFF75AFD6661687900F07F00C4F83805C5
:1036A8001820C4F80403F8BD3000002010B5044CFD
:1036B800207E00F0030007F08DFD0028F8D010BD33
:1036C8003000002001490120087070479C0200204A
:1036D8004FF08040D0F8000118B90348007800285E
:1036E80000D00120704700009C0200204FF080406D
:1036F800012141600021C0F80011014801707047A4
:103708009C0200200248006800F003007047000097
:103718001C04004010B531B1012907D04FF44271A3
:1037280005A000F00FF8D0F8140401E0D0F8080460
:1037380000F0010010BD00006E72665F636C6F637D
:103748006B2E6800024A526802B11047FEE700007B
:1037580050000020064810B50021016001210160D9
:10376800084607F05EFDBDE81040012007F04CBD9B
:10377800FC1F0040074810B501214160891EC0F8B0
:1037880008130C2007F04DFDBDE810400C2007F091
:103798003BBD000000C00040FEB5104A5568E5B1C9
:1037A800002203466E460A2403E0B0FBF4F0521CE4
:1037B800D2B20028F9D1B0540AE000BFB3FBF4F04C
:1037C80004FB1030B3FBF4F3521ED2B23030B054C5
:1037D800002AF3D13046A847FEBDFEE7500000207E
:1037E80070B5174C06460D46607810B14FF0FF30A3
:1037F80070BD06B9134E62602570FFF7ABFFFFF787
:10380800B9FF3046FFF792FE0600F1D1FEF7F4FE4D
:10381800FFF70AFF07F0C8FB284607F0F5FC012070
:10382800002D09DB05F01F0100FA01F16A09920079
:1038380002F1E022C2F800116070304670BD00004D
:10384800500000204CB2000001484078704700004A
:1038580050000020074890F90000002809DB00F01C
:103868001F02012191404009800000F1E020C0F8CA
:1038780000127047500000202DE9F04101264FF05A
:10388800E02231034FF000084046C2F88011BFF330
:103898004F8FBFF36F8F164CC4F800010C2007F050
:1038A800DFFC144D2868C04340F30017286840F037
:1038B80010002860C4F8046326607F1C02E000BF83
:1038C80000F090F8D4F800010028F9D01FB9286852
:1038D80020F010002860084805686660C4F808638E
:1038E800C4F800810C2007F0BBFC2846BDE8F08135
:1038F80000C0004010ED00E008C5004010B50246C9
:1039080005200C4904E000BF01EBC0031B7933B16B
:10391800401EC0B2F8D24B216920FFF73DFF41F8A5
:10392800302001EBC00100224A718A7101220A711C
:1039380010BD0000800D002010B5052801D35A21C4
:1039480006E00A4901EBC0000179012903D05B2197
:103958006920FFF721FF41798279491CC9B28A425F
:1039680000D04171BDE81040FFF774BF800D002002
:1039780070B505250E4E0F4C16E0217806EBC100F8
:103988000279012A08D1427983799A4204D042798E
:10399800827156F8310080472078401CC0B22070F0
:1039A800052801D3002020706D1EEDB2E5D270BD50
:1039B800800D00209D02002000B507F080FC40B972
:1039C80007F087FC28B907F09BFC10B907F0ACFC9E
:1039D80008B1024800BD024800BD00000C050040C7
:1039E80000E7014010B507F09FFC30B3EFF31080FB
:1039F800C8B1002172B6124802680368C2F3001207
:103A080043F0100303604FF0E023D3F80042D3F8EB
:103A180004321C4300D040BF20BF00BF00BF00BF1E
:103A280000BF12B105E00121E4E7026822F01002AC
:103A38000260002900D062B610BD20BF10BD000092
:103A480010ED00E0A1B50000BDB50000ABB5000069
:103A5800B7B50000A5B500009FB500009DB50000F2
:103A6800C3B50000B1B5000097B500008FB50000E0
:103A780093B5000089B50000014800680068004758
:103A880058000020014800680069004758000020DD
:103A9800014A1268926810475800002001480068DF
:103AA800C068004758000020014A12685268104751
:103AB8005800002001490968096A08475800002091
:103AC80001480078704700009E0200201FB5174C7F
:103AD800A079022800D202208DF80100607903281D
:103AE80000D203208DF800002079ADF80400E078BA
:103AF800ADF80200684605F0EFFC08B1AE2110E011
:103B0800A068029002A805F0FDFC08B1B22108E007
:103B180007480068039003A80AF03CFA002803D07D
:103B2800B621032000F0CEF81FBD00006800002079
:103B3800743D000010B528B11422044907F046FC72
:103B4800002010BD6FF0150010BD0000A63D00005C
:103B580070B56FF02C05B0BB1D4CA07808B1A8114A
:103B680070BD21B36FF01500002AF9D008292AD2B8
:103B7800DFE801F02904070A0E11141E10782073DB
:103B880018E01078607315E01068C4F80F0011E0B1
:103B9800106860610EE01078A0730BE0217911B114
:103BA80011780229DCD30A4910780C31087301E036
:103BB80010886083064901220C31002007F0FFFCC1
:103BC800B0F5803F01DB284670BD0121E17070BD72
:103BD8005C00002038B50D46040020D0FDB100F08F
:103BE80013F9F8B12046FFF789FE104C002204F1C2
:103BF8000C012070284607F0E2FC0AF064FD002161
:103C0800207805F03BFE60788DF8000068460AF0E1
:103C1800B5F9FFF75BFF0120A070002038BD6FF0F9
:103C2800150038BD4FF0FF3038BD00005C000020A3
:103C380070B505000BD0FFF707FE4FF0FF3420B139
:103C4800FFF7C6FCB0F5FA7F04D9204670BD6FF0C7
:103C5800150070BD0022164B114600BF33F82140F5
:103C6800844203D303EB8100827803E0491CC9B284
:103C78000C29F3D30F4C10486270A56000F0D6F9F8
:103C88000020A070E0702071EFF3108472B60B482A
:103C98006FF00C0100F04CFD094800F00DFE18B162
:103CA800C421032000F00EF804B962B6002070BDEC
:103CB800763D00005C000020D53A000000C00040BE
:103CC8003D3E00000EB572B6154A9568D5B1002282
:103CD80003466E460A2403E0B0FBF4F0521CD2B24D
:103CE8000028F9D1B05409E0B3FBF4F004FB10301C
:103CF800B3FBF4F3521ED2B23030B054002AF3D1E1
:103D08003046A847BFF34F8F06480168064A01F4BA
:103D1800E06111430160BFF34F8F00BFFDE7000072
:103D28005C0000200CED00E00400FA05064810B520
:103D3800C1788078014302D04FF0FF3010BD05F004
:103D4800BDFD002010BD00005C000020064810B535
:103D5800C1788078014302D04FF0FF3010BD05F0E4
:103D6800BFFD002010BD00005C0000200100010024
:103D78000B0002000A00050009000A0008001400F0
:103D880007001E000600320005004B000400640016
:103D9800030096000200FA000100F40100003F470A
:103DA800708E81954E869DD3A29588F6300A7F53F2
:103DB80049FD0000054A10B5526812B1BDE810402F
:103DC800104783210420FFF77DFF0000A80D002085
:103DD800054A10B5126812B1BDE8104010477D21A0
:103DE8000420FFF76FFF0000A80D0020054A10B55A
:103DF800926812B1BDE81040104789210420FFF7EE
:103E080061FF0000A80D00200548016829B141683C
:103E180019B1806808B10120704700207047000080
:103E2800A80D002002490DC881E80D000020704748
:103E3800A80D0020F8B5124C0026256811E000985E
:103E4800022802D003280CD106E0206810B1002017
:103E5800266005E028210CE0206868B10120266072
:103E6800A847684600F0FAFC0028E8D0052805D0E5
:103E780035210420FFF726FF2D21FAE7F8BD0000C1
:103E8800780000207CB5214C0546207840B1A27806
:103E9800611C2846921C07F099FA0020207025E042
:103EA8001A48443805F06EFB002820D0174C443CD3
:103EB8002078112804D10A213E2007F01DFC18B1F2
:103EC8002078082806D00AE010492846443907F027
:103ED8001CFE0BE005213E2007F00EFC40B10B490B
:103EE8002846443907F066FC002800D001207CBD34
:103EF800A088ADF8000001A9684607F082FE0028F6
:103F0800F5D098210820FFF7DDFE0000880E00207C
:103F180070B50A7882703AB3012A25D81323037042
:103F280000230AE001EB430400EB4305A678EE709A
:103F38006488240A5B1C2C71DBB29342F2D3002301
:103F48000BE000BF01EB430500EB43042E796671DB
:103F5800AD882D0A5B1CA571DBB29342F2D3012117
:103F680001EB8200C0B270BD002070BD01210C4A77
:103F780040280CD2202803D8401E8140106802E057
:103F8800213881405068014207D100207047FF283E
:103F980003D0403881409068F5E701207047000061
:103FA8007C0000200121401E81400448C068014275
:103FB80001D0012070470020704700007C000020DD
:103FC80001490068C86070477C0000200449026805
:103FD800406842F48C220A60024A104348607047E5
:103FE8007C000020F807400201490068886070479B
:103FF8007C00002005484FF0FF310160C90C41608A
:10400800002181601F21C160704700007C000020F2
:1040180010B5FFF7EFFF0AF07DF804460248006884
:1040280000B18047204610BD8C000020014908607F
:10403800704700008C00002002210180418000218F
:1040480001713F21417147F24701C18001498160F7
:10405800002070478E81954E3EB50446694608F0AB
:104068001EF970B140F2122108E000BFBDF804004B
:10407800214600F0A9F820B140F217211720FFF7D8
:1040880021FE684600F050F80028EFD03EBD000041
:1040980010B5022804D340F26B111720FFF712FE67
:1040A8000149085C10BD0000B40D0020F8B50546B4
:1040B8000090914201D2144600E00C4655B1002709
:1040C800E81C20F00300A84206D040F23F11172058
:1040D800FFF7F8FD0127F3E7124E6846317072705A
:1040E800394600F0EDF8002003460099C91C21F07C
:1040F8000301009167B906EB8002D160002105E059
:10410800D2F80CC04CF82130491CC9B2A142F7D3EF
:104118000099401C01EB8401C0B200910228E4D34D
:10412800481BF8BDB40D002070B5044608F021F90D
:1041380008B1102070BD257800F0FEF802460C4842
:10414800618800EB85000EE0C36853F8213043B165
:104158004A1C6280A180C06850F82100A06000203D
:1041680070BD491C89B29142EED36180052070BDB3
:10417800B40D00202DE9F04121B1012902D0002021
:10418800BDE8F0810F4C00273B464FF6FF7604EB65
:10419800810514F801C00AE0DC19D5F80CE0A4B2D6
:1041A8005EF824E0BEF1000F04D05B1C9BB29C4576
:1041B800F2D8344604802046B442E0D0BDE8F0414D
:1041C80000F034B8B40D00202DE9F0410646A0F502
:1041D8007F400C4643F20207FF3820D0022C02D35E
:1041E8000720BDE8F081304600F05AF8050016D0E7
:1041F8000C48294650F82420304690470A480021A8
:1042080000EB8407F86840F82610204600F08AF88A
:1042180002462946786808F00FF80020E1E738469A
:10422800DFE7000060430000B40D00202DE9F041F5
:1042380090460D46074608F043F848B1164800EB8B
:104248008506F06850F8270028B140F2091115E0FA
:104258004FF4847112E0706800281AD0284600F0E4
:1042680061F80146706807F099FF040010D0F06803
:10427800022D40F8274004D34FF48A711720FFF726
:1042880021FD06484246214650F8253038469847D1
:104298002046BDE8F0810000B40D0020584300001E
:1042A80070B50C46054608F00BF8002805D0034801
:1042B80000EB8400C06850F8250070BDB40D0020E4
:1042C8002DE9F843164E8846054600242868C01C88
:1042D80020F003002860204600F024F8315D4843B0
:1042E800B8F1000F01D0002200E02A6801460092D0
:1042F80032B100274FEA0D0007F07DFF1FB106E03D
:1043080001270020F8E706EB8401009A4A60296833
:10431800641C0844E4B22860022CD7D3BDE8F883B3
:10432800B40D0020034931F810004FF6FC71C01C91
:1043380008407047544300000348017840788142A0
:1043480000D3084670470000B40D00201002E800B2
:10435800DDC20000DDC2000079D900001BCF0000DB
:104368002DE9FF4F264C804681B020689A46934637
:1043780058B1027A424503D9416851F8280040B142
:1043880043F2020005B0BDE8F08FA5211820FFF721
:1043980099FC1946029807F0B5FF86B258460E995F
:1043A80007F0A7FF85B27019001D87B22068A146E3
:1043B8003946006807F0F2FE04001FD067802580A8
:1043C8002946201D0E9D07465A460123009507F0F1
:1043D80044FE2088314638440123029ACDF800A0D3
:1043E80007F03BFE2088C119384607F067FED9F868
:1043F80000004168002041F82840C3E70420C1E7D5
:104408009000002070B5144C23688BB1197A814252
:1044180012D95A6852F8201071B1002542F820507C
:104428004A88186807F008FF216800200A7A0CE01B
:10443800C8211820FFF746FC43F2020070BD4B6804
:1044480053F8203033B9401CC0B28242F7D808680C
:1044580007F0E7FE002070BD900000202DE9F04134
:104468000D46040090464FF0000609D00027E01CD6
:1044780020F00300A04205D086211820FFF722FC77
:104488000127F4E7CDB11146002007F0B4FE0C3047
:1044980000EB85068FB90A4F04F10C00AA003C60B6
:1044A8002572606000EB850020600021606807F0DD
:1044B80007F84146386807F09EFE3046BDE8F081AF
:1044C8009000002070B5084D286800280AD0002404
:1044D80004E02046FFF796FF641CE4B22868007ADF
:1044E800A042F6D870BD000090000020094910B520
:1044F80002460968002049B10B7A934205D94968F8
:1045080051F82210002900D0081D10BDEE211820F6
:10451800FFF7D8FB900000200A4910B50246096849
:10452800002059B10B7A934207D9496851F82210F3
:10453800002902D031F8040B084410BDFC211820D2
:10454800FFF7C0FB9000002070B5064609480D46ED
:1045580000880AB1440800E084082146286807F06A
:104568001DFE00212A7964F31F41521C2A71C6E9F5
:10457800000170BD940000202DE9F84F8846050021
:104588000AD00027E91C002021F00301A94205D028
:104598002E210920FFF796FB0127F3E71D4900EBC1
:1045A800C80607B94D601F2A04D84FF6FF7000EA05
:1045B800820007E07C20B0EB420F01D2500000E0FF
:1045C8007C2080B24FF6FC72C01C1040002408808A
:1045D800A246894616E0A81900900FB1002000E015
:1045E8006846B9F8001007F006FE47B9D9F8041074
:1045F80001EBC40383F804A0009A41F83420641C3A
:104608000644E4B24445E6D3F61D26F00700BDE8AB
:10461800F88F000094000020064910B54A6802EBA4
:10462800C004002020710988204607F0E4FD2046D8
:1046380010BD000094000020094910B50748086023
:10464800084B112003EBC0040022C4F81025C4F85D
:104658001425401CC0B21428F4D310BD0000FEFF7E
:1046680008F5014000F0014070B520240021012325
:1046780020FA01F2D20720D04AB2002A10DB00BF8C
:104688004FEA52164FEA860602F01F0506F1E026A9
:1046980003FA05F5C6F88051BFF34F8FBFF36F8F4C
:1046A8000BDB02F01F054FEA52124FEA820202F1B9
:1046B800E02203FA05F5C2F8805201F10101A14296
:1046C800D6D370BD70B542004FF0000101D5144A31
:1046D8001160C0F38032C0F3C0339A4203D0642122
:1046E8001B20FFF7EFFA10F4404F14D00D4A0120B9
:1046F8005060831EC2F808330B4A9060C2F800125B
:10470800C2F80833094C2160251D28609060C2F862
:10471800083321602860BDE87040FFF78DBF0000B6
:1047280004E5014000E0004000F0004000F50040D2
:1047380070B50A4C0D462060FFF7C4FF2068FFF7EC
:1047480093FF00F077F8FFF777FF07F007FE28469A
:1047580000F0AAF8BDE8704000F0C2B89C00002044
:104768002DE9FC5F2F4E83463068019001272E48C3
:1047780006F083FDDFF8B08020B9002708F10100BA
:1047880006F092FD294C00254FF0030901206060D6
:10479800C4F80051C4F80451C6F800B02060DFF82E
:1047A80090A017E0DAF80000C00613D50E2007F035
:1047B800C6FDEFF31080009072B6C4F80493D4F8E5
:1047C800000120B9D4F8040108B9FFF70BF90098E3
:1047D80000B962B6D4F8000118B9D4F80401002869
:1047E800E0D0D4F804010028D0D137B10198306066
:1047F80008F1010006F041FD11E008F1010006F0A2
:104808003CFD0028BAD1C4F80893C4F80451C4F890
:1048180000510E2007F093FD034806F045FD0020E7
:10482800BDE8FC9F04E500409F02002000E0004036
:1048380010ED00E010B5084806F032FD08B124215B
:1048480006E00548401C06F02BFD002803D028216F
:104858001D20FFF737FA10BD9F02002070B51149DF
:104868000A68EAB100231D4601244A68521C4A60BE
:10487800092A00D34D600E7904FA06F20E68164232
:104888000BD0EFF3108372B60C6894430C6003B935
:1048980062B649680160002070BD5B1C092BE4D337
:1048A800052070BDA0000020024800210160416081
:1048B80070470000A000002010B5084C617809B1CD
:1048C8000F2010BDFFF71AF82070FF2801D0002034
:1048D80010BD76211F20FFF7F5F90000A800002081
:1048E8000149002048707047A80000200648074A80
:1048F800818C5288914204D190F8220008B100209E
:1049080070470120704700008A0F00208C020020A9
:1049180001494880704700008C0200200848094A75
:10492800818C5288914209D14FF6FF71818410F829
:10493800221F19B100210170012070470020704723
:104948008A0F00208C020020074810F8221F012936
:1049580007D0012101700548034900888884012097
:1049680070470020704700008A0F00208C0200204A
:104978000649074B8A8C5B889A4205D191F8222018
:1049880012B1016001207047002070478A0F002093
:104998008C02002009498A8CA2F57F43FF3B02D094
:1049A8000021016007E091F822200449012A02D081
:1049B8000160012070470020704700008A0F002026
:1049C80001490880704700008C020020054900203A
:1049D80081F822004FF6FF708884034908804880D8
:1049E800704700008A0F00208C02002005498A8C3D
:1049F800824205D1002081F822004FF6FF7088849A
:104A0800704700008A0F00200A4A10B1012807D019
:104A18000EE0507860B1D2F802000860D08804E057
:104A2800107828B1906808609089888001207047C4
:104A380000207047A1020020084A012338B101284C
:104A480004D113700868906088889081704753700B
:104A58000868C2F802008888D0807047A102002048
:104A6800064910B1012802D005E0487800E008782E
:104A780008B101207047002070470000A102002003
:104A88000149487470470000BA0900200148C078FD
:104A980070470000C40000200148007970470000FA
:104AA800C400002078B513494A7C0AB30A7C8DF803
:104AB8000020009A00929DF80020CAB1002301F15D
:104AC80010021A24A1F152050E7C8DF80060009E98
:104AD80000969DF800604EB1137043700470D5F8CD
:104AE8005A604660D5F85E608660EDE7012078BDC3
:104AF800002078BDBA09002010B5044600F046F938
:104B080018B1BD212720FFF7DDF80348012107F080
:104B180075FF0248C46210BD98090020C400002037
:104B28000149012088717047C40000202DE9F04731
:104B3800574D089C2E78002E6ED1002A6CD0002B81
:104B48006AD0002C68D005F11406C5E90E0186E884
:104B58001C000027AF716F71EF70AF702F71AF81BC
:104B6800EF8100F04BF9064600F042F9044605F0E3
:104B78003FFB05F017F894F9660005F0C1FB04F156
:104B8800100005F0ABFC04F10C0005F09BFC96F856
:104B9800230005F0BDFC05F13800406890F86C0171
:104BA80008B105F073FA94F86310012005F09EF936
:104BB800002866D0BA46012005F0A8FA354805F065
:104BC80011FA2088FFF7A8FC28632088FFF78EFCDD
:104BD80006F160016863DFF8C0908EC909F1080822
:104BE80088E88E00316FC9F82110716FC9F8251057
:104BF80000F076F90146208E07F001FDA18D814273
:104C080000D208462872A84694F86310E08EF77C14
:104C1800A58E082904D102E04FF48A7135E00421F9
:104C280007F0EDFC0FB9001D80B2854200D228467E
:104C3800C0B288F80900F27C02B104221044C0B264
:104C480088F80700B4F84C10091D814202D240F2DE
:104C5800A1111AE05546012000F046FB0F480068F4
:104C6800032810D00B280ED0484640F8525F456004
:104C78000948B188523041802188018096F8231074
:104C88000171BDE8F08740F2B1112720FFF71AF84B
:104C9800C40000201C550000680900205015004081
:104CA8002DE9F047054600F0A9F8334E0446706A2E
:104CB80047780DB1012D03D1716B06F0F5FC7070CA
:104CC80070784FF000084FF0010950B101281AD050
:104CD800022834D0032848D040F2F1312720FEF7CB
:104CE800F1FF012D32D000F0E7F839460122706B50
:104CF80007F048F828E000BF84F8088031E000BFDA
:104D080084F808902DE0012D08D000F0D5F8394638
:104D18000022706B07F036F8022D0BD0D4E916018B
:104D2800401C41F10001C4E91601207A012803D092
:104D380084F80890BDE8F08784F80880FAE7012D28
:104D480004D0706B07F024FA022DF3D0D4E91601D1
:104D5800401C41F10001C4E91601207A0128CFD195
:104D6800CAE7BDE8F04704F065BB012DE2D0706BDF
:104D780007F00EFAF5E70000C40000200248C089D9
:104D8800C0F3802070470000C40000200448007869
:104D980008B10C2070470349002048747047000090
:104DA800C4000020BA0900200C4810B5017849B1A8
:104DB80000F138010078022808D040F2CD112720F0
:104DC800FEF780FFBDE8104000F0A6B94868D0F8AB
:104DD8000001BDE8104005F00DB90000C400002036
:104DE800024A93890343938152691047C400002003
:104DF8000148406870470000FC00002001484068F6
:104E080068307047FC000020014A002152691047B1
:104E1800C400002070B5FFF7F1FF0446FFF7E8FF74
:104E28000546214607F060FCA97F012914D1002816
:104E380012D00A4842682888A2F8EE01607A82F8FF
:104E4800F001A07A82F8F10102F5F67201201070E3
:104E5800BDE8704004F0EEBA70BD0000FC00002010
:104E680070B50546012918D8124CA1698847A0B128
:104E7800607990B9E5B904F110000178C80605D445
:104E8800E06A0078C00601D4012000E00020A26A90
:104E98002AB962891AB1C90601D4012070BDA18955
:104EA8008A0703D5226AD278022A01D00843F4D1AE
:104EB800002070BDC400002010B5084CA06A38B1AD
:104EC8006289616AD21C06F081FAA06A606210BD2C
:104ED8004FF487612720FEF7F5FE0000C40000208C
:104EE80010B5FFF785FF0446FFF788FF0146427BB0
:104EF8001548242A0ED0897B24290BD01F2A0DD0CF
:104F0800202A0BD022290FD094F86200042800D15F
:104F1800082010BD406890F88E110EE0222903D0B9
:104F2800406890F8A80105E0416891F8A80191F857
:104F38005B10084007F06EFA014694F86200BDE87D
:104F4800104007F07FBA0000FC0000202DE9F8436C
:104F580088460646FFF752FF4A4C002705468DF85B
:104F680000702078022804D040F289412720FEF7FB
:104F7800A9FEA07B400606D44020FFF745FFE08944
:104F880040F04000E081E87CC6B304F083FE04F002
:104F980067FE68B9E87C58B1606A417841B1007829
:104FA800297AC0F3C000884202D10120A0704AE0EB
:104FB800606A4178618121B1606B07F0B6F8A06240
:104FC80000E0A762E08940F48070E081606AE979D6
:104FD8000078C0F38000884205D000F037F9E089F6
:104FE80040F48060E081606A297A0078C0F3C000EC
:104FF80088420ED1684600F0E5F80AE0FFE708B1FC
:1050080004F042FEE078401CE070E08940F4007053
:10501800E0811D4DB8F1000F04D1E1780120FFF7C0
:105028001FFFA0B19DF8000010B10020FFF738FE67
:1050380036B1E7706879401C6871FFF7EBFE02E053
:10504800A879401CA87100F067F8BDE8F8839DF8BE
:10505800000010B10120FFF723FE002000F08EF9B8
:105068009DF8000010B10220FFF71AFE36B1E77074
:105078006879401C6871FFF7CDFEE6E7A879401C07
:10508800A871E2E7C4000020BA0900202DE9F04128
:105098000E468046FFF7B2FE1E4D044628780128CA
:1050A80004D040F247412720FEF70CFE6078012724
:1050B80030B10020607001460420FFF791FEE770D0
:1050C800296A0878C043800709D1A079D0B902209D
:1050D800FFF786FE286A0078C043800712D0286A46
:1050E800407810B10220A07100E0A77136EA0806E6
:1050F80004D000210846FFF7B3FE28B1BDE8F0410F
:1051080000F00AB80320EEE7BDE8F041002000F007
:10511800EBB80000C400002010B504F053FE04F002
:1051280041FD0D4CE089FFF76FFEE2696179A078D7
:1051380090470A48407C58B10848523850F8521FE6
:1051480081604168C16005480121017404F072F969
:105158000020207010BD0000C4000020BA09002003
:10516800084810B50078022804D040F20121272011
:10517800FEF7A8FD04490120C871BDE81040FFF7FB
:10518800CBBF0000C4000020BA09002030B40C4B8B
:1051980042B9DA79FF2A05D190F8632090F8624085
:1051A800A2420BD031B1DA7990F8631030BC1046C6
:1051B80005F09CB9FF2290F86210F7E730BC704701
:1051C800C40000202DE9F0410746FFF717FE04460A
:1051D8001D4800260125416A0A7802F00302012AC7
:1051E80015D0022A13D0032A03D0417941F00401D3
:1051F80024E06570C28942F40062C2810120FFF791
:10520800EFFD1DE02672BDE8F0812572FBE74978C5
:10521800B1B1C28942F40062C281826A002AF2D026
:10522800FB2908D8807920B1BDE8F0412020FFF79C
:10523800EBBD3D70E7E7417941F010014171E2E7CC
:10524800207A0128E1D1DDE7C400002070B5FFF71E
:10525800D5FD0446807900282ED002280DD11C489F
:10526800006B06F068FD40B3D4E91401401C41F11D
:105278000001C4E9140104F0DDF80025A571E07807
:1052880020B1E57000211020FFF7AAFDA07870B1C9
:10529800A570FFF743FB98B100210820FFF7A0FD98
:1052A800D4E91401401C41F10001C4E91401E0797A
:1052B80001280AD00120E07170BD4FF4637101E04C
:1052C8004FF469712720FEF7FDFCE57170BD000001
:1052D800C400002003480078002801D0FFF71CBF55
:1052E80070470000C40000202DE9F0478146FFF711
:1052F8007FFD0646FFF782FD1D4C05464A46E06ADB
:10530800606201213046FFF741FFE87C4FF000085A
:10531800C0B1677A174804F0F9FF174801210176F0
:10532800D5E91612C0E90412124A616A04F02AFC8F
:1053380096F8630007F078F802463946012004F031
:105348004FFC04E0606A04F0E1FF04F02BFCB9F1C3
:10535800000F02D1404604F071FE002196F8623039
:105368000122084605F05CF802202070BDE8F087AD
:10537800C400002068080020700900202DE9FC47BF
:105388000446FFF73BFD0546FFF732FD0646DFF80A
:10539800789122460021FFF7F9FEA87901274FF0FE
:1053A8000008A9F1200440B101281FD0022830D0FC
:1053B80003283CD040F29E2158E0207A4821ADF8DD
:1053C800040088534846FFF7D3FA28B18020216AA1
:1053D800FFF706FDAF702EE06A4601A9206B07F0C3
:1053E8003BF8206210B195F8431011B1474820628C
:1053F80021E09DF8001031B9A0F8008080F8028003
:10540800012107F0FBFABDF80410206A07F0C4FA7E
:1054180011E0B6F84800ADF804006A4601A9206B0F
:1054280007F01AF8206230B940F28F211EE0484692
:10543800FFF79EFAC0B1206A0823017821F008011D
:105448000170EA7903EAC202114321F004010170F4
:105458002A7A042303EA8202114321F01001017021
:10546800C943890705D007E04FF426712720FEF7C6
:1054780029FCC07802280FD0206B06F081FD08B106
:1054880001210AE0206A0078C043800704D0FFF7B2
:105498002DFA80F0010100E00021206A027842EA3A
:1054A80001110170A97CD1B14178C1B1184804F04B
:1054B8002DFF1648283880F81880D5E91412C0E95D
:1054C80004121349226A04F05DFB96F8620006F0A4
:1054D800ABFF0246FB21002004F082FB03E004F04E
:1054E80015FF04F05FFB012296F863301146002097
:1054F80004F096FF2771206A018821828078A074C1
:105508002770BDE8FC870000E4000020980900200F
:105518006808002069510000554F000095500000B0
:10552800DD520000004870478311002004498A7842
:10553800824203D9084490F843017047002070471D
:10554800B00F002004498A78824203D901EB001089
:105558008330704700207047B00F0020054A01EBE8
:10556800410102EB41010268C1F80B218088A1F8D2
:105578000F017047B00F002004498A78824203D98E
:1055880001EB0010C01C704700207047B00F0020CE
:1055980010B540F2D3120021084805F091FF082207
:1055A800FF21074805F08CFF05480021001F017006
:1055B80041704FF46171418010BD0000B00F0020B0
:1055C800940200200B4B10B59C7884420FD91844E4
:1055D80090F8030103EBC00090F853310B70D0F83A
:1055E80054111160B0F858019080012010BD0020BE
:1055F80010BD0000B00F002007498A78824209D9FF
:10560800084490F8030101EBC00090F85A0100F03B
:105618000100704700207047B00F00200148408803
:10562800704700009002002005498A78824203D919
:10563800084490F83B0108B10020704701207047EA
:10564800B00F002070B50D46064600F0C3F8104CA8
:10565800102807D004EBC00191F85A11C90701D0EE
:10566800012070BD6178082910D2102808D004EBF9
:10567800C000012180F85A116078401C6070EFE783
:1056880001222946304600F089F8F5E7002070BD70
:10569800B00F002070B50B4D2878401E44B20AE0C8
:1056A80005EBC40090F85A01C00702D0E0B200F040
:1056B800D9F8641E64B2002CF2DA0349002048705D
:1056C80070BD0000B00F0020900200202DE9F041CD
:1056D80000242546184E29E006EBC50797F85A011D
:1056E800C00721D0284600F045F80346FFF744FFDD
:1056F80001460020102B09D0F21892F83BC1BCF1EA
:10570800010F02D092F84B2102B10120401E014244
:105718000AD10A4807F5AA7103552046641C97F870
:105728005321E4B204F0EEFF6D1CEDB23078A842CC
:10573800D2D8BDE8F0810000B00F0020940200200C
:1057480070B50A4B1B7873B1094B9C785CB145184E
:1057580021460AB1D81C01E0054883302A4604F0E6
:1057680033F9012070BD002070BD000090020020B8
:10577800B00F0020084910B5034600208A7806E0DB
:105788000C1894F803419C4204D0401CC0B28242D9
:10579800F6D8102010BD0000B00F002070B50C4BDB
:1057A80004461878451C1D70102803D3462128206C
:1057B800FEF788FA03EBC0030D68C3F854518988D3
:1057C800A3F8581183F8534183F85A2170BD00009B
:1057D800B00F00202DE9F0410F46064600240D4D7C
:1057E8000FE000BF05EBC40090F85311B14206D199
:1057F8000622394600F5AA7005F0D6FD38B1641CBA
:10580800E4B22878A042EDD81020BDE8F081204607
:10581800FBE70000B00F002070B50546FFF7AAFFB0
:1058280010281CD10E4C2078401EC0B22070A8420F
:1058380015D004EBC00204EBC50102F58070D2F864
:105848005321C1F85321D0F85700C1F857012078E7
:10585800FFF790FF102802D0204480F8035170BD54
:10586800B00F002005494A78521E4A7001EBC0016A
:10587800002281F85A21FFF7CFBF0000B00F0020A7
:10588800F0B56FF01F02010C02EA90261F25A1F562
:10589800AA4054380DD0A1F5AA40553809D0A1F531
:1058A8002850AA3805D0A1F52A40AA3801D00120ED
:1058B80000E00020002213464FEA020482EA0107B2
:1058C800FF431F437F1C0FD006F00107520842EA2E
:1058D800C73205F001075B0876086D08641C43EAC7
:1058E800C733162CEAD3F0BD0020F0BD2DE9F047F0
:1058F800044600F168054FF0010971B104F17E0713
:105908007E1E012921D0022946D003291BD1394600
:105918003046BDE8F04706F0B1BF4FF404720021ED
:1059280005F0CEFD04F040F844F62B11084085F848
:10593800159085F84C00000A85F84D00FE2085F882
:105948007C007F206872BDE8F0874FF00008A4F85B
:10595800068184F8FB80616814480A460844B0FB55
:10596800F1F0C4F8940040F6B830A4F898006389C0
:10597800284600F01DF83946304606F07FFF05F04E
:10598800EFFC18B1E068FFF77BFF10B184F86C8179
:10599800D9E784F86C91D6E74168B4F89A31D4F81D
:1059A80094212846BDE8F04700F002B87FC3C9013A
:1059B80030B500248486048F134D4C43B4FBF2F4B5
:1059C800048742F210746343B3FBF2F35B1C9BB28F
:1059D80003FB02F4C386AC4201D95B1EC3860B4BA2
:1059E80040F27124B3FBF2F35B1C8387038E63439D
:1059F80002EB03135B1EB3FBF2F3C362836A4B43F0
:105A0800B3FBF2F1816230BD0048E801005A62023E
:105A180070B590F8222090F82130012403FB012171
:105A28002522B1FBF2F302FB131100EBD10280F83F
:105A3800221001F00703927D04FA03F31A4203D0FF
:105A480080F82310002070BD90F82020B1FBF2F3FD
:105A580002FB1311491CC9B20023C518EA7E8A4209
:105A680011D395F81650002204FA02F6354201D0F7
:105A7800491EC9B221B1521CD2B2082AF4D304E09B
:105A880002EBC301DCE7891AC9B25B1CDBB2052B48
:105A9800E3D31F2070BD0000417841B1C0781928B8
:105AA80003D2044A105C884201D1012070470020CB
:105AB8007047000028E9000010B50122C1701929BB
:105AC80002D2064A525C06E0FF2904D04FF46E71F8
:105AD8002A20FEF7F7F8427010BD000028E9000000
:105AE8002DE9F0475FEA000906D0214D05F11000C5
:105AF800697B824619B10BE04FF4747105E000210F
:105B080007F07BF820B140F2D3312B20FEF7DAF80A
:105B18002E8A0020FEF7BCFA164FDFF85C80044698
:105B2800386858B1288AA04208D3001BC0B20121A6
:105B380006F0ABFB48B149463A6804E0D8F80020C3
:105B48001AB1288A4946904768B90021504607F09B
:105B580054F810B9288AB042E2D10848016829B13E
:105B68004846884710B10120BDE8F0870020FBE7D0
:105B7800C80D002040020020440200204C020020F2
:105B880070B505000C462ED0184802685AB328464E
:105B9800904740B32078112802D0142803D020E081
:105BA8002079F0B10AE0207920B1284607F00AFAF6
:105BB80020B116E00E490020487312E0E488002165
:105BC800204606F062FB60B1008806F0D7FB002192
:105BD8002046FEF7F9FA20B14FF49A712B20FEF710
:105BE80071F8012070BD002070BD00003C0200204B
:105BF800C80D00202DE9F34F87B00C4602A907987D
:105C080006F06DFC00287DD1DFF820914FF0010AE5
:105C18008046039890F8680000280CD0D9F8002036
:105C280062B121460798904740B1204600F01AF922
:105C38000028EED1012009B0BDE8F08F039D95F84A
:105C48002C01683550B995F824008DF804000198A6
:105C580001909DF8040008B1012000E0002083466F
:105C680095F84500C0B195F84600800714D584F82A
:105C7800018084F800A084F804800799A4F805102E
:105C880095F84710E171B5F848102181B5F84A1028
:105C9800618185F84580C8E70798FEF73DFC070055
:105CA8000DD006F000F9060015D084F801800D200B
:105CB80020700798E080268184F804A007E040F26D
:105CC8003A212DE0002138460A4606F0FAF9761EF8
:105CD800B6B2F7D2A9E70798FEF708FCF0B1BBF116
:105CE800000F20D006F017F860B1079806F046FBC1
:105CF80000210798FEF768FA84F801800A214046D7
:105D0800217000E00FE084F804800799A4F80510DA
:105D180095F82510E1712435287086E74FF416713F
:105D28002B20FDF7CFFF002085E700004802002068
:105D38002DE9F041124C07460E46E07D10B1208B4C
:105D4800002812D00E480E30804606F000FFA8B991
:105D5800E589E0893246394606F008FF38B1E07D2A
:105D680010B1208B401E20830120BDE8F081404601
:105D780006F0EDFE10B9E089A842EAD10020F4E768
:105D8800C80D002010B5017919B1012906D00020ED
:105D980010BD428883680088022103E04288836836
:105DA8000088012100F008F810B9024901200870A4
:105DB800012010BDC80D00202DE9FF478A469946ED
:105DC8001546044601A906F08AFBE0BB029F4FF086
:105DD800000868378DB12046FEF79EFB04000FD0FF
:105DE800294606F09FF8060003D01D488088A8427F
:105DF80008D2002004B0BDE8F0870120387529E0FA
:105E080089212AE02046314603AA06F084F803983F
:105E1800A0F8008080F80280397D09B14FF0020AAD
:105E2800514606F0EBFD3146032620464A462B46EE
:105E3800009605F059FF2046294606F010F858B19B
:105E4800444601A800E005E006F084FE0298A0F8A8
:105E5800F2403C750120CDE79F212B20FDF732FF52
:105E6800C80D002010B52C4986B08A7D0178D3076B
:105E780001D1192904D018291ED0122945D049E08A
:105E88008088ADF8000002A906F029FB08B1582166
:105E980035E0039810F85E1F8DF8021041788DF8F0
:105EA80003104088ADF804000221684608F058F94C
:105EB80040B340F24D1122E091072BD4848803A906
:105EC800204607F0E0FF10B14FF4AA7117E0ADF8D3
:105ED8000040BDF81200ADF80200BDF81400ADF89E
:105EE8000400BDF80E00ADF80600BDF81000ADF8CE
:105EF8000800684608F056F820B140F25D112B20E2
:105F0800FDF7E0FE012006B010BD510702D4807BEA
:105F1800C007F7D00020F6E7C80D002070B504468A
:105F2800007C00B302281ED05FF0010004F1490193
:105F380084F848000D46C0B1E07DF0B1D4F81100F6
:105F4800C4F84900B4F81500A4F84D00207C06F008
:105F5800A7FF20760820607694F84800294606F0C6
:105F68008BFFA8B90EE00020E0E70020FEF74CFD0B
:105F78000028EBD140F27F4101E040F283412D201F
:105F8800FDF7A0FE94F84800294606F07EFF00B110
:105F98000120A076207E10B9A078400706D594F895
:105FA8004F0004F1500106F066FA6076002525647A
:105FB80005F08CF860640021204607F0BFF884F8EB
:105FC8005650A078400708D5207E002805D02046E6
:105FD800BDE87040002100F0CDBD70BD08B590F857
:105FE800A8208DF80020009A00929DF80030002229
:105FF80063B14A7017230B7050F8A93F4B60436890
:106008008B60037A0B7300F8012C3BE090F8A23008
:106018008DF80030009B00939DF8003043B14A7022
:1060280005230B70D0F8A4304B6080F8A22029E03B
:1060380090F878308DF80030009B00939DF8003080
:106048001BB100BF07F051F81CE090F89A308DF8AA
:106058000030009B00939DF80030ABB190F8783089
:106068008DF80030009B00939DF80030002BE9D19B
:106078004A7014230B7050F89C3F4B6083880B8147
:1060880000F8022C012008BD002008BD30B50C46E0
:106098008DB005460146202202A805F097F90AA806
:1060A80007F0F9F8A07A8DF8180020788DF8080024
:1060B800B4F80100ADF800009DF8000000F00101FF
:1060C800C0F3400241EA4201C0F3800241EA820182
:1060D800C0F3C00241EAC201C0F3001241EA021152
:1060E800C0F3401241EA4211C0F3801041EA801027
:1060F800ADF80A00207D012806D0022804D040F21D
:1061080085210620FDF7DEFD8DF80C00617A0AA8CE
:1061180007F0A8F8207D0121022802D1607D401CEB
:10612800C1B2A07E401CC2B20AA807F062F8BDF84E
:106138000A00000701D5002020E00AA807F06BF844
:10614800BDF80A10282200F0BDFD40F2712100F2CE
:10615800D520B0FBF1F04843D4F8021040F2712387
:106168000A0A40F271214A43D4F80510090A594332
:10617800904201D8049204E0884201D8049000E0DB
:106188000491A07C8DF81700207E012800D0002003
:106198008DF8140095F8740095F87500202202A96E
:1061A800284605F013F90A982862BDF82C00A8843F
:1061B800E07A68B102280BD05FF0010085F84F0043
:1061C800E0682865208AA5F854000DB0002030BD8D
:1061D8000020F3E70A4A10B500211170094C6060ED
:1061E80000F022F810B14FF4487104E0A0680028CC
:1061F80004D140F223312D20FDF764FD10BD0000CD
:10620800E40D00200401002002490148886070471D
:10621800B46C00000401002002490860896809681C
:106228000847000004010020084810B5017811B1A2
:106238000C24204610BD0024046044608460C460BF
:1062480003F096FD03F0D8FBF3E70000E40D00200F
:10625800044910B50978012901D100F077FB002025
:1062680010BD0000E40D0020024901480860704795
:10627800A16A0000100100202DE9F0410F0004463A
:1062880023D004F12000054606F0EEFFB0B9A0784F
:10629800C0F3C00050B3284606F0BDFF06462846A6
:1062A80006F0E2FF301AC0B207F033F8014635486D
:1062B800426811444160284606F0F4FF284606F07B
:1062C800B6FF0146204606F075FF2F4D94F856603C
:1062D80000216868018006F083FF6088132813D0C6
:1062E80009DC102836D0122809D131E02046BDE853
:1062F800F04100F02BBB15280FD01D280DD040F21F
:1063080096612D20FDF7DEFC0021686806F0D8FBB9
:106318000121686806F064FF20E00121686806F042
:10632800CFFB0121686806F05BFF36B104F1570125
:10633800686806F0E0FB012106E004F15001686896
:1063480006F0D9FB94F84F10686806F0DAFB05E010
:10635800062100E00221686806F0B2FB204600F042
:106368007FFC60881D2806D0152804D0A28E216BDA
:10637800686806F095FB39462046BDE8F04100F014
:10638800E5B90000E40D0020040100202DE9F041EA
:10639800284D80462878022805D02878032802D07E
:1063A80040F691411FE0244C2068017B09B106F0BA
:1063B8000CFF60680027B8F1000F007800F00F06A6
:1063C8001FD003F0E3FEE0B13946606806F02EFB0B
:1063D800B8B12A7820683146022A07D02A78032AD9
:1063E80004D040F66A412D20FDF76CFCA2682B789A
:1063F80052696FF0070606EB8303D25890470646AA
:1064080000E00126A87B18B103F0B2FC03F0F4FA0F
:10641800002E0DD0206806F092FF20B1A068806899
:10642800BDE8F04100472068BDE8F04100F08EBAB1
:10643800BDE8F081E40D00200401002010B5032917
:1064480002D005290AD102E000F05AFB03E0044912
:10645800096809B1884708B1002010BD012010BDA6
:1064680010010020094A0300106801D000F06EBA3C
:10647800002909D09168064A096912786FF00F035C
:1064880003EB820289580847704700000401002086
:10649800E40D002070B5044640880025102814D06B
:1064A800144EB07B20B103F0C7FA402003F070FC13
:1064B8001148406803F02AFFA078400713D4E07B16
:1064C800012808D0032806D006E02046BDE8704021
:1064D8000121FFF7D1BE1025002145F00E022379D6
:1064E800084603F09DFF002003F0A8FD022030704D
:1064F80070BD0000E40D00200401002010B5124C0E
:10650800206800F025F8206806F019FF00282068A8
:106518000BD00E490A78022A0BD00A78032A08D031
:1065280040F6A5312D20FDF7CDFBBDE8104000F069
:106538000DBAA2680978D2686FF0070303EB8101EE
:106548005158BDE81040084704010020E40D002020
:1065580010B5017B09B106F038FE0548807B00289C
:1065680005D003F005FCBDE8104003F045BA10BDA6
:10657800E40D00202DE9FF5F5A4D04462878E8BB5A
:106588002078FF2849D04FF00009A5F80C90C5F8ED
:10659800049085F8019085F8029084F86190484647
:1065A80003F0B4FD504BDFF844A10FCB8DE80F008A
:1065B800DAF8080040680390684603F013FD03F01A
:1065C80017FE03F0D5FB03F017FA4748401F03F006
:1065D80079FF4548083803F081FF04F1200006469A
:1065E80006F060FE304606F022FE0146204606F020
:1065F800E1FD94F90E0003F083FE00E00DE021793F
:10660800002003F073FC0126A86050B10F2105207B
:1066180003F0D2FBA07E58B905E00C2004B0BDE819
:10662800F09F2E705BE0207E10B9A07840072BD534
:1066380004F04CFD83465946606CFAF7D1FFDFF849
:10664800B080074690FBF8F108FB117041425846AC
:10665800FAF794FF606497FBF8F0216C0844206413
:10666800FEF7DCFF216C88420ED8C4E9109B01219B
:10667800204606F063FDA078400705D5207E18B1B6
:106688000121204600F076FA94F8481004F14900F8
:1066980003F00CFF94F8740002280AD12246D2E9CC
:1066A8001937D4E90C01C4E90C37C4E9190184F895
:1066B800746094F87500022809D1D4E90E10D4E961
:1066C8001B23C4E91B10C4E90E2384F87560FEF788
:1066D800FDFF0321DAF8040005F0C0FEA8730020CE
:1066E8009CE70000E40D0020946C000004010020E9
:1066F80040420F0010B50446FFF73CFF002808D1C0
:1067080004480078012803D000212046FFF7B4FD93
:10671800002010BDE40D00200A4810B50A4904689D
:10672800087800280DD00878022802D008780328B5
:1067380002D12046FFF70CFF2046BDE8104000F0CC
:1067480005B910BD04010020E40D00202DE9F04139
:10675800044627480D46406803F0D8FD254E04201E
:10676800307025B3608810282AD004F120008046B4
:10677800B56806F050FD0746404606F075FD381A24
:10678800401EC0B26188282200F0BCFA0544A078F7
:10679800C0F3C00030B17068054406F0BEFD28445F
:1067A800C4F8C40022792946002003F0BDFD6088A2
:1067B800132813D009DC102818D0122809D10DE0AD
:1067C8002179002003F046FBF1E7152806D01D28A3
:1067D80004D040F61C512D20FDF774FA2379BDE84A
:1067E800F04101221146002003F01ABEBDE8F081F5
:1067F80004010020E40D002010B5044600780B4683
:1068080084F8A900FF2910D004F1AB02511E1846E4
:10681800FEF7D8FE30B194F8AA0040F0020084F8E0
:10682800AA0011E040F62C711DE01048406801787C
:10683800C1F3801184F8AA10D0F80310C4F8AB1083
:10684800B0F80700A4F8AF0094F926007F2808D014
:1068580084F8B1007F2084F8260092340120A075C6
:1068680010BD40F6CE512D20FDF72CFA0401002072
:106878002DE9F0470446408817468846032906D084
:1068880000F0010594F8600018B1012002E0C0F39F
:1068980040050020814603F089FA0646B8F1030F47
:1068A80025D00120804635EA090546D02548807B59
:1068B80038B105F0D6FD3870FF2802D0FEF79CFEEF
:1068C8000643214D94F84F2068680178C1F3801180
:1068D800914206D1062204F15001C01C04F064FD67
:1068E80038B100203978FF2909D0B8B903E002206F
:1068F800D8E70120F6E7607E88420FD008E038B17B
:10690800696811F8030BC0F3801006F0D5FB28B1B5
:106918000020A178490703D590B90EE00120F8E7D7
:1069280076B9E07B08B1404507D1696811F8030BD7
:10693800C0F3801006F0C0FB10B10020BDE8F0875E
:106948000120FBE7E40D00200401002070B5044697
:10695800806A104D401CA062A87B002620B103F07D
:1069680007FA03F049F8AE732E7094F8610008B185
:1069780001210AE0607B38B1A16A884204D801216C
:10698800204606F0F1FC70BD00212046BDE87040AD
:1069980006F0EABCE40D00202DE9F843044690F81F
:1069A800780090460D468DF80000009800909DF8FC
:1069B800000010B140F6D93158E084F87A302888C0
:1069C800A4F87C00002B63D1686805F099FDA4F851
:1069D80092002889A4F894006889A4F8960095F88C
:1069E8006D0184F89800217E04F14906002704F11E
:1069F800800929B194F84800314606F046FA40B9B2
:106A080094F8620070B194F84800314606F034FA00
:106A180040B1D4F84900C4F88600B4F84D00A4F891
:106A28008A0003E0C4F88670A4F88A701948B8F19F
:106A3800FF0F40680178C1F3801184F87F1050F887
:106A4800031F16D0C4F88C108088A4F890004A461A
:106A580004F17F014046FEF7B5FD28B114F87F0F19
:106A680040F0020020700CE040F6FA312D20FDF7CE
:106A780029F9C4F880108088A4F8840044F88C7F31
:106A8800A7802888FDF732FDBDE8F84305F0D3BAA2
:106A9800BDE8F8830401002038B50446FF208DF8CE
:106AA800000001256A4605212046FFF7E1FE00B3F4
:106AB800114AE069526810F87D1F1278C2F340123B
:106AC8001140017001222046E16900F081F800239D
:106AD8009DF800202046E169FFF75EFF012084F859
:106AE8007800064A0021E0691170052100F01AFAC1
:106AF80000E00025284638BD04010020E40D0020F0
:106B08007CB50446FF208DF8000001256A46032164
:106B18002046FFF7ADFE28B3207B68B194F8A800A3
:106B28008DF80400019801909DF8040020B99DF8A3
:106B380000102046FFF760FE0C4E002170680180AF
:106B4800042105F0BDFF204600F08AF8A28FA16B52
:106B5800706805F0ECFF064905200870706803F0BE
:106B6800D5FB00E0002528467CBD0000040100207C
:106B7800E40D002070B504460E46407EFEF7FCFC8E
:106B8800050019D0102105F0F2FD002814D10120CC
:106B980084F8560004F1570132460C46284605F0A1
:106BA80002FC2146054C606805F0A5FF6068BDE859
:106BB8007040012105F0A5BF70BD00000401002050
:106BC800024801210068FFF757BB000004010020BC
:106BD8002DE9F041214E80460C467068154650F864
:106BE8000F1FE160818821828179A174408905F0B5
:106BF80083FC0746606070683946807D05F0B2FD09
:106C0800A08270683946B0F8170005F0A7FDA061AA
:106C1800706830F81B1F2181418861814168C4F880
:106C28007E10017A84F88210417A01F01F0184F8FD
:106C38008910407A400984F86D0104F15A00012155
:106C48000572457281720021363806F0ABF898F863
:106C58000E0084F86600BDE8F08100000401002001
:106C680070B5074D044600F14901686805F050FF0A
:106C780094F848106868BDE8704005F04FBF000000
:106C880004010020555555D6BE898E0005650000C3
:106C9800956300006D64000000000000456400007A
:106CA8009D640000E7D00000EDD00000FD66000004
:106CB80021670000C96B0000B06C0000A86C0000E0
:106CC800A46C000010B5421E022A01D9CA2109E0AD
:106CD800401E102909D012290CD013290AD01529D1
:106CE80005D0D8212F20FCF7EDFF054904E0044921
:106CF800891D01E00249891F31F8100010BD00000C
:106D08003AD30000421E10B5D2B2012A03D91D2978
:106D180001D0EE210DE0132913D004DC10290BD08B
:106D2800122904D10DE0152908D01D290ED04FF4E1
:106D380081712F20FCF7C6FF074804E00648083099
:106D480001E00548001D30F8120010BD40F25A312C
:106D580010FB01F010BD000028D300002DE9F04120
:106D6800044690F8C80015460F4600285DD1214614
:106D78004448FBF7D3FA0646202856D0342200218F
:106D880004F1B40004F09CFB84F8B4600126C4F854
:106D9800B87084F8C8605FB1012107F58E70FDF7FF
:106DA80025F897F81C0100F00700401C87F81C0123
:106DB800204606F063FCA4F8D400032084F8D6002B
:106DC80084F8D760002704F8CC7FFAF741FD2189C1
:106DD800CC3C884200D8084600F2BF601FFA80F811
:106DE800204606F0EFF818B32748007800F0E4F8DA
:106DF80000F5CD6081B2284604F0A7F92844C4F80C
:106E0800D000B83404F062F94146FAF7B7FB2062C3
:106E180004F8037C2671012006F07BFA00F20710C3
:106E2800281AA762A060B83C17E00C20BDE8F081E2
:106E3800204606F0D1FB44F8D00F04F81B6C04F090
:106E480045F90646002006F0C8FC00EB080130466C
:106E5800FAF794FB2561A060D03C04F1CC0194F8CA
:106E6800B40006F009FC38B1A4F8DC700021204613
:106E780006F008F90020D9E74FF4FD713020FCF73F
:106E880021FF000079760000140100200448012148
:106E9800002201704270C170827006F0A7BA00002B
:106EA80014010020014908707047000014010020F7
:106EB80001494870704700001401002005494FF44B
:106EC8007A72B1FBF2F110B501F28B2105F083FF64
:106ED80080B210BD7D5201002DE9F041104CD4E97B
:106EE800015703F019F90646607828B13246394649
:106EF800284605F00BFB05466068854205D0E16829
:106F0800281A0844E060FBF70BFB6560AE4201D825
:106F1800A07810B10020BDE8F0810120FBE7000057
:106F28001401002070B5224C054606293CD2DFE842
:106F380001F0050B030E0F25002100E00121284672
:106F4800BDE8704000F04CB9032085F82C0170BDF5
:106F580003F016F9C5F8680195F8630007F032FCEC
:106F6800D5F86811081A616801446160A16808448D
:106F7800A0602846BDE8704000F0D2B803F0CCF815
:106F880001460022A06906F0DDFBA0690949D0F896
:106F9800B82090F8B400FBF787F80028D7D140F262
:106FA8007A713020FCF78EFE40F29171F9E700000B
:106FB800140100200DD8000010B50C2804D34FF49C
:106FC80040710620FCF77EFE014931F8100010BD23
:106FD800EED80000FEB5184C0120A0704FF6FF75E2
:106FE8000BE0002105F051F9060010D096F8600179
:106FF800FBF78CF8304606F098FB6946002005F050
:107008004EF980B140F211113020FCF75BFE40F2DE
:107018003111F9E7029830B190F82C1119B10088B4
:10702800A842DED104E06846FDF77EF80028F1D0DA
:107038000020A070FEBD0000140100202DE9F047DB
:10704800044636481E469046C0788946002568B3EF
:10705800FCF7E2FA50B3B4F81801022826D394F8E2
:107068002C01022822D094F84201F8B994F86D0155
:10707800FFF7A2FF00F5C86081B2318094F82C01B7
:107088000027012815D0606804F05FF8B4F80621DD
:1070980080B24244A2EB0901D4F83421C4F8340187
:1070A800821A01FB0275012084F842012846BDE8D6
:1070B800F08794F8790003282CD00121002005F0EE
:1070C800D1FAA1694718D4F824013188C83404F0EA
:1070D8003CF8A26D216E821A01FB0255A065318829
:1070E800384604F032F8A16EA066411A0D44318882
:1070F80054F8C40C04F029F8E28F4244A2EB0901C9
:10710800226E891AE26E491E821A01FB0255E06658
:10711800C83CC8E7D4F82401D3E7000014010020D4
:107128002DE9F047044690F84201002853D094F81E
:107138002C0103284FD1294894F863900078FFF771
:107148003BFF054694F86D01FFF736FF284486B2E9
:1071580094F86D01FFF730FF00F5C8601FFA80F85A
:10716800484607F02FFBD4F868110D1A484607F077
:1071780037FB4FF47A7A00F2E730B0FBFAF02D1AB9
:10718800484607F01FFBD4F800110F1A484607F0CD
:1071980027FB4AF2A1310144B1FBFAF0391AA1F1F7
:1071A80060007043B0FBF8F2292000EB5100603218
:1071B800A0EB520100EB5200A94201D8854201D947
:1071C800FCF70CFA3146606803F0BFFF0021C4F8F1
:1071D800340184F84211BDE8F08700001401002052
:1071E800F8B50E46044602F097FF0025C4F864017E
:1071F800012E02D10F48807868B1042084F82C0150
:1072080006F021FAA4F85E51B4F86C00A4F83E0127
:1072180084F84151F8BD0095B4F8F4100123002218
:10722800204600F009F80028EAD040F2E261302058
:10723800FCF748FD140100202DE9FF4F044685B0F6
:1072480090F86300DFF824B4CDE9003099460F4682
:107258009BF80000FFF7B0FE054694F86D01FFF7B4
:10726800ABFE2844ADF8080094F876000D2804D049
:1072780000200390079810B12EE00120F9E794F858
:107288002C01032828D1039830B3B4F88C01B842F4
:1072980022D1D4F83401C4F820016068C4F824016C
:1072A800B4F85E01B4F806110844C4F82801204671
:1072B80006F02FFBD4F89001A061B4F88E01A082EB
:1072C800D4F894016060B4F898012081B4F89A0168
:1072D8006081022084F82C01B4F86C0004F5A275D2
:1072E800381A0FFA80FAB4F85C01381A0FFA80F8E5
:1072F800B8F1000F06DAD4F85401C4F85801012097
:10730800D046009002AB524641462046FFF796FE13
:10731800049094F82C0140B101287CD002285AD05E
:10732800032879D04FF4AC619CE1D4F86401E8B348
:107338000121002005F096F90646A069BDF808105D
:10734800304403F002FFC4F83001BDF8081060684B
:1073580003F0FBFEC4F8340101A9684602F03AFEC6
:10736800DDE90012D4F85801FBF78CF98246204673
:1073780006F05BF994F86300D4F8648107F030FAFA
:107388004AF2A13101444FF47A70B1FBF0F0A169DF
:10739800D4F830213144081A811A41442039A1EB2C
:1073A8000A065000A18A6030014400E010E094F819
:1073B800630006F04FF92030CBF81000D4F86401D0
:1073C8005946301AB0F5D77F5CD840F2F94149E107
:1073D80040F2D74146E1D4F82411A0690844BDF829
:1073E800081003F0B2FEC4F83001BDF80810606858
:1073F80003F0ABFEC4F83401204606F016F9B4F8E1
:10740800060110BBB9F1000F1FD094F86380404605
:1074180007F0E6F901E036E052E04AF2A131014412
:107428004FF47A70B1FBF0F0D4F83011A269084437
:10743800D4F8241111440E1A404607F0C3F9D4F8C1
:107448006811081A0644203E06E0A169D4F8240110
:107458000844D4F83011461AD4F82821D4F8201159
:10746800D4F8300101FB02004000A18A60300144D9
:1074780094F8630006F0EEF8CBF8100001205946A6
:1074880084F82C0166E0D4F834116068B4F8062159
:10749800461A02EB0A00D4F82821D4F820C1801A31
:1074A800D4F83031401E0CFB023200FB01204000B2
:1074B800A18A6030014406FB08F694F8630044E0B2
:1074C8006068D4F8341100FB08F008FB110694F842
:1074D8007500242803D094F87600242809D1B4F83C
:1074E8008C01381A00B2002803DB94F88F0100B130
:1074F80001900098F8B1B4F80601E0B9D4F8680131
:1075080000287DD0D4F86401002879D094F863006D
:1075180007F066F94AF2A13101444FF47A70B1FBE1
:10752800F0F0361A94F8630007F04CF9D4F86811B3
:10753800081A0644203EB4F8061101EB0A00D4F8F4
:107548003411484341006031019806F083F85946E8
:10755800CBF8100004980969331AD4F834616068CC
:10756800801BA0F23D20CBF81400814200D80846C9
:10757800C4F800010020287064202881D4F858013C
:107588001946DC34F9F7FAFFE86054F8B40C616A7C
:1075980008446860E868E067A4F880700120A87271
:1075A800A18ADC3CC91B09B2002901DD0321A972AB
:1075B800039931B3B9F1000F27D000BFB4F81821EF
:1075C80092B3B4F81A1100BFA4F81A1194F81C3138
:1075D800491C4B43934218D2A97A491E002914DD4D
:1075E800A872B4F81A010121401CA4F81A0104F584
:1075F8008E70FCF7DFFB94F81C0100F0070001E037
:1076080013E015E0401C84F81C0194F86001294639
:1076180006F032F820B3079880F0010084F84001A2
:10762800002009B0BDE8F08F18E040F24B5119E096
:10763800B9F1000FC2D194F82C010028E5D0D4F894
:1076480034116068411A284605F01EF80004000C41
:10765800DBD0129901B108800120E2E70021B3E7ED
:1076680040F2AB513020FCF72DFB00001401002044
:1076780070B540B109294AD2DFE801F007173D3D4E
:1076880039492B414500D5213EE02249044688610D
:10769800FEF7C2FD10B140F2872135E0D4F8D000E2
:1076A800BDE87040F638FAF73BBF054605F08AFC9E
:1076B800A8B9284605F090FF0446D5F8D000A042A6
:1076C8000BD2201A0421F9F797FE30B12846C5F8E5
:1076D800D040BDE8704005F046BCC5F8D04028460B
:1076E800FEF7B6FD002814D040F2BB210CE0BDE83F
:1076F800704002F013BFBDE8704005F007BFBDE859
:10770800704005F060BFF7213020FCF7DBFAFB2161
:10771800FAE770BD1401002070B50446FAF798F82E
:10772800642801D9054600E0642594F863002821FF
:1077380005F0EAFE2844D4F8341100F237200E1878
:1077480094F86300282105F0DFFE00F29B22204612
:10775800616A05F0B4FA054632462046616805F0CC
:10776800AEFA07498542886000D228464860D4F8B6
:107778004801A0F5B270C860BDE87040FAF7D0BE05
:10778800140100207CB5044603F0A0FC0146D4F89F
:107798005401F9F725FF616811B1B0FBF1F000E081
:1077A800002094F876100D290CD0B4F86C20B4F8A9
:1077B8003E111318CB1A1BB2002B06DB491CA4F888
:1077C8003E1106E0B4F83E010CE0401C1044A4F859
:1077D8003E0194F8410140B9B4F83E01B4F8F41000
:1077E800884202D1401CA4F83E01B4F85E01401C56
:1077F800A4F85E01B4F89E00B4F89C10401AB4F8DE
:107808006C10401E084485B223E001A800230090B4
:107818001A462046FFF710FD002836D0012804D06C
:1078280040F262613020FCF74DFAB4F83E11B4F82A
:10783800F0000A1A12B2002A06DABDF804200A4437
:10784800AA1A12B2002A02DBBDF804000844A4F800
:107858003E01B4F83E11681A00B20028D5DA94F84F
:10786800790080B15FF0080084F88D00012084F869
:107878008C00204606F082F8204605F056FFBDE849
:107888007C4001F0D7BD3E20EEE77CBDF8B50D4643
:107898000746002104F0F9FC041E4FD094F8680054
:1078A80000284BD094F8B0018DF8000000980090A3
:1078B8009DF800000026D8B16E70072028700BE0F4
:1078C80084F8B061A683D4F8B2016860D4F8B60130
:1078D800A860B4F8BA01A88194F8B0018DF8000046
:1078E800009800909DF800000028E9D12E710BE166
:1078F80094F8BC01A0B394F8BC010B2816D00C284E
:1079080004D040F6CE213120FCF7DCF92088FCF7C2
:10791800EDFD074604F074FB78B96E700C202870F2
:1079280094F8BE0128712088E88013E02088FCF7CD
:10793800DDFD074604F064FB08B10020F8BD6E7059
:107948000B20287094F8BE0128712088E88094F8EC
:10795800C201287284F8BC61384604F066FBD3E0A3
:10796800FFE794F8F2018DF80000009800909DF868
:10797800000030B16E700E202870AF8084F8F2617C
:10798800C2E094F8C4018DF80000009800909DF8BA
:10799800000098B16E70082028702088A880D4F85C
:1079A800C811C5F80610D4F8CC11C5F80A10B4F8F7
:1079B800D001E88104F5E2742670A5E094F8EC01A2
:1079C8008DF80000009800909DF80000A0B16E703E
:1079D8001620287005E000BF84F8EC61D4F8EE01A9
:1079E800686094F8EC018DF80000009800909DF80C
:1079F80000000028F0D187E094F802028DF800001A
:107A0800009800909DF8000070B16E7006202870F4
:107A1800D4F804026860D4F80802A860D4F80C020C
:107A2800E86004F501743AE094F8D2018DF800009A
:107A3800009800909DF80000D0B16E701220287058
:107A48000BE000BF84F8D261D4F8D4016860D4F8A0
:107A5800D801A860D4F8DC01E86094F8D2018DF868
:107A68000000009800909DF800000028EAD14BE043
:107A780094F8E0018DF80000009800909DF800004F
:107A880080B16E7018202870D4F8E2016860D4F8CC
:107A9800E601A860B4F8EA01A88104F5F17404F8D5
:107AA800026C31E094F8F4018DF800000098009021
:107AB8009DF8000038B119202870D4F8F6016860E4
:107AC80084F8F46120E094F8FA018DF80000009839
:107AD80000909DF8000000283FF430AF6E7013202E
:107AE800287007E084F8FA61D4F8FC016860B4F8FB
:107AF8000002288194F8FA018DF80000009800909F
:107B08009DF800000028EDD10120F8BD1B481A4956
:107B180081601B4941601B4901601B4981621B4907
:107B2800C1621B49C1601B4981611B4901631B4933
:107B380001621B49C1641B4981641B4941641B499B
:107B480041631B49C1611C481A4981601B49C161D5
:107B58001B4941621B49C1621B4901611B494161C3
:107B68001B49416441631B4981611B4901631B49EE
:107B780081641B49C16470473D8D000044010020A9
:107B8800E18900003D8A0000718C0000B58C00007E
:107B9800E98A0000158D0000598E0000958B0000C1
:107BA800458C0000198C0000D58C0000058D000064
:107BB800718D000019910000A8010020419100007A
:107BC800B98F0000319000008D8F00008190000077
:107BD8005D900000A590000099910000E98F0000D9
:107BE800199000002DE9F8430127734C002567F32D
:107BF8000701658065702570A0608946804680F819
:107C0800FB700088FCF788FC80B1A0680088FCF74E
:107C1800D7FEA0680088FCF77BFEA068B0F8F210D9
:107C2800A9B1683005F0B9FE28B110E040F6A931D5
:107C38003120FCF747F8A06890F8701139B190F836
:107C4800782001231946683004F073FC80B1A068DD
:107C5800683005F0A2FE28B1A06890F8E40000BFE3
:107C680000F028FBA06890F8FD1089B1A5801EE0FF
:107C7800A068A0F8A05090F8711180F8E6100021D3
:107C8800022000F0A3FDA06880F8FA500220E7E780
:107C980090F8B0118DF80010009900919DF800102F
:107CA80019B9818B0289914200D80189A18030F8E5
:107CB800F61F491E8EB230F8021F314420F85C19B5
:107CC80001883144018001F091FA20B1A06850F890
:107CD800901F31440160A068B0F8F210012902D861
:107CE800491CA0F8F2100EB180F8045180F8FA503F
:107CF80090F876100B2901D00C2918D1B0F86C2017
:107D0800B0F88C31D21A12B2002A10DBD0F88E11DA
:107D1800C0F87E1090F8921180F882100321FDF7C8
:107D2800E5FDA06880F8765080F8B67024E0242934
:107D38000FD1B0F86C10B0F88C21891A09B200295B
:107D480007DB00F0EFFDA06880F8765080F8A651B8
:107D580012E090F87510242901D025290CD1B0F82B
:107D68006C10B0F88C01081A00B2002804DB00F08F
:107D7800D9FDA06880F87550A0680146B0F8F620D3
:107D8800683004F05AFD0D4800900D4B0D4A4146ED
:107D98004846FCF7CBFEA0680123052190F8762021
:107DA800683004F0C6FB002803D0BDE8F843FCF7B0
:107DB800B7BEBDE8F8830000300100206D840000E4
:107DC800857F00007988000070B50F4CA56895F88C
:107DD8007510202902D0262903D011E000F0D8FD23
:107DE80008E095F8762001230B2105F1680004F0DE
:107DF800A0FB38B1A168002081F8750081F8A600C1
:107E0800002070BD2A20E9E7300100200448002145
:107E1800806820F8A81F8178491C8170704700008D
:107E280030010020074810B5816811F8AA0F401EDC
:107E380040B20870002804DA40F28F113120FBF7B5
:107E480041FF10BD30010020174910B5896891F82D
:107E58007620B8B1102A06D0142A07D0152A08D0DF
:107E68001B2A1CD108E001210B2007E001F04CF887
:107E780006E000F0C9FC03E00121062000F0A6FCA2
:107E8800012010BD212A0AD191F8A601022808D0A4
:107E980091F8A601012802D191F8A70108B10020A4
:107EA80010BD01211720E9E73001002010B5E8BB1B
:107EB800314CA06890F87710CA0702D00121092038
:107EC80052E08A070AD501210C2000F07FFCA06847
:107ED80010F8AE1F41F00101017047E04A0702D5D2
:107EE8000121132040E00A0705D510F8E11F417170
:107EF8000121072038E011F0300F3BD090F89D1198
:107F0800A1B990F89C11E1B190F8761024292FD0EE
:107F180090F8751024292BD05FF0000300F5C77284
:107F280000F5CE7104F0BDFEA16800E022E011F872
:107F3800770F20F0200040F010000870002081F832
:107F48002501A06890F87710C90613D504F0C4FE7F
:107F580000F0A6F8A16801F12400C28B21F8E62FF1
:107F6800408C48800121152000F030FC012010BD14
:107F78000123D3E7002010BD300100200C49024640
:107F8800487898B90846806842B18978090703D5C6
:107F980090F87800082809D00120704700F12401E2
:107FA8008A8C818D8A4201D8FEF796BF00207047DF
:107FB8003001002070B5394C0546A068683005F0DE
:107FC800ECFC002869D1002D67D1A068012319466F
:107FD80090F87820683004F0ACFA00285DD1A068E9
:107FE80090F8701149B10021A0F8A01090F8711113
:107FF80080F8E6100021022045E090F87620012361
:108008000421683004F095FA0546FFF74FFF002871
:1080180043D12846FFF718FF00283ED1A068012366
:10802800002190F87520683004F083FA78B1A068D0
:108038000123042190F87620683004F07AFA30B9E8
:10804800A06890F89A0010B1002112201BE0A068E7
:1080580090F875100A291AD0002D1ED100F016FBD1
:1080680000281AD1A0680123002190F875206830F3
:1080780004F05FFA002810D0A06890F88401002866
:108088000BD00021FF20BDE8704000F09FBB10F826
:10809800E21F017100210720F5E770BD30010020C3
:1080A8000A4810B5816891F85800012809D0088855
:1080B80001F5E972243104F0D0FDBDE8104001F06B
:1080C800B9B9022081F8580010BD00003001002025
:1080D80070B5254C05002FD100F0A4F800F048F841
:1080E800050029D16088410706D5A16891F8781064
:1080F800072901D101212170800712D5E068C078D5
:10810800192805D2194951F8201009B1884708E003
:10811800FF2804D040F23C713120FBF7D3FD00F07A
:1081280025FFA078C00607D5A06890F876100B291F
:1081380002D10C2180F876106078000711D5A0686C
:108148000123052190F87620683004F0F2F928B16F
:10815800A1680825002081F8BC0102E00020FCF796
:108168009FFD284670BD000030010020A8010020B6
:1081780070B52A4C0020A178C90715D020690123C1
:108188000521C578A06890F87620683004F0D1F908
:1081980058B1AD1E0A2D06D2DFE805F00707050520
:1081A800070705050707082070BD2069FDF774FC5F
:1081B80038B12069C57845B1012D06D0162D18D1E2
:1081C80003E0BDE8704000F00BBDA06890F87500B2
:1081D80004F0FDF968B1A16891F875001F2808D06E
:1081E800202803D0162D0CD0022070BD262081F83F
:1081F8007500192D07D20A4850F8250018B1804794
:1082080003E0202070BD00F0EBFCA268F2E9301317
:10821800491C43F10003C2E9001370BD300100207E
:108228004401002070B5224CA07800073ED5A06814
:10823800683005F0B2FB48B1A068FE21002580F83F
:10824800E41090F8761019290CD104E040F2467138
:108258003120FBF737FD80F8AB50FFF7E3FDA0684E
:1082680080F87650A06890F875101F2902D0272949
:1082780013D10BE090F8760004F0A9F908B1262094
:1082880000E02020A16881F8750006E0012180F84F
:10829800851180F8755080F8A650A06890F878107D
:1082A800082903D10221217080F8E41070BD000074
:1082B80030010020FEB505466846FCF76BFB18B395
:1082C80022220021009803F0FBF80321009804F013
:1082D80095FB0098017821F0100101702946FDF7FF
:1082E800EBFB00215E4C44F62F160E2D7ED00EDCE3
:1082F800A5F102050C2D1CD2DFE805F01E1B45A7D1
:10830800A71E1B511BA7233740F66B11A3E0152DA1
:1083180058D008DC112D1FD0122D1CD0132D1AD0C7
:10832800142D06D14EE0162D23D0172D65D0FF2D24
:108338007ED040F6DD118EE0A168009891F8E61035
:1083480015E000980B2202715922427181715B215C
:10835800C1711221017278E00321009804F02AFB10
:108368000621009804F028FB6FE0009806210171AF
:108378006BE00098D4F8081091F8A821027191F8E0
:10838800A911417161E0A168009801F5887104F0B4
:1083980026FBA1680098DC3104F01EFB55E0019132
:1083A800029101F001FBA168304091F8B41001403E
:1083B8008DF80410000A8DF8050001A9009804F052
:1083C80018FB42E0A068B0F84410009804F01EFBC7
:1083D800A068B0F8E810009804F01CFBA068B0F89A
:1083E8004010009804F01AFBA06800E010E0B0F814
:1083F800E610009804F016FB27E0A16891F8A601A2
:1084080001280098B8D011F85E2F02714978B8E7B2
:108418000191029101F0C8FAA168304091F8B410B6
:1084280001408DF80410000A8DF8050001A900E04C
:1084380003E0009804F0D8FA07E0A06890F88721D4
:10844800D0F88811009804F0B9FAFCF77DFA0028F2
:1084580004D140F6E1113120FBF734FCFEBD0000E9
:10846800300100202DE9F047874C82468946A068F4
:108478000088FCF751F806000AD060884FF0000524
:10848800C005A06809D5A0F89C5080F8045108E000
:1084980040F681513120FBF715FC30F89C1F491C30
:1084A800018000F0A3FE4FF0010820B360880005AA
:1084B80006D5A06890F87B1011B1C0F890501AE06A
:1084C800A068D0F89010491CC0F89010D0F89430EB
:1084D8008B4201D35A1A00E00022A7887F1DBA42B6
:1084E80001D880F89A80994205D3C0F8905080F856
:1084F800F28100F09FFF60884FF0020710F4407F80
:108508000ED0A06890F8791011B1032908D102E0C3
:1085180080F8798001E080F879700121FEF702FD8A
:10852800A06890F87910012904D16188490501D51E
:1085380080F87970BAF1000F75D1A178490602D593
:10854800A0F8185104E0B0F81811491CA0F8181147
:108558004846FFF7BDFD40EA09008146FFF72AFDBE
:10856800A768B7F8F800401CA7F8F80097F8FC00CF
:1085780028B1FCF703FCA8B1A7F8F85012E0FCF703
:108588008BFA08B1A7F8F850FCF780FA50B197F8C1
:108598000401401CC0B287F80401022802D927F858
:1085A800F85F3D73A0680123002190F876206830B9
:1085B80003F0BFFF20B9A06890F876000C285FD1BF
:1085C800A0680123002190F87520683003F0B1FFFE
:1085D80050B3A0680123002190F87820683003F098
:1085E800A8FF08B3A06890F87910022948D190F83C
:1085F8000401C8B9304603F08EFBA8B1A068683002
:1086080005F0CBF980B9A168B1F8F200012837D993
:1086180081F8FA80B1F89E20B1F89C00931E984228
:1086280003DB012004E01DE02AE0101A401E80B29E
:10863800B1F8F820A3889A4201D3012202E09A1ADD
:10864800521C92B2904200D91046012802D100BFB4
:1086580081F8FA50A168B1F86C201044A1F8F40030
:1086680000F084FEA0784A46C0F38011504600F01E
:10867800D1FDA06880F8FB50BDE8F047FCF74EB983
:108688000120A168E4E700003001002070B54E4CDD
:1086980001230021A06890F87520683003F049FF95
:1086A800002876D0A06890F8AD11002539B10021D6
:1086B8000E2000F08BF8A06880F8AD5182E090F8A9
:1086C800AC1119B190F8AE1089070AD090F89C1136
:1086D80011B190F89D1189B190F8A61101292FD0F8
:1086E8006AE000210C2000F071F8A06810F8AE1FB5
:1086F80041F00101017080F8FE5063E090F87610B7
:1087080024291BD090F87510242917D05FF0000396
:1087180000F5C77200F5CE7104F0C3FAA06880F8BE
:108728009C510021142000F051F8A16801F12400A7
:10873800C28B21F8E62F408C488043E00123E7E70D
:1087480090F8A71121BB90F8762001230B216830FF
:1087580003F0EFFEE0B9A06890F8620005F025F993
:108768000546A06890F8630005F01FF90646A06862
:1087780090F8A811284605F023F958B1A06890F898
:10878800A911304605F01CF920B1002000F000F9CD
:1087980012E012E0A0680123032190F876206830E7
:1087A80003F0C7FE40B9A0680123022190F87620A3
:1087B800683003F0BEFE08B1002070BD002116200D
:1087C80000F004F8012070BD3001002070B50D4C98
:1087D80006460D46A068683005F0DFF820B140F67F
:1087E800F4113120FBF76EFAA268002082F8E460E9
:1087F80015B1A2F8A80070BD22F8A20F01201071CF
:1088080070BD00003001002070B5184C0025A0682C
:1088180090F8731101290AD0022925D190F8AC10DB
:10882800A9B1062180F8E6100121022017E090F88E
:10883800BC11002918D100F1C80300F58471002289
:1088480000F5BA7003F02DFE0121052007E090F82D
:10885800B400400701D5112000E00D200121FFF7E9
:10886800B5FFA06880F8735170BD0000300100208A
:1088780070B52B4A03465088184350801046402B49
:1088880080680DD09E074FF000054FF001044FEAB5
:10889800C3760CD54EB140F6EE413120FBF712FA03
:1088A800BDE870400421FEF73DBBD1601CE0C6B1B5
:1088B8001161C978062902D00B2912D109E090F874
:1088C800761017290DD10021C0E92E1180F87A40C1
:1088D80007E090F87610112903D180F87A5080F8D3
:1088E800AC40990716D5D168C978052902D00B295B
:1088F80010D109E090F8761015290BD10021E0E994
:10890800301100F8454C05E090F87610102901D197
:1089180080F87B50980601D50820507070BD000083
:108928003001002070B5194CA06890F88E1109B17B
:10893800012600E0002690F88F210AB1012500E009
:1089480000250EB990F862100DB990F8632000F177
:108958005A0319725A720121997290F8A6010128D6
:1089680001D006B915B1002000F012F8A06804F093
:10897800B3F9002808D0A16801F5E9720888BDE8B4
:108988007040243104F069B970BD00003001002046
:1089980010B5104CA1680A88A1F8FE2181F8FC01E5
:1089A80091F8620005F001F8A16881F8000291F8D9
:1089B800630004F0FAFFA26802F5FD7182F8010273
:1089C80001200870002082F8A601BDE8104000F0E0
:1089D80031BD00003001002010B5154C01230021E5
:1089E800A06890F87620683003F0A3FD90B1206964
:1089F80003F0A7FFA168A1F88C01B1F86C1004F08E
:108A0800EDFF48B1A068282180F88D106E30012153
:108A180081770BE0012010BDA168206901F5C771BD
:108A280003F08AFFA1680B2081F87600002010BDB2
:108A38003001002070B5294C01230021A06890F86E
:108A48007620683003F075FDB8B10021206903F085
:108A58004BFFA0B12069A168B0F80D00A1F88C0106
:108A6800B1F86C1004F0BAFF68B1A068282180F84A
:108A78008D106E30012181772EE0012070BDBDE898
:108A8800704000F0ADB8206903F05EFF03F034FDDC
:108A98000546A0682946C0F894512069007903F07A
:108AA80061FEA168A1F88E0120692946B0F8050089
:108AB80003F054FEA168C1F89001206903F047FF54
:108AC800A168A1F89801206903F044FFA168A1F802
:108AD8009A010D2081F87600002070BD3001002039
:108AE80038B5294C01230021A06890F87620683019
:108AF80003F01FFD70B9A06890F87620122A09D0FB
:108B080001230521683003F014FD08B1082038BDA1
:108B1800012038BDA06890F8AC0008B9FFF776F9D5
:108B2800A168206901F5847103F023FFA168206919
:108B3800D83103F015FFA16891F8C4018DF8000041
:108B4800009800909DF8000020B140F29D2131204E
:108B5800FBF7B8F80888A1F8C60101F5E4712069A7
:108B680003F002FFA168206901F5E87103F0F5FE42
:108B7800A0680146012280F8C421142081F87600FB
:108B880000F058FC002038BD300100201CB5134C03
:108B9800A06890F87700C00701D001201CBD694685
:108BA800206903F0ECFE00F0FFFE44F62F110840A8
:108BB8009DF80020A168024001F8B42F9DF801201B
:108BC80002EA10204870FFF721F9A06810F8771F13
:108BD80041F00101017000201CBD0000300100209F
:108BE8000A4A10B5906890F877100B0701D5012054
:108BF80010BD41F0080180F877101169C97880F834
:108C0800E110FFF703F9002010BD0000300100203B
:108C180010B5094CA06890F87700400701D50120ED
:108C280010BDFFF7F3F8A06810F8771F41F00401B2
:108C38000170002010BD00003001002010B5094C63
:108C480001230921A06890F87520683003F071FCB1
:108C5800002806D0A168002001F89A0F087301F8CF
:108C6800250C10BD3001002010B50F4C0123002148
:108C7800A06890F87620683003F05BFC38B1FFF705
:108C8800C5F8A168102081F87600002010BDA06802
:108C98000123052190F87620683003F04AFC08B1DA
:108CA800082010BD012010BD300100200648806852
:108CB80090F87610112901D002207047122180F80F
:108CC80076100020704700003001002010B50A4CD3
:108CD800A06810F8B41F41F004010170206903F086
:108CE80065FE162801D0002010BD206903F060FE43
:108CF800BDE81040FFF768B830010020024800695D
:108D08000079FFF761B800003001002010B5084C69
:108D1800A06890F87600172801D0022010BDFFF750
:108D280081F8A1681B2081F87600002010BD0000A2
:108D38003001002010B50B4C01231946A06890F8AB
:108D48007820683003F0F5FB08B1002010BD2069D9
:108D580003F01EFEA16881F87201072081F87800EF
:108D6800F3E70000300100202DE9F041374D0026DF
:108D78002846A9680069012791F8753000790E2BFB
:108D880001D1122806D0314A00249268B4321C2B33
:108D980004D005E0FFF752FF064653E0142802D03E
:108DA800042B0BD00CE081F8754081F8A640052112
:108DB800104604F0A4FDFFF773F943E00E2802D033
:108DC800202B0FD010E081F8754081F8A640088864
:108DD800A1F806021A2081F8040281F8027200F054
:108DE80029FB2FE0162806D0262B01D1162802D001
:108DF800172814D026E001F8754F81F831404878DB
:108E080021281FD00821104604F079FDA8680B21FD
:108E1800B43004F074FD1A20FFF7BAFD12E091F89F
:108E2800760022280ED181F87640FEF7FBFFA8686D
:108E380090F8A601012802D10020FFF7A9FDA86833
:108E480080F8A6413046BDE8F081000030010020DE
:108E580070B52C4CA06890F87710890707D590F862
:108E6800752001230821683003F063FBE8B1A0688E
:108E780090F8AE00800712D4206903F08BFDA1683A
:108E880081F8AF00206930F8052FA1F8B02040889C
:108E9800A1F8B20011F8AE0F40F002000870A06807
:108EA80090F8AE10C90702D010E0012070BD90F80C
:108EB80077108A0704D540F2D9213120FAF702FF4A
:108EC80041F0020180F87710FEF7A0FFA0680025A6
:108ED80090F87510062905D180F8755080F8A650CD
:108EE80000F0A8FAA06890F8AC1149B180F8AC512C
:108EF80000F0A0FAA06890F8751009B980F8A6509B
:108F0800002070BD3001002010B5174CA36893F8FD
:108F1800EA0008280ED200F10802C0F10800C1B228
:108F2800981800F58470FAF745FFA16811F8EA2F40
:108F380010440870A36893F8EA000838042811D28E
:108F4800021DC0F10400C1B29818D830FAF732FFF8
:108F5800A068002180F8EA100121BDE81040042033
:108F6800FFF734BC10BD0000300100200448272161
:108F7800806880F87510002180F88411704700001F
:108F880030010020094810B5806890F8761014293F
:108F980004D040F289613120FAF794FE012180F86B
:108FA800AB10152180F8761010BD000030010020AC
:108FB80010B50A4CA06890F87700C00708D0FEF7F3
:108FC80031FFA06810F8771F21F00101017010BD72
:108FD80040F272613120FAF775FE0000300100207E
:108FE80010B50A4C01230021A06890F8752068305C
:108FF80003F09FFA20B1A1680E2081F8750010BD1A
:1090080040F2EA613120FAF75DFE000030010020ED
:109018000448806810F8771F21F004010170FEF7FA
:1090280001BF000030010020094810B5806890F8A1
:109038007610102904D040F281613120FAF742FEFF
:10904800012180F8AB10112180F8761010BD0000C6
:1090580030010020074810B5806890F8761015296F
:1090680004D040F296613120FAF72CFE192180F8DD
:10907800761010BD30010020074810B5806890F8C0
:109088007610152904D04FF4D2613120FAF71AFE70
:10909800172180F8761010BD3001002070B51B4DE7
:1090A800A86890F876101B2902D04FF4D66107E023
:1090B800002480F8AB4090F8BC1121B140F2B461B3
:1090C8003120FAF7FFFD90F8AC1041B180F8AC40C0
:1090D8000188A0F8C01180F8BE410C2108E0018881
:1090E800A0F8C01180F8BE41012180F8C2110B21FF
:1090F80080F8BC110088FBF7F9F902F09CFF00F03A
:1091080099F9A86880F8764070BD00003001002009
:1091180010B5084C01231946A06890F878206830EB
:1091280003F007FA002803D1A168082081F8780025
:1091380010BD000030010020144810B5C1688068D7
:10914800097990F875200A2A09D190F8E2208A4214
:1091580005D1002180F8751080F8A61010BD90F890
:109168007720130707D522F0080180F87710BDE8AB
:109178001040FEF757BEFF2904D040F26C61312041
:10918800FAF7A0FDBDE81040FFF7F0BE300100205F
:1091980010B5154CA06890F8AE10890711D490F856
:1091A800752001230021683003F0C3F920B1A168BC
:1091B800062081F8750009E040F2D6613120FAF7FF
:1091C80081FD002180F8A61080F8AC11A06890F805
:1091D8007700800707D5FEF725FEA06810F8771FEF
:1091E80021F00201017010BD30010020084810B5BF
:1091F800806890F87B1041B990F876200123062109
:10920800683003F096F9002800D0012010BD000056
:1092180030010020F8B5544C06461546A06809B13F
:10922800002104E0B0F80611B0F8F6201144A0F8C7
:10923800061190F8701139B990F878200123194671
:10924800683003F076F930B1A06830F8A01FB0F8A4
:10925800562011440180A06890F8A62032B1B0F8D9
:10926800A210B0F8F6301944A0F8A21090F9AA702C
:10927800002F06DDB0F8A810B0F8F6301944A0F8B1
:10928800A81001213D2316B180F88D3013E0247811
:10929800022C0AD0012C12D045B300F18C021170B7
:1092A80015F0140F0ED01E2118E090F8E620062ABB
:1092B8003ED016223CE000F18C02117041E090F89B
:1092C800722135E0290702D580F88D3039E0A906EA
:1092D80001D5232102E0A90703D02A2180F88D10A7
:1092E8002FE040F69B413120FAF7ECFC2AB1B0F8A8
:1092F800A220B0F8A4309A4210D2002F05DDB0F8B1
:10930800A820B0F8A4309A4208D2B0F8A030B0F83B
:109318009E20934204D390F870310BB1222207E0CB
:1093280090F879303BB1B0F89C30934209D30822C9
:1093380080F88D20BFE7B0F89C20062A01D33E2292
:10934800F6E790F88C108DF80010009900919DF8C0
:10935800001019B1BDE8F84004F010BBBDE8F840B2
:109368000021FDF7DFBD00003001002070B52D4D54
:10937800A86890F8791051B1012908D0022909D0BC
:10938800032907D040F65F213120FAF79BFCB0F89B
:10939800F41035E090F87810082934D0B0F89C1013
:1093A800B0F89E2000248B1C9A4206D3511A891EBD
:1093B8000C04240C01D0641EA4B290F89A1039B1A0
:1093C80090F8752001230921683003F0B2F830B312
:1093D800FFF70CFF68B1A9680020903106C98B1C03
:1093E8009A4203D3501A801E00D0401EA04200D2D9
:1093F80084B20CB1641EA4B2A868B0F8F410214479
:10940800A0F8F01070BDB0F89C100329BFD330F855
:109418006C1F428E1144491CA0F8841070BD0024B2
:10942800EAE7000030010020014908707047000099
:10943800AF02002001480078FAF77EBAAF02002098
:1094480003498A880280897881700020704700006B
:10945800C80D00207CB50C4605460088694603F017
:109468003EF8002228B1C4F80220A271228002200E
:109478007CBD019911F1680181F84E20D1F81600E0
:10948800C4F80200887EA0712888208091F84E00D8
:109498000028F1D17CBD00001CB50088694603F0A6
:1094A8001EF800280BD10B48007888B1019805F008
:1094B80031F828B1019890F8AD0118B13A201CBDD7
:1094C80002201CBD0199012081F8AD0100201CBDBE
:1094D80011201CBD0C020020017879B1417869B1D6
:1094E80041881B290AD381881B2907D304490268AC
:1094F800C1F802208088C880002070471220704779
:10950800C80D0020006840F2E241884203D30349B5
:10951800886000207047122070470000C80D0020A6
:10952800034AD2E90012016042600020704700003F
:109538006498000010B502F035FFFCF729F80F48D1
:109548004FF6FF710E4BC18101820021C175018365
:1095580001801B221A804FF4A4745C809A80DC80FE
:109568008174C174032383700223C3708280C28014
:1095780040F6A66282608175017310BDC80D002097
:109588001402002010B558B10A490A786AB10022BD
:10959800427003230370012303710A70184610BD3B
:1095A8004FF4BE513920FAF78DFBBDE81040FCF7A7
:1095B80097BA0000C80D00202DE9F04188B00C468C
:1095C800064603F00CFD98B1304603F0FBFC30B1C1
:1095D800B4F80110122000290BD0802909D8304690
:1095E80003F0DBFC40B1304603F062FC30B109E027
:1095F800422008B0BDE8F0810C20FAE7304603F0BD
:10960800DBFCA8B3304603F0EEFE0028F4D1304668
:1096180003F069FC0028EFD13046FCF77FFCB4F872
:10962800010042F2107100FB01F8E178304603F0C6
:10963800ABFC304603F0C2FCE8B10022114601A899
:10964800FAF798FD04006AD00021FCF74FF9BDF83D
:10965800040020802146304603F0D4FC04F051FF7A
:109668003A4D002804F124000FD0AA88E9880EE0BA
:10967800FFE71220BDE7424600213046FDF76EFBAA
:109688000028B6D041F2FD3153E01B221146C284B6
:109698000185A868606241F64C57304603F096FC95
:1096A80010B9304603F0ACFC67602188ADF80810AB
:1096B800A97C8DF80A10E97C8DF80B10A98AADF801
:1096C8000C1005A90091012004AB02AA214604F060
:1096D800D9FE40B10021BDF80400FAF775FDF0B1DC
:1096E80041F2484125E09DF810008DF818009DF8DA
:1096F80014008DF81900BDF80C00ADF81A0006A981
:10970800204602F0ABFFE8780090AB78EA88A98899
:109718002088FAF725FE20B141F2534109E00920DB
:1097280067E7424621463046FDF718FB20B141F273
:1097380055413920FAF7C6FA0548436823B1002293
:1097480004F5CE7120469847002052E7C80D002046
:109758000C0200202DE9F04188B00446008806A9D3
:1097680002F0BDFE002847D10798002790F8E011C5
:109778008DF80810029902919DF808108DF80C10C8
:1097880090F877106830890602D59DF80C1049B119
:109798005FF000018DF8041005214C3004F02AF91F
:1097A80010B104E00121F5E79DF8040018B3218900
:1097B800E08804F023FE00281ED1A188608804F008
:1097C8001DFE002818D12189E08804F00DFE00282C
:1097D80012D1A188608804F007FE06000CD1079812
:1097E8004FF0010800F5CE7580F89D819DF80C10AA
:1097F80029B13A262FE01A2008B0BDE8F081394691
:1098080003AA04F009FE6188BDF81200814200D263
:109818000846E880A188BDF81400814200D20846B5
:109828002881E288BDF80E108A4200D2114669806C
:109838002289BDF810108A4200D2114640F648022B
:10984800A980914200D31146A980904200D20246D5
:109858002A8185F800806F703046CDE70B5B120BCC
:1098680059005B120807060504030200FCF8F4F02F
:10987800ECD8040300FCF8F4F0ECD80010B5FFF7BE
:10988800D3FD0448406804F0F8FEBDE8104004F039
:1098980065BC00001C02002010B5074CA06804F04D
:1098A800ECFEE06804F0E9FE02F07CFDFBF770FED8
:1098B800BDE81040FFF73EBE1C02002000B5054978
:1098C800054804F0BBFE04480449001D5DF804EB9C
:1098D80004F0B4BE2C020020200200203402002034
:1098E80000B50849084804F0A9FE07480749001DC3
:1098F80004F0A4FE0448064908305DF804EB04F0BF
:109908009DBE0000580200202002002060020020B6
:109918005002002001480078704700001C02002017
:1099280010B5FCF771FCFDF7B1FA0548FCF752FCDD
:1099380005490448086006490448086010BD00004D
:1099480093110020E55F00003C020020895B0000C5
:10995800400200200C4910B501200870FCF784FC77
:10996800FEF7D4F802F00CFD0848FBF7C5F8002014
:10997800FAF772FB07490648086008490648086074
:1099880008490748086010BD1C02002093110020F8
:10999800AD4A00004C0200209578000048020020E3
:1099A800FD5B000044020020014800687047000089
:1099B8006802002003480088C0F300204000401CD3
:1099C800704700006802002070B5054616460C4630
:1099D800022000F099F906490120F61E0870054892
:1099E8000660044808380560001F046070BD000068
:1099F800B002002010F5004010B50C4C207880B162
:109A08000B494FF40000086000F06AF8002120B10B
:109A1800012060700748006801E061701020A070A4
:109A28002170BDE81040002000F06EB9B00200209F
:109A380008F5014000F4004010B5022000F064F978
:109A480004490120087000F059F803494FF4000058
:109A5800086010BDB002002004F501400348002151
:109A6800017041701021817070470000B002002021
:109A7800074810B5017841B100F032F818B105482F
:109A88000068C0B210BD102010BD807810BD000065
:109A9800B002002000F40040084810B5017859B120
:109AA8000748D0F8000128B100F00CF8002800D0D1
:109AB800012010BD022010BD407810BDB00200206A
:109AC80000F000400548D0F8041111B1D0F80801A1
:109AD80008B10020704701207047000000F00040E6
:109AE800054810B5D0F8000120B1FFF7EBFF08B129
:109AF800012010BD002010BD00F0004004480021E6
:109B0800C0F80011C0F80411C0F80811704700002F
:109B180000F00040084A10B5C2E9020107491046A2
:109B2800F9F7B6FF002805D0401C03D07D2140205E
:109B3800FAF7C8F810BD00006C020020749B000002
:109B4800084A10B5C2E9020107491046F9F7ACFF07
:109B5800002805D0401C03D072214020FAF7B2F843
:109B680010BD00006C020020749B00000100000082
:109B7800101100400000000000000000000000007C
:109B88000000000070B5064614460D46012000F09E
:109B9800BBF803480660001D0460001D056070BD29
:109BA80008F500400A48017871B10A4A4FF000717F
:109BB80011600949D1F8042100211AB1074A126835
:109BC800427000E041700170002000F09DB8000074
:109BD800B302002008F5014000F0004000F4004006
:109BE80070B5044616480E4601250570154944EA25
:109BF800024040F08070086001F096FB30B91148CF
:109C08001430016821F0FF01314301600E49002240
:109C1800C1F804210D4B4FF0007018602CB1012CD5
:109C280007D085213C20FAF74DF8C1F800520D60A5
:109C380070BDC1F800220D600449091F086070BD9D
:109C4800B302002004F5004000F0004008F5014090
:109C5800024800210170417070470000B3020020E3
:109C68000648017841B10648D0F80401002802D01E
:109C780004480068C0B2704740787047B3020020BB
:109C880000F0004000F4004001490120886070475E
:109C980000F000402DE9F04700282CD01748007844
:109CA800B0B1174DD5F80401002824D10227C5F812
:109CB8000473144C2068C04340F30016206840F039
:109CC800100020604FF400484FF0E029761C07E0B0
:109CD800FD213C20F9F7F6FFC9F88082F9F782FEEA
:109CE800D5F804010028F7D01EB9206820F010002C
:109CF8002060C5F80873BDE8F0870000B3020020B3
:109D080000F0004010ED00E010B5044600F022F825
:109D1800002C17D00C4A0C480C4914320C4B012C5F
:109D280005D0022C08D07D213D20F9F7CBFF022475
:109D380004601160200604E00324046011604FF4FD
:109D48000000186010BD000000F5004095120020CA
:109D580004F50140044800210160016003494FF007
:109D6800207008607047000000F5004008F50140C9
:109D78000548D0F8001221F04001C0F8001203494C
:109D88000020086070470000001000406015004087
:109D9800044908600448D0F8001241F04001C0F8B6
:109DA800001270476015004000100040014890F80C
:109DB8002A007047040E0020014A51701070704745
:109DC800040E0020F8B51E4CD4F804031027C0F385
:109DD8000016C4F808730220C4F8000219480025C8
:109DE8001A4980F834501848086019480068B0B11A
:109DF800FF208DF80000C4F810510120206104E014
:109E08009DF80000401E8DF800009DF8000018B174
:109E1800D4F810010028F3D09DF8000050B100F0EC
:109E280007FDC4F8105100F09FFE002E01D0C4F8C1
:109E38000473F8BD40F2C3713E20F9F743FF0000F8
:109E480000100040040E002000000E0C08F5014030
:109E5800501500402DE9F0411F4C0746884694F8FC
:109E68003400C10718D01D4A4FF0406111601C4DE5
:109E7800D5F8001241F00101C5F8001240F00200C7
:109E880084F83400404600F0D5FE00F07FFC01263F
:109E98003FB1012F0ED016E040F255613E20F9F790
:109EA80011FF404600F092FC404600F053FCE67279
:109EB8002E6008E000F0B2FC00F020FE0220E07204
:109EC80000F028FD6E600748C664074801683846F8
:109ED800BDE8F04104F096BC040E002004F50140F2
:109EE80000100040008000404C8500402DE9F047FC
:109EF800354D06464FF0406089462860334C94F84B
:109F0800340040F0020084F83400084600F092FE65
:109F180000F03CFCDFF8B880002716B1012E27D0EE
:109F28003FE0484600F052FC607A012805D1D8F895
:109F3800001241F00801C8F80012484600F00AFC77
:109F48000120E072206B40F4801020634FF48010F1
:109F580028604FF47A71B9F1020F07D040F6340047
:109F680049F6EC721044B0FBF1F71AE00846F7E73F
:109F780000F054FC00F0C2FD607A012805D1D8F841
:109F8800001241F00401C8F800120220E072206BB0
:109F980040F4001020634FF400102860292700F0D7
:109FA800B9FC00F0A3FC01F08BF80068012806D08A
:109FB8000021304604F026FC3846BDE8F087FFF75C
:109FC80001FF0020F9E7000004F50140040E00201D
:109FD80000100040024A936B0360D06B0860704722
:109FE800040E002010B51DC8014981E81D0010BDF0
:109FF800F40D00200E4910B54A6A824202D340F699
:10A0080043010AE001220A7448610A494A640A4A7B
:10A018001368834204D340F64C013E20F9F752FE00
:10A028000023C1F844311060BDE8104000F074BD51
:10A03800040E0020008000404485004070B5104C9C
:10A04800064602202074962500F06CF8024694F823
:10A05800290094F8281001280DD0284604F0EAFBBE
:10A06800084960610020C1F844016169606A0844D8
:10A078000549086070BD3346284604F0F7FBEFE752
:10A08800040E0020008000404485004010B501F017
:10A0980067F9002806D00448016821F0010141F061
:10A0A8008071016010BD0000741700402DE9F04177
:10A0B80040220021134801F003FA00F055FD01F099
:10A0C80008F9114D104E00240F4F0835103628B9E5
:10A0D80001F016F910B901F01DF908B1242206E0C3
:10A0E80001F058F910B901F04BF940B14022FF21B5
:10A0F800384601F0E5F92C603460BDE8F08138227B
:10A10800F5E70000040E0020000E00400149087029
:10A1180070470000840200200148406A7047000030
:10A12800040E0020144810B590F82910C07A41B1E7
:10A1380002290BD0022809D001290BD0012809D007
:10A1480015E00028F6D14FF4EB710DE0BDE81040A2
:10A1580000F06EBC0948006800F00F00032806D024
:10A16800042806D040F20B213E20F9F7ABFD012070
:10A1780010BD022010BD0000040E00201015004084
:10A188000148006A70470000040E00200148407F23
:10A1980070470000040E002010B500F0CBFCFFF75C
:10A1A80011FE04F0C5FA0F480F4A016B41F4800113
:10A1B80011600024046304744462046200F0BAFC71
:10A1C8000A48C0F84841C0F84441C0F84041C0F8C6
:10A1D8004C41012004F0E5FABDE81040012004F0EC
:10A1E800D3BA0000040E002008F5014000800040AA
:10A1F80070B5012004F0D5FA374800240460012620
:10A20800066001F09DF8354D18B1286840F480606B
:10A21800286001F089F828B12868314920F06900E0
:10A228000843286001F09CF838B12C48001D0168EB
:10A2380021F47F4141F4B0510160284929483C315B
:10A248000860F9F73DFC40B14FF08050D0F830037A
:10A25800411C02D02149103108604FF01020006ED7
:10A26800411C04D020490A6860F317420A601E495D
:10A2780040F25B6054390860091F40F2031008601F
:10A28800081F0660012000F0D5FC174940F20110B4
:10A29800C4310860154E0225C6F800521549144805
:10A2A8000860154806F5007604871030446280F887
:10A2B8003440012004F068FA1020C6F804014FF079
:10A2C800E020C0F800510D484068002802D0BDE8E1
:10A2D8007040004770BD0000FC1F00403C17004064
:10A2E800960000802C0000898C150040001000406A
:10A2F80000000E0C08F50140F40D00208402002037
:10A308000149087670470000040E002004490860DF
:10A31800044810F8341F41F00101017000F0AEBA92
:10A3280004150040040E00202DE9F047354E07467D
:10A338004FF040608A4614463060104600F07AFCC0
:10A3480000F024FADFF8C090304D4FF0010827B133
:10A35800012F1DD040F244714AE0204600F036FA41
:10A36800204600F0F7F9022C0FD040F6340000BF69
:10A3780049F6F8510144504600F000FC04464846AE
:10A3880000F0E6FB85F80B8014E04FF47A70EFE7F5
:10A3980000F044FA00F0B2FB00F0BCFA49F6BA71DA
:10A3A800504600F0EBFB04461748001D00F0D0FBB8
:10A3B8000220E8721648046017491648C1F81005CB
:10A3C800286B40F4002028634FF0006030601021B3
:10A3D800C9F804130012306000F088FA0F49C1F878
:10A3E8004C800B480C300068A04204D340F26971DD
:10A3F8003E20F9F767FC21463846BDE8F04704F0EF
:10A4080001BA000004F5014000100040040E0020CD
:10A41800408500404081004098F0014000800040A5
:10A4280010B54AB1124C60726373D00707D0012A85
:10A4380005D040F63E110CE040F6371109E059B15D
:10A448000220A0722273012808D002280FD040F6FB
:10A4580055113E20F9F736FC0120F2E7E07A022890
:10A4680005D100F0DBF9BDE8104000F047BB10BD96
:10A47800040E00200A4908B5D1F81C21012A01D090
:10A48800002008BD074A126802F07F02524202709B
:10A498000020C1F81C01044800680090012008BD94
:10A4A80000100040481500401C110040044A036891
:10A4B800C2F812308088D08202F110000172704711
:10A4C800F40D0020044AC1781160006802490002B6
:10A4D80008390860704700002415004000680249E8
:10A4E80020F07F40086070473C15004010B500F030
:10A4F8007DFB06480068032801D00B2804D140F2F0
:10A50800A5213E20F9F7DEFB10BD000050150040E4
:10A518000149487670470000040E00202DE9F05FDD
:10A528006F4D0127EF646F48D0F800A06E480068AF
:10A538006E4CDFF8BC81C4E90E0A98F800000428C4
:10A5480002D34FF42D61C0E000F072F96949206B25
:10A558000860DFF8A4B100262663DBF8001240F299
:10A568001D129143CBF8001284F83460DBF80C011B
:10A5780000B9AF6400F0E0F905465A48001F0068CA
:10A588006062FFF7CFFD84F82800E07A84F829009C
:10A598005A492662022807D1607828B10A681278D9
:10A5A80002402078904311D02677DFF85491A8070D
:10A5B80002D5D9F800002062280702D5D9F8000092
:10A5C800206298F80000C00702D01CE02777ECE76B
:10A5D800D1F8008098F8000000F00F00072811D289
:10A5E800062208F10901A01C00F0DEFE38B9207A25
:10A5F80098F80010B0EBD11F01D1012000E0002035
:10A60800607700E066774FF000085146284600F072
:10A6180023FA18B9CBF810704FF00108334EE80749
:10A62800A6F1100602D03068804731E0A80726D589
:10A6380068071ED400F094FED8B900F081FEC0B9B6
:10A648002E48B4380068C0F34257C0F3006300F0E6
:10A658000F02C0F30311C0F3032053B10AB101B1D3
:10A6680038B92648B038006818B1032F01D245F030
:10A67800040545F380004146401C726807E015F068
:10A68800280F05D045F34011B2684046491C904751
:10A69800E80601D5F0688047E07A02281ED1207CC0
:10A6A80000281BD0022804D0012808D040F66631C3
:10A6B8000BE06169606A0144C9F800100AE0616A48
:10A6C8006069884204D840F667313E20F9F7FAFA03
:10A6D800C9F80000BDE8F05F00F01EBABDE8F09FC1
:10A6E800008000404C85004004B50040040E002066
:10A6F8008402002008F501400010004004150040C5
:10A708004485004070B5114B8C8803EB8003C3F877
:10A7180020460C78D1F8011044EA0121C3F800164C
:10A728000B4D296800F10806012404FA06F332B13A
:10A73800012A06D040F2F1413E20F9F7C3FA9943C5
:10A7480000E0194384400C432C6070BD00100040A9
:10A758004016004010B5044600F002FE00280ED056
:10A76800094A11685006022CD0F8200308D0C0F31B
:10A77800062000BF21F4FE4141EA0020106010BD10
:10A78800C0F30660F6E70000881500400D48407EDB
:10A79800252807D0262807D0272807D00A2807D831
:10A7A800042206E0022107E01A2105E0502103E017
:10A7B800062202EB4001C9B2034A116002494C313A
:10A7C80008607047040E002008150040124908B5BB
:10A7D80091F91820497E01280AD002280AD00428B5
:10A7E8000AD008280AD040F2D7310620F9F76AFAC9
:10A7F800002004E0012002E0032000E002206B4674
:10A80800F5F7D0FD18B14FF4A4613E20EEE79DF9AD
:10A81800000000F009FA08BD040E00200348817A00
:10A82800012902D1407BFFF7D1BF7047040E0020F9
:10A838000548C07A012803D0022803D103F060BF7D
:10A8480003F06ABF70470000040E0020094808B5ED
:10A858000021C0F80011C0F80C11C0F81011C0F8A0
:10A868000411C0F81411C0F81811034800680090CA
:10A8780008BD00000010004018110040164810B52F
:10A8880090F83400C10726D0810713D51348D0F8B3
:10A89800001241F00101C0F80012114800680B28AD
:10A8A80005D00A2803D0032801D0022813D140F28A
:10A8B8004B510DE040070ED508480A490830C1F849
:10A8C80014050948D0F84001012804D140F252513A
:10A8D8003E20F9F7F7F910BD040E002000100040E3
:10A8E8005015004098F0014000800040084801469B
:10A8F800427A91F8341012B1012A03D006E041F0EF
:10A90800020101E041F0040180F83410FFF7B6BFFE
:10A91800040E002010B500F023FD002808D100F037
:10A928000FFD002804D10348016841F4C0210160EB
:10A9380010BD00006815004038B5364D0024287C4D
:10A9480020B13548D0F84401012807D00022E97A1F
:10A958003248012904D002290AD019E00122F6E779
:10A96800D0F80C11012901D0002411E008240FE0CF
:10A97800D0F80C11012906D00021294B1B68012BA6
:10A9880003D0042402E00221F7E700240C43144317
:10A9980014F00B0F05D1D0F81011012906D00021B1
:10A9A8000C4320490978C90702D023E01021F7E7B2
:10A9B8001D49096811F0FF0F03D0D0F81421012AAE
:10A9C80000D0002285F82A2011F0FF0F03D0D0F81C
:10A9D8001801012800D0002085F82B0010481030FD
:10A9E800006885F82C00FFF757F8012800D00020F0
:10A9F80085F82D00FFF72AFFE00606D5200704D4C6
:10AA0800E87A012801D144F0200408480068009041
:10AA1800204638BD040E0020008000400010004091
:10AA28000014004084020020401600404481004089
:10AA3800084810B5006800F00F00032806D0042865
:10AA480006D040F236213E20F9F73CF9012010BD2E
:10AA5800022010BD101500402DE9F041254C0D468F
:10AA6800A27A9AB1217B8B0703D5830701D54307C7
:10AA78001CD4CB0605D594F82B3013B194F82D309F
:10AA8800A3B10B070BD5237F83B908E01A494FF010
:10AA98004060086000F068F80020207428E049074A
:10AAA80001D5617F11B110F0110F02D0FFF78AF9BB
:10AAB8001EE0012A01D0012600E00026607A012864
:10AAC8000ED0002700F050F89621304600F064F8C8
:10AAD80001464FB13B358D4204D90020BDE8F081D5
:10AAE8000127EFE701206072627B3046FFF71CFC0C
:10AAF8000120F3E7040E002008F501400548002175
:10AB0800C0F81C11D0F8001241F48871C0F8001286
:10AB180070470000001000400448016B41F48001B8
:10AB2800016303494FF4800008607047040E002059
:10AB380004F50140054900200860091F0860091F45
:10AB480008600249091D08607047000048850040F8
:10AB58000349497A002902D10249C1F8140570470E
:10AB6800040E002098F001400348002141728172D0
:10AB7800C172012101737047040E0020054A527A00
:10AB8800012A06D04FF47A7201F5FA71B1FBF2F19D
:10AB9800401A7047040E002070B5134C03460D464A
:10ABA80094F8292000205AB1214691F8281063B161
:10ABB800012B11D1012A284612D003F07BFE09E0AF
:10ABC80040F286713E20F9F77DF8012A284604D024
:10ABD80003F07EFE616A084470BD03F093FEF9E756
:10ABE80003F081FEF6E70000040E002010B50022F5
:10ABF800012908D0022904D04FF421713E20F9F729
:10AC080061F84FF0807205490A4305490A60054911
:10AC180008430349091D086010BD00000801100021
:10AC280014150040000003020149C0B208607047D3
:10AC38000C15004010B50749012805D0022805D099
:10AC480097213F20F9F73EF8032000E00420086030
:10AC580010BD00001015004070472DE9F0410D00AF
:10AC680004464FF002064FF0010708D02878D0B10B
:10AC7800012807D0022814D003283BD116E080F819
:10AC880020700EE06868C82803D30421F6F7B4FBE7
:10AC980008B1002607E02046696800F02AF9012675
:10ACA80001E0F5F7C7FB3046BDE8F08120780028C1
:10ACB800F7D16868F5F790FBE0B16968087828B1C2
:10ACC800A078052807D040F2791110E0204600F05E
:10ACD80018F96770E5E7204600F02BF9E07804F1F1
:10ACE8000C0100F00AF80028DBD140F27B116A2041
:10ACF800F8F752FD84F82070D3E7F6F7B3BD2DE9D5
:10AD0800F0410D4604000BD0267900270220092DBA
:10AD18007BD2DFE805F008102E2E5B647C97860056
:10AD280040F29311E2E0A07804286FD00328FCD009
:10AD38004FF4CF71DAE0A078042804D0032802D0B9
:10AD48004FF4D171D2E00520A07084F820702078EB
:10AD580080BB0021204600F0CCF8207B012804D0DD
:10AD6800A069E0610021A26841E0E078F6F75CFCA8
:10AD7800F7E7A178042904D0032902D04FF4E07141
:10AD8800B4E0227822B12146304600F0EEF8A4E083
:10AD9800042900D00120A070A268022D0BD0062142
:10ADA8003046904700286BD00078002868D04FF4D0
:10ADB800ED719BE031E0052130469047002871D0C5
:10ADC800007800286ED040F2D5118FE0A0780528D1
:10ADD80002D040F2E11189E00221A26807E0A078E0
:10ADE800052802D040F2E71180E0A2680121304630
:10ADF800904701462046FFF730FF02286DD0F0B398
:10AE0800012864D040F2272170E05DE067E0A07877
:10AE1800052802D040F2ED1168E0BDE8F041F5F7F1
:10AE280009BBA078052802D04FF4F9715EE0A2684A
:10AE38000A213046904701462046FFF70EFF40F2B0
:10AE4800F51153E0A178052906D062780AB10329E3
:10AE580002D040F2F91149E0217829B12146304663
:10AE6800BDE8F04100F081B894F8201089B184F869
:10AE78002070A070A26808213046904701E029E0C0
:10AE88002BE000280ED0007800280BD040F20521D6
:10AE98002CE0617859B1E07804F10C01FFF72DFF3F
:10AEA80010B16770BDE8F08140F209211EE0A07082
:10AEB800A2680721304690470028F3D00078002880
:10AEC800F0D040F2112111E040F216210EE00421E9
:10AED800A2688CE70321A26889E7002DE2D100F07F
:10AEE800F2F800680028DDD040F231216A20F8F736
:10AEF80053FC0246037B0069084410615938F7F790
:10AF08000FBB012202730022C2750A796AB10022BE
:10AF180082824A795AB1042282758A686A32026149
:10AF2800C96881610321817070472B22F0E70322F1
:10AF3800F2E710B5044600202073E075087980B167
:10AF48000020A082487970B10420A075C8686A30D2
:10AF580020618968E069F6F711FBA0610420A07000
:10AF680010BD2B20EDE70320EFE770B505460C4632
:10AF7800C878F7F7A9F878B1204600F010F8A26869
:10AF8800092128469047002808D00078002805D0D5
:10AF9800DB216A20F8F700FCD721FAE770BD002111
:10AFA800817001704170704770B5F5F79DFA0546DC
:10AFB800002406E02046F5F79DFAFFF7F0FF641C31
:10AFC800E4B2AC42F6D370BD2DE9F0410D46F5F779
:10AFD80091FA040007D0A0786FF02206012806D065
:10AFE800022810D103E06FF00100BDE8F0816FF096
:10AFF800150755B12846F5F7EFF930B1287830B183
:10B00800A078022808D03046EFE73846EDE7294611
:10B018002046FFF776FF03E029462046FFF789FF21
:10B02800E07804F10C01FFF768FE08B10020DCE7C6
:10B038004FF42B716A20F8F7AFFB10B50446F5F70B
:10B0480059FA010004D008786FF0220268B902E0CA
:10B058006FF0010010BD887838B1022807D00128A8
:10B0680005D001200870002010BD104610BD2046F4
:10B07800FFF77BFFF7E72DE9F0410E460746F5F7A6
:10B0880033FA054600240AE02046F5F733FA8078BB
:10B0980018B14FF0FF30BDE8F081641CE4B2AC4257
:10B0A800F2D3082E02D96FF01500F4E717B1314634
:10B0B800384601E000210846BDE8F041F5F700BA3E
:10B0C8000020F7F7A7BF0020F7F78ABF10B5F7F7FA
:10B0D80073FCBDE8104000F00BB8410A43F6095272
:10B0E8005143C0F3080010FB02F001EB50207047F9
:10B0F800410A43F609525143C0F3080010FB02F01D
:10B1080000F5807001EB50207047F6F7A1BA0028CF
:10B1180009DB00F01F02012191404009800000F185
:10B12800E020C0F88012704700280DDB00F01F02F5
:10B13800012191404009800000F1E020C0F8801111
:10B14800BFF34F8FBFF36F8F704770B50246002073
:10B1580000291DD0A2FB0101400A40EAC150490A5A
:10B16800401C41F1000140F2A172831841F1000135
:10B178005B1C41F100040021D3F1FF33A14103D24C
:10B1880071216D20F8F708FB00F5F460B0FBF2F0D0
:10B1980070BD4058002800D001207047D0F80C241A
:10B1A800D0F80C0402F00102C00303D58A4201D191
:10B1B800012070470020704710B501218807F8F773
:10B1C800A9FA002800D0012010BD4FF080400121CD
:10B1D800016070474FF08041D1F81824D1F8181455
:10B1E80002F00302C90303D5824201D1012070474E
:10B1F8000020704710B500214FF08040F8F78AFA18
:10B20800002800D0012010BD002809DB00F01F0233
:10B21800012191404009800000F1E020C0F880122F
:10B22800704700280DDB00F01F0201219140400902
:10B23800800000F1E020C0F88011BFF34F8FBFF30A
:10B248006F8F704700100200FA000000AC8A32CD00
:10B258000B6DDD090BD89484B72EF3BF0818D87B83
:10B26800002809DB00F01F020121914040098000FD
:10B2780000F1E020C0F880127047EFF3108172B639
:10B288000278012A01D0012200E000220123037084
:10B2980001B962B60AB1002070476FF0220070470A
:10B2A8000021017008467047EFF3108172B6002242
:10B2B800027001B962B600207047F8F759BB4FF029
:10B2C8008050D0F830010F2801D0002070470120AD
:10B2D80070474FF08050D0F830010A2801D0002084
:10B2E80070470120704700B5FFF7F3FF20B14FF01A
:10B2F8008050D0F8340108B1002000BD012000BD05
:10B308004FF08050D0F830010E2801D0002070474F
:10B31800012070474FF08050D0F83001102801D03C
:10B3280000207047012070474FF08050D0F830015E
:10B33800062803D0401C01D0002070470120704728
:10B3480000B5FFF7F1FF48B14FF08050D0F8340155
:10B35800062803D3401C01D0012000BD002000BDF9
:10B3680000B5FFF7E1FF38B14FF08050D0F8340155
:10B37800062803D3401C01D0002000BD012000BDD9
:10B388004FF08050D0F830010D2801D000207047D0
:10B39800012070474FF08050D0F83001082801D0C4
:10B3A8000020704701207047002A04BF0020704722
:10B3B800521E07D0037891F800C0634504BF401CB3
:10B3C800491CF5D000780978401A7047F0B480EA33
:10B3D800010C03461CF0030F3CD113F0030F0BD0F4
:10B3E800002A04BFF0BC704711F801CB03F801CB69
:10B3F800521E13F0030FF3D1032A4FD9B2F1004FB5
:10B408004CD2C2F1000C4FEAEC740CEB947C4FEA7E
:10B41800AC0CCCF1000CBCF1000F1BDD0D1F1C1F88
:10B428001CF0010F03D055F8046F44F8046F5FEA6D
:10B438006C0607D06F68676055F8087F44F8087F86
:10B44800761EF7D101EB8C0103EB8C03CCF1000CD9
:10B4580002EB8C02002A04BFF0BC7047B2F1004F27
:10B4680026D2002ADCBFF0BC7047491E5B1E12F0D2
:10B47800010F03D011F801CF03F801CF521004BF18
:10B48800F0BC704791F801C083F801C011F802CFF1
:10B4980003F802CF521EF5D1F0BC7047042AD9D365
:10B4A80051F804CB121F43F804CB042AF8D2D1E791
:10B4B80011F801CB03F801CB521EF9D1F0BC70474B
:10B4C80070B4034601F0FF0C10F0030F09D0002AF6
:10B4D80004BF70BC704703F801CB521E13F0030F72
:10B4E800F5D1C9B241EA012141EA0145032A39D916
:10B4F800B2F1004F36D25142CC1701EB947189104A
:10B508004E42002E11DD191F16F0010F18BF41F829
:10B51800045F741004D04D6041F8085F641EFAD1CE
:10B52800714203EB860302EB8102002A04BF70BC60
:10B538007047B2F1004F1DD2002ADCBF70BC7047C3
:10B54800591E12F0010F18BF01F801CF521004BFA5
:10B5580070BC704781F801C001F802CF521EF9D1C2
:10B5680070BC7047042AE0D3121F43F8045B042A16
:10B57800FAD2DAE703F801CB521EFBD170BC704750
:10B588004FF0FF30704700207047002070474FF0A1
:10B59800FF30704770477047002070474FF0FF300A
:10B5A80070474FF0FF3070470021017070474FF02F
:10B5B800FF3070474FF0FF30704700207047F8B5F4
:10B5C800044600F1030020F00300160000900D4629
:10B5D8008A78497800D00020F8F768FD0099084477
:10B5E8000090A97839B1EA8906B10020F8F7C4FFBC
:10B5F80000990844009032462946684600F007F84A
:10B608000098C01D20F007000090001BF8BD2DE930
:10B61800F04706460C4608784978002708449146C2
:10B6280000F0FF083D460EE0A379022B00D202236A
:10B638006279032A00D203222179E07800F04BFED8
:10B648006D1C0744EDB24545EED33068C01C20F0B0
:10B6580003003060B9F1000F00D000203A4641469F
:10B66800F8F7FCFE316808443060BDE8F08730B573
:10B678000D468DB01446014610226846FFF7A6FE17
:10B688001022294604A8FFF7A1FE6846F9F768F8D2
:10B6980018B16FF015000DB030BD1022204608A972
:10B6A800FFF794FE0020F6E7002070473EB50446F9
:10B6B800011D6846FAF73CFB002804D0694620467D
:10B6C80000F048F801203EBD0EB50146684600F07E
:10B6D80027F86846FAF756FB0EBD10B50446204613
:10B6E800F8F7D0FB002806D0A178207800F004F8FD
:10B6F8000028F4D0012010BD70B50C460546F8F7B7
:10B7080035FC002802D03E2D01D0012070BD122C3E
:10B7180004D02046BDE87040F8F744BC002070BD56
:10B728000A88C2F30B0202804A8842804A78930949
:10B73800002242714B78C3F301131BB1012B05D0D2
:10B74800022B05D00271091D816070470122F9E7BB
:10B758000222F7E710B50C4609780170417821F00C
:10B768000F0141702288C2F3032211434170A2786D
:10B778008270628821F03001120AC2704170227909
:10B7880002F0030241EA021121F0C001417062791E
:10B7980041EA82114170A168021D914206D0628877
:10B7A800FB2A00D3FB22001DFFF710FEA078001D26
:10B7B800C0B210BD2DE9F04104460F7800200C25D9
:10B7C80005263E22FF231B2F7DD2DFE807F0EB0E74
:10B7D80025272D636D819BAFB1BCC7E2F5EBEB313B
:10B7E800D2D5FEF2F1F0EFEEED0025700879A070E9
:10B7F8004879E070B1F80500000A2071C8796071D5
:10B80800087AA0710889000AE071887A207248894C
:10B81800000A60720820C2E0102000E01A202070A0
:10B828000879A0700120BAE0204600F047F9B4E09A
:10B8380022700A20A07011F8040FE0708878207137
:10B848004888000A60710879A0714879E071D1F8D8
:10B858000600A0604889A081C868C4F80E00088A5C
:10B868006082D1F812006061C88A2083087EA076C1
:10B87800088B000AE076887E2077488B000A60777C
:10B88800087FA077888B000AE077887F84F82000FB
:10B898001F2084E022701420A0700879E070888846
:10B8A800000A20718879A8E022700420A070087925
:10B8B800E07088792071C888000A60718868C4F8C7
:10B8C8000600C86800E06DE0C4F80A000C2066E0D5
:10B8D80022700320A0700879E07088792071C888E8
:10B8E800000A6071087AA0710889000AE071887AF4
:10B8F80020724889000A6072087BA0728889000A51
:10B90800E072D9E02270A6700879E0708888000A91
:10B918002071D1F80600C4F80500D1F80A00C4F86F
:10B928000900C889A4F80D000D2038E0112044E072
:10B9380026700879A0704879E070B1F80500000A0F
:10B948002071C87959E0082020700879A07088799A
:10B95800E070C888000A2071087A4EE03020207014
:10B968000879A0708879E070C888000A20710320DF
:10B9780015E02270072045E02270A5700879E07074
:10B9880088792071C888000A6071087AA071487A9D
:10B9980028E02046091DF8F7BBFA002802D060709D
:10B9A800801CC0B2BDE8F08173E047E028E053E0B6
:10B9B80061E01AE009E0FFE7572020700879A070DD
:10B9C8008888000AE0700220E9E722701220A0703F
:10B9D8000879E0704879207188796071C888000A10
:10B9E800A071087AE0710620D9E72370A120A07021
:10B9F8000879E07048792071002060710420CEE752
:10BA08002370A220A0700879E0708888000A20714D
:10BA180088796071C888000AA071087AE07108897D
:10BA2800000A2072887A60724889000AA072087B2E
:10BA3800E0728889000A20730B20B0E72370A320E6
:10BA4800A0700879E0708888000A20718879607190
:10BA5800C879A0710520A2E722701320A070087988
:10BA6800E07048792071D1F80600C4F805004889CB
:10BA7800A4F8090020E02370A420A0700879E070E1
:10BA88008888000A207188796071C879A0710720B8
:10BA980085E723708020A0708A88A4F80320CA88CC
:10BAA800A4F805200A7AE2714A7A22818A7AA27277
:10BAB800C97A01F00101E1720A2070E73E220270A2
:10BAC800012282700A79C2708A790271CA88120AC0
:10BAD80042710A7A82714A7AC271D1F80A20826068
:10BAE800CA8982810A7C82730A8A120AC2738A7C92
:10BAF80002744A8A120A42740A7D82748A8A120A75
:10BB0800C274897D0175132070473E22027001229C
:10BB1800827011F8042FC2708A7802714A88120A5A
:10BB280042710A7982714A79C271D1F8062082601D
:10BB38004A8982810A7E82730A8B120AC2738A7EBC
:10BB480002744A8B120A42740A7F82748A8B120A20
:10BB5800C274897F0175132141700846704710B57A
:10BB680020B1FFF7A3FD20B1002010BD6FF0150034
:10BB780010BD6FF0220010BD10B56FF0150420B194
:10BB8800FFF7A2FD08B1002010BD204610BD10B57A
:10BB980020B1FFF7A2FD20B1002010BD6FF0150005
:10BBA80010BD6FF0220010BD02F059BA02F09BBA26
:10BBB80010B5F8F70BFA002010BD10B5F8F714FA15
:10BBC800002010BD02F0ABBA08B500788DF800006F
:10BBD800684602F0DFF908BD01207047FDF792BC06
:10BBE80001207047007800B1012002F047B902F047
:10BBF80047BAFDF795BC01F05EBF01F073BF01F0D5
:10BC08007BBF02880A8001F080BF02880A8001F0A9
:10BC180095BF01F0BDBF01F0C1BFFDF711BCFDF735
:10BC280019BCFDF739BC01F0C2BF01F0C9BF01F072
:10BC3800CBBF01F0DEBF02F018B802F049B810B56A
:10BC4800F8F7BEF9002010BD02F0D4B802F0E0B851
:10BC580001F0E1BE02F020BA70B50B88047F00F154
:10BC6800240523F4004602883544A41D2D88224467
:10BC780092B22544541E2C4494FBF2F402FB046255
:10BC8800408892B2904203D903F40040104302E086
:10BC98004FF400409843088070BD20F4004221F41E
:10BCA80000439A4207D100F4004001F40041884261
:10BCB80001D0012070470020704770B5007F1C46F6
:10BCC800801D084413460988049AC91C89B21519AD
:10BCD800C01E8D4205D8811822461846FFF776FB0C
:10BCE80000E00024204670BD70B5007F1C46801D12
:10BCF800084413460988049AC91C89B21519C01E3C
:10BD08008D4205D8104422461946FFF75FFB00E034
:10BD18000024204670BD8188C088884201D1012056
:10BD280070470020704781880089884201D101202E
:10BD380070470020704770B5044600F124018088E0
:10BD480020F400400144208A00281AD0A289002546
:10BD5800104480B2A0810A88904205D94FF4A57199
:10BD68004FF01400F7F7AEFF09D1A06908B1407F82
:10BD7800887004F104012046FFF76EFFA581258233
:10BD8800012070BD2DE9F041044600F12403C0886C
:10BD98000E4620F40047608AD91908B1B04202D291
:10BDA8000020BDE8F081E089002540B1B1F800C06D
:10BDB800604508D040F21F211420F7F783FF607F09
:10BDC80088700D800EE094F81CC018440CF1060C25
:10BDD800BC446044B4F81EC020F803CC94F820C0DA
:10BDE80000F801CCE0893044E081088830440880BC
:10BDF8006AB1A11D2046FFF72FFFE581607F401C37
:10BE08006077A07D08B1E088A082A5750BE0207F4F
:10BE1800E189801D38441944084430F8031DE18342
:10BE2800807884F820006582E5750120B9E710B5AF
:10BE38000446C088A188814207D0A08928B9208AF1
:10BE480018B9A088A18A884201D1002010BD211DFF
:10BE58002046FFF701FF00202082012010BD10B509
:10BE6800044600F12402C08820F4004002442088DF
:10BE7800452800D24520884204D24FF4807114200E
:10BE8800F7F720FFE07D002803D01088884201D210
:10BE9800002010BD1180A11D2046FFF7DDFE002007
:10BEA800E075012010BD2DE9F041418986880446DE
:10BEB800002500F10A0706E039462046FFF7CCFEC8
:10BEC8006D1C6189ADB2B142F6D12846BDE8F0815A
:10BED80030B5C488818800F1240221F4004313445A
:10BEE8008288858AAA4212D0A14210D0818971B96C
:10BEF800826972B11046FFF716FF50B910892432D3
:10BF080020F40040104499788078884201D10020BC
:10BF180030BD184630BD007F801D0844C01E10602B
:10BF2800088870472DE9F0410E46C1880289044609
:10BF380000F12408008821F4004522F40047452830
:10BF480000D24520B04203D2C2211420F7F7BAFE2E
:10BF58001046FFF7A2FE10B10020BDE8F081AF4205
:10BF680008D9217F781B401A801F864202DD0020F5
:10BF7800E075F1E708EB050001210680E175ECE7C3
:10BF880038B5C488818800F1240221F400431A449A
:10BF9800A14210D08389058A12882B44934208D382
:10BFA800ADF800106946FFF757FEBDF80000A04243
:10BFB80001D0012038BD002038BD70B5C6888588FD
:10BFC800034600F1240425F400402044B54202D180
:10BFD8000020188270BD04889D891E7F641B35442B
:10BFE80028440D88A4B2C01CA54200D90C809C89A5
:10BFF80024B1002414700988198270BD0124F9E75E
:10C0080010B5818AA1F57F42FF3A02D0827D52B9EC
:10C0180004E040F255311420F7F754FE808881423D
:10C0280001D1002010BD012010BD4FF6FF718182A3
:10C0380000218175704710B5818AA1F57F42FF3ACA
:10C0480004D04FF44E711420F7F73CFEC18881826A
:10C05800C18901B10121817510BD2DE9F0411D464D
:10C068001646069F0B4604463A462946304600F0D7
:10C078004FF8834201D2A12118E0E01C20F003010F
:10C088002046A14201D0A22110E024220021FFF77E
:10C0980017FA4FF6FF70A082A819801D784380B266
:10C0A80025776080B0F5004F03D9A8211420F7F751
:10C0B80009FE268000206077BDE8F08181618861F3
:10C0C80070472DE9F0410B46044600F1240105892B
:10C0D8004689808825F4004739440F46854202D1B5
:10C0E8000020BDE8F0810AB1C81C106023B1227F8E
:10C0F800F91C1846FFF76AF93F8804F10801204641
:10C10800FFF7AAFDB54201D1208960813846E8E7EA
:10C118000144891D51438AB20021452801D2C0F14A
:10C1280045012432501880B270472DE9F0478846FF
:10C13800C1880446008921F4004604F1240520F44E
:10C14800004705EB0609FFF7A8FD002298B92088EB
:10C15800452800D24520B74206D9237FB91BC91A02
:10C16800891F814200DA0846E18911B1B9F8003027
:10C17800C01A404503DA62820020BDE8F087207FBC
:10C188002944801D30440844A4F81280C01EF4E7F6
:10C198000021C1814182C1758175704770B5002346
:10C1A800082904D240F2CB111520F7F78BFD02685D
:10C1B8000AB91EE01046026893888B4202D01368C1
:10C1C800002BF7D1948813468C4201D111680DE0F9
:10C1D80001F10805AEB20025B44209D3641A11442E
:10C1E8000D608C800268126802600A60016000E0DD
:10C1F8000023184670BD10B50C0006D0082C09D2D3
:10C2080040F295111520F7F75DFD08B10021016096
:10C21800002010BD18B1A1B2006800F014F8201D6C
:10C2280010BD0021026803E093881268194489B29E
:10C23800002AF9D100F007B800230B608A80026851
:10C248000A600160704700234360021D018102609B
:10C258007047A0F57F43FF3B01D0022901D300209E
:10C268007047F7F7E3BF0EB5694600F018F820B13C
:10C278004FF4B2711720F7F725FD6846F7F754FF1A
:10C2880008B100200EBD01200EBDA0F57F42FF3A87
:10C2980001D0022901D300207047F8F701B870B522
:10C2A80005460C46084600F064F808B1102070BD39
:10C2B800022D01D3072070BD25700020608070BD5D
:10C2C80010B50446F8F738F8A04201D9012010BD8E
:10C2D800002010BD704770B50E461D46114600F08F
:10C2E80011F804462946304600F003F82044001DA2
:10C2F80070BD10B50A460121FFF70AFFC01C20F0E7
:10C30800030010BD10B50A460121FFF701FFC01C4C
:10C3180020F0030010BD10B50B680446002B0DD0AB
:10C32800CA8819462068FFF787FF2079012802D1BB
:10C338002068FFF776FF2079401E207110BD002885
:10C3480009DB00F01F02012191404009800000F143
:10C35800E020C0F880127047F8F702BA4FF0804129
:10C368000020C1F808014FF0E0210120C1F80001C8
:10C37800704708B10020704701207047F8F736BBB6
:10C38800F8F724BB10B5002904464FF0060102D087
:10C39800F7F710FD01E0F7F729FD607920F0C000FC
:10C3A800607110BD704730B50C4605468DB04FF032
:10C3B800030104F1030012B1F7F7FCFC01E0F7F701
:10C3C80015FD60790D2220F0C00040F0400060713A
:10C3D800002104A8FFF774F8E0788DF81F00207991
:10C3E8008DF81E0060798DF81D00102229466846D8
:10C3F800FEF7ECFF6846FFF7AFFF9DF82F002070AF
:10C408009DF82E0060709DF82D00A0700DB030BD15
:10C41800F8F782BEC10701D001207047800701D517
:10C42800022070470020704710B5012808D0022864
:10C4380004D040F297310620F7F744FC012010BDE4
:10C44800002010BD002904D0012803D0012901D003
:10C458000220704701207047FFF7AFBD0122F9F7AE
:10C468006FB910B502F03AF918B1BDE81040FDF700
:10C47800FFBAFF2010BD10B5F9F7ACF9102803D0AA
:10C48800F9F778F9102800D1082010BD10B5F9F790
:10C49800A1F9102803D0F9F7E5F9012010BD002013
:10C4A80010BD70B50E468CB0144601461D461022CC
:10C4B800684600F00CF91022314604A800F007F98C
:10C4C8006846FFF749FF08A94FF0100228461CB13B
:10C4D80000F0FDF80CB070BDFEF778FFFAE710B574
:10C4E8000C460021FFF7D1FE606018B101202070D2
:10C4F800002010BD022010BD40F2E24148437047C1
:10C5080040F2E241B0FBF1F080B2704770B50446EA
:10C5180090420BD2101B642800D2642025188D424B
:10C5280003D80421F4F768FF08B1204670BD2846F7
:10C5380070BD10B5A2F10F030C2944D2DFE801F059
:10C5480006080D1215181C2427412A31C2B33AE0F7
:10C55800072A3AD0082A38D035E00C2A35D00B2AD9
:10C5680033D030E00D2A30D02DE00C2B2DD92AE025
:10C57800103A0B2A29D926E0032B26D990F8440033
:10C5880008B31B2A21D91EE0042A1ED01BE0062A64
:10C598001BD018E01C2A18D01D2A16D01E2A14D029
:10C5A80011E01F2A11D0202A0FD0212A0DD0222ACB
:10C5B8000BD0232A09D0242A07D0262A05D002E046
:10C5C80003E00E2A01D0002010BD012010BD0C2868
:10C5D80013D00B2811D00D280FD01F280DD02028DC
:10C5E8000BD0212809D0222807D0232805D02428B9
:10C5F80003D0262801D0002070470120704711F091
:10C608000C0F16D04A074FF41671002A02DA4FF0C1
:10C61800100201E04FF0400201DA4FF0960101F5F7
:10C62800BC71A0EB0103884210D993FBF2F080B2F1
:10C638007047022902D070280AD807E03C2805D99B
:10C648003C38C11700EB91708010F0E70020EEE74E
:10C658007038C11700EB5170C010E8E70968C0F8DE
:10C668005E10704710B540F6C412012906D00229A1
:10C6780005D040F229412920F7F724FB08B11046DC
:10C6880010BD40F2E24010BD2DE9F0410C460546D0
:10C69800C668F5F79FFA98B1BCB13046E968F4F777
:10C6A8009FFF002811DD2044401EB0FBF4F707FB74
:10C6B80004F13046F4F762FFE8603846BDE8F081DF
:10C6C80040F2AE212920F7F7FDFA0020F6E730B551
:10C6D800134606E0CC18D51A14F8014C5B1E4455D5
:10C6E800DBB2002BF6D130BD38B505460C4668469E
:10C6F800FDF7C0FE08B39DF90000607294F823109E
:10C70800A17294F90B100022411A00D54942EB7F1F
:10C718008B4210DCFF2B0ED0217B491CC9B2217340
:10C7280095F82030994202D8E17A7F2903D1E07246
:10C73800002020730122104638BD7F20607200203F
:10C7480038BD00238362028640F271235A4301EB0D
:10C758000212521EB2FBF1F1C162704740F2E2418F
:10C768004843704740F2E24110FB01F0704710B5B2
:10C7780000231A4603E0845C2343521CD2B28A4247
:10C78800F9D30BB1002010BD012010BD70B58B7816
:10C798000C78C57A6340CC7849784C4043EA042346
:10C7A80083EA02010022CCB2090A94FAA4F491FAAD
:10C7B800A1F1240E090E44EA012101EB0111521CDA
:10C7C8001944D2B289B2032AEDD359402522B1FBCC
:10C7D800F2F302FB131200EBD20302F007065B78B8
:10C7E800012404FA06F6334201D0104670BD4D43C9
:10C7F800290C491CC9B20023C518AA798A4211D349
:10C808006D78002204FA02F6354201D0491EC9B2F9
:10C8180021B1521CD2B2082AF4D305E002EBC300BE
:10C82800C0B270BD891AC9B25B1CDBB2052BE3D359
:10C838004FF487714620F7F745FA10B5044690F88B
:10C84800200008B1252801D9122010BD2AB1607D29
:10C8580028B1012809D01F2010BD002010BD204696
:10C86800BDE810401146F9F7D3B8A28804F11500C5
:10C878000C31FFF78BFF84F82300EEE730B5421C3C
:10C888008A4204D00A68C0F80120097941714179C7
:10C8980001F01F0141710021C1724318491C5C78E5
:10C8A800C9B204F00102640804F0010515446208E5
:10C8B80002F001042C44520802F001052C445208ED
:10C8C80002F001052C44520802F001052C445208DC
:10C8D80002F001052C4404EB52029A71C37A05292F
:10C8E8001A44C272D9D330BD70B5B0F80720B0F879
:10C8F800095030F8054F10F8013CC08831B1B2F545
:10C90800506F03D940F607518A420BD9911F40F660
:10C918007A46B1420ED86BB1082B0BD8934209D294
:10C92800944207D8B5F5FA7F04D2B0F5486F01D81C
:10C93800012070BD002070BD42680A60007A08714D
:10C948007047B0F809007047B0F807007047B0F8B2
:10C9580009007047B0F80B0070478089088070475D
:10C96800D0F816000860704742680A60806848601E
:10C97800704750F80E2F0A60406848607047426858
:10C988000A60806848607047007800F003007047CC
:10C99800007970470079704710B5FB2904D940F237
:10C9A8005B512A20F7F78EF9417010BD0079704766
:10C9B80040797047017170474171704710B51B2A63
:10C9C80004D940F2C2312A20F7F77CF94270BDE859
:10C9D8001040C01CFEF7FABC0968C16070470A68BD
:10C9E80042604968816070470A68426049688160AE
:10C9F80070470A684260496881607047027801F0B0
:10CA0800030122F003020A43027070470171090A08
:10CA1800417170478171090AC17170470172090A31
:10CA2800417270478172090AC172704770B5027805
:10CA380002F00F02032A2CD0052A2DD1B0F81920B4
:10CA4800B0F81B50B0F81740837D41B1B2F5506F74
:10CA580005D940F607518A4201D8012100E000219A
:10CA68004678222E18D159B9911F40F67A46B1421C
:10CA780012D88BB1082B0FD893420DD294420BD801
:10CA8800B5F5FA7F08D2B0F81D00B0F5486F05D9A2
:10CA980002E040780C2801D0002070BD012070BD54
:10CAA80070B5144605461F2A03D9B2212A20F7F784
:10CAB80009F905F10900FEF789FCA41D6C7070BD29
:10CAC80010B5027801F00F0322F00F021A4302702A
:10CAD80007290CD2DFE801F0040604060408040064
:10CAE800062102E00C2100E02221417010BD6E21D8
:10CAF8002A20F7F7E7F80A6840F8092F8988818023
:10CB08007047027822F0800242EAC1120270704730
:10CB18000A6840F8032F898881807047027840238B
:10CB280022F0400203EA81110A430270704770B58F
:10CB3800144605461F2A03D9D4212A20F7F7C2F83C
:10CB480005F10900FEF742FCA41D6C7070BD0121BF
:10CB580000F053B84168002291F8FA30002B04D055
:10CB680081F8FA20406800F074BC70472DE9FC4158
:10CB78000E46A0F57F411746FF3914D030800021BA
:10CB88007171F7F7B3FC0446FFF7A2F905000AD064
:10CB98002046294601AAFFF7BEF9708030B1FB286C
:10CBA80006D9C92126E00020BDE8FC81C82121E082
:10CBB8000198FFF7E9FE012803D0022801D0D82107
:10CBC80018E0307129467388032520463A460095B7
:10CBD800FFF773F82046B760FFF729F938B100214D
:10CBE80020460A46FFF76DFA18B10120DCE7E82174
:10CBF80000E0ED212B20F7F765F82DE9FC4104460C
:10CC08000E460020F7F744FA0546002016B9012021
:10CC1800F7F73EFA0026B0462F1817E02088401C88
:10CC280080B22080B84202D34046A4F8008080B287
:10CC3800A84204D3B84202D20020BDE8FC8169466C
:10CC4800FFF74DFC0028F8D0761CF6B2B742E5D8BD
:10CC58004FF6FF7020801220EFE770B550800C89E6
:10CC680094808B89D38048891081CD895581CE8D58
:10CC7800AE4208D14D8D854205D10D8E9D4202D11F
:10CC88008B8DA34201D0012300E000231373488554
:10CC98005089C88590888885D088088601201070BA
:10CCA80070BD10B58C880A894B88C988A0F84030B7
:10CCB800A0F84410A0F84240A0F8462010BD70B576
:10CCC80015460C4600F0AEF896302844A04201D82C
:10CCD800201A70BD002070BD2DE9F0470446C78DAD
:10CCE800468EB0F84450008F854200D30546204652
:10CCF80094F8631000F088F80146E5856186A28EF5
:10CD080004F12400E38E8046AA4200D22A468B42D0
:10CD180000D20B460282A8F81230BD4201D1B142BE
:10CD280001D0012000E000208146B4F84050608F17
:10CD3800A78D268E854200D3054694F862102046BA
:10CD480000F069F894F85810022908D1AF4200D2CF
:10CD58003D46864200D23046002184F85810A8F893
:10CD68000850A8F80C00BD4201D1B04201D0012002
:10CD780000E0002040EA0900BDE8F0872DE9F04115
:10CD880016460F46044600F04DF805463A466168D7
:10CD9800606A00F034F8A919814200D30846A062FD
:10CDA800BDE8F0811B2202848283C2828282428192
:10CDB8000282028142858285828400290AD14FF449
:10CDC800A4714184C18341830183C18141828181EE
:10CDD800C18501867047006801F19C02904203D921
:10CDE800401A9C384008704700207047022903D039
:10CDF800C000703080B2704780003C30FAE788424B
:10CE080000D30846801A7047B0F84610808F8142D8
:10CE180000D208467047B0F84210C08F814200D255
:10CE280008467047962190F8633090F8622000F029
:10CE380000B82DE9F0410D46064698461746808D04
:10CE48001146FFF7D3FF044639463046FFF7E3FFA4
:10CE5800A04200D20446B08E4146FFF7C7FF0746FE
:10CE680041463046FFF7D0FFB84200D33846204449
:10CE78002844801DBDE8F081012802D14879800945
:10CE880001D00020704701207047012806D1487959
:10CE98000121B1EB901F01D101207047002070479C
:10CEA800022803D0032801D00020704701207047D2
:10CEB80010B50446007CFFF7F3FF48B194F84F0023
:10CEC80004F15001FFF7D7FA082801D0012010BD5E
:10CED800207C18B1022801D0E07D10BDBDE81040CB
:10CEE8000020F7F7BDBD08B590F878108DF8001050
:10CEF800009900919DF8001009B1012008BD90F833
:10CF08009A008DF80000009800909DF8000000201D
:10CF180008BDFF200870704770B50D460446E8222A
:10CF28000021FEF7CDFAFF2020707F2084F826002C
:10CF3800132060802846F7F76FFBE062022084F830
:10CF4800740084F875000020A07304F12000BDE887
:10CF5800704000F0A0B98078C0F3800008B10020CC
:10CF680070471F207047F9F7F1BC806870470120AF
:10CF7800704710B50446203000F04DF96188BDE8CF
:10CF880010402822F9F79EBE0022826243881D2B9A
:10CF980001D0417370474273704790F875200021A3
:10CFA800022A04D1B0F8700008B1012000E0002086
:10CFB800814381F00100704700207047807800F0BD
:10CFC800010070478078C0F3C000704701207047A7
:10CFD8008078C0F34000704790F90E0070470078E1
:10CFE800FF2801D001207047002070470A6840F8E8
:10CFF800112F89888180012181717047007B7047DA
:10D0080001207047C161704790F8742002B1012275
:10D01800002380F8743019B1D0E91930C1E9003023
:10D0280010467047022180F874107047D0E9192023
:10D03800C1E900207047012280F87420D1E900215D
:10D04800C0E91921704790F8752002B10122002328
:10D0580080F8753019B1D0E91B30C1E900301046AD
:10D068007047022180F875107047D0E91B20C1E98C
:10D0780000207047012280F87520D1E90021C0E91D
:10D088001B21704780F86010704770B5044680789F
:10D098000125C0F3C00038B13C23FF222046E169D6
:10D0A800F9F77AFC84F8785084F8615070BDC07B39
:10D0B800002800D00120704710B5FFF7DCF90446BE
:10D0C800F8F7B2FA38B12046F8F756FA18B1102135
:10D0D800FFF74DFB08B1002010BD012010BD012154
:10D0E800F9F7CAB80121F9F7C7B82DE9F0410446A4
:10D0F80000274F7011200D460870202204F17A0194
:10D10800281DFEF763F901262E7284F878702879B5
:10D11800002811D1E888A4F8A400E06990F87D10EF
:10D1280084F8A61084F8A2600088F7F7DFF9FEF704
:10D138007CFFE06980F86860BDE8F0812DE9F04186
:10D1480004460F46407EF8F7FDF90646207E04F1B6
:10D15800490520B11EB1607EF8F7E8F9A0B194F84E
:10D168006200002824D0A07E002821D094F848002E
:10D178002946FFF78AFEA8B1F8F7D4F93A462946B6
:10D18800BDE8F041FFF70FB9012084F848003A469E
:10D1980029463046FFF707F9617E2846BDE8F04189
:10D1A800F8F7DCB939462846BDE8F041FFF7EAB898
:10D1B800BDE8F08110B504460846FDF7A9F92179C4
:10D1C800BDE81040252001F01BBB10B504462630F1
:10D1D800FDF750F9002802D17F2084F8260010BD01
:10D1E8000278202322F0200203EA41110A43027048
:10D1F800704770B50170427014460D46807800F093
:10D208007FF810FB05F06043FF2803D35C212E2034
:10D21800F6F758FD70BD10B50446807800F070F838
:10D228006178227811FB02F14843C0B210BD10B5F5
:10D23800044600F04DF86179491CC9B26171627801
:10D2480091420BD100226271E1780143E170A37829
:10D25800994203D1E2702179491C2171BDE810403F
:10D2680000F025B88170704770B50446807800F0EA
:10D2780047F8617811FB00F5E07800F041F8617833
:10D28800627910FB012021782279891A11FB05F1B6
:10D29800081AC0B270BD002101608180012141706F
:10D2A800017070470021C17041710171704710B55C
:10D2B800012807D0022807D0042807D039212E20BA
:10D2C800F6F700FD252010BD262010BD272010BD33
:10D2D800014600208A78D30702D0CB78DB0706D036
:10D2E800930706D5CB789B0703D40220704701200B
:10D2F80070475207FCD5C9784907F9D4042070470C
:10D30800C0F38001C0F34002114400F0010008445A
:10D31800704740F25A314843704740F2EF20704757
:10D328000E021C043006600C5A03B406C505F50B42
:10D338002512A301B103BF05EF024906A30910B5E1
:10D3480090F8E41009B1002010BDD0F8E01049B9F8
:10D3580090F8BC1031B1D0E930128A4202D9FFF7F7
:10D3680094FEF0E7012010BD10B531B1012908D0B5
:10D3780040F2A3713020F6F7A5FCBDE8104000F09C
:10D3880099B9002180F8BC1000F05DF9BDE81040A3
:10D39800FCF750B810B5044690F8C800002819D01A
:10D3A800012084F8E40001462046FFF76BFE94F85C
:10D3B800C80070B114F8B40FF4F76AFD2078F4F7D8
:10D3C800A5FE14F8B409F4F77FFE20B1002084F814
:10D3D800C800002010BD40F217213020F6F772FC7B
:10D3E800D0F8B800704790F8C80070470EB5694685
:10D3F8000120FEF754FF38B140F245113020F6F70E
:10D4080061FC0298FFF7C6FF6846F6F78DFE002814
:10D41800F7D0F9F7DFFD00200EBD0EB569460120F3
:10D42800FEF73DFF50B140F2AE713020F6F74AFCEE
:10D43800029890F8C80008B100200EBD6846F6F7BB
:10D4480073FE0028F4D00020FEF70DFF80F00100E5
:10D458000EBD7CB5044690F8FB00002853D194F823
:10D468002C0103284FD1FDF731FE0146D4F85401B1
:10D47800F4F7B6F8002846DD616811B1B0FBF1F0A9
:10D4880000E00020B4F86C10401C0844A4F83C01EB
:10D49800B4F83C01B4F8F410081A00B2002832DDE0
:10D4A80094F86001F4F7F4FC00282CD0012084F8EB
:10D4B8004101B4F89E00B4F89C1001AE401AB4F8CB
:10D4C8006C10401E084485B217E00096B4F83C1171
:10D4D800002301222046F9F7AFFE002813D00128C7
:10D4E80004D040F215613020F6F7ECFBB4F83C01AB
:10D4F800BDF804100844A4F83C01B4F83C01281A0B
:10D5080000B20028E1DA7CBD0020704770B50446FF
:10D51800012600F0B3F8A4F8D400002084F8CC0069
:10D52800012084F8D70094F8BC0004F1CC0560B160
:10D538004FF47A71D4F8D800F4F720F8C4F8D8007A
:10D5480000212846FFF7A0F80FE02046FFF70DFD61
:10D5580006463146D4F8D800F4F710F8C4F8D800D5
:10D5680031462846FFF790F8461CB4F8DC00411C09
:10D578000A2902D23044A4F8DC00D4F8B80030B14B
:10D58800B4F8DC00401C0A2801D3022000E0032084
:10D5980084F8D6000021204600F024F830B1204657
:10D5A80000F011F8BDE87040FBF744BF94F8B400F0
:10D5B800294600F061F8002804D140F2B661302015
:10D5C800F6F780FB70BD10B5044614F8B40FF4F7F5
:10D5D8007BFD0020207510BD10B5FFF7CAFC00F2D6
:10D5E800071010BD70B5044690F8E4000D4608B168
:10D5F800012070BDD4F8E000A8B12046FFF7B5FCC3
:10D6080005442046FFF7E8FF4119D4F8E0008842B6
:10D6180006D20120C4F8E0002046FFF736FDE7E710
:10D62800401BC4F8E000002070BD10B5044690F817
:10D63800630000F04BF902462046BDE8104040F276
:10D648001711FFF79BBB10B5FCF7A6FDBDE810400E
:10D65800F4F78CBE70B50C46054601F0C1F84AF2E5
:10D66800A13108444FF47A71B0FBF1F6284601F075
:10D67800A9F83044204470BDF4F7F4B810B5044656
:10D68800FFF7A4FCA0B12046FFF798FC18B9204684
:10D69800FFF79EFC20B1492401F060F828B901E0A9
:10D6A8004224F9E701F050F800B1E41D204610BD0E
:10D6B8006B2010BD70B5044690F8B500002518B170
:10D6C800012000F08AF805462046FFF74EFC411974
:10D6D800D4F8D800CC34F3F751FF0026E06004F802
:10D6E8000B6B012004F80109032004F8D609204631
:10D6F800FFF7C4FFA4F8D40029462046FFF772FFBD
:10D7080030B994F8B40004F1CC01FFF7B5FF38B193
:10D71800A4F8DC60FFF797FFBDE87040FBF78ABE0E
:10D7280040F204713020F6F7CDFA10B50446002017
:10D7380084F82C0194F86001F4F7C6FC202084F8E2
:10D74800600110BD2DE9F843002580F8BC50D0F8E1
:10D75800D8608846044680F8C850012780F8C97008
:10D76800D0F8B8003946B434F8F7C0F86068C0F8A3
:10D7780054616168207881F860016168C1F864814A
:10D788006068C0F85861646884F82C510023A4F8D4
:10D798005C511A46194620460095F9F74DFD20B10F
:10D7A80040F22B213020F6F78DFAC4F82851C4F83E
:10D7B800205184F82C71A4F83E51A4F83C5184F807
:10D7C800415134F86C0F401E24F8BC0BE586FFF776
:10D7D8003AFFBDE8F843FBF72DBE08B500284FF027
:10D7E8000101684602D0F6F7E5FA01E0F6F7F0FA2B
:10D7F8009DF8000042F210710002B0FBF1F201FB4B
:10D80800120008BD10B5040008D009295CD2DFE871
:10D8180001F007363E3E3A5B434A57009E2150E0EE
:10D828000021C4F8681194F84011204689B1B0F875
:10D838003E21B0F86C108A4206D1B0F8F420511A93
:10D84800A0F8F61011460DE0511AA0F8F61091B2A2
:10D8580008E0B0F83C11B0F86C20891AA0F8F6106E
:10D86800B0F83C11A0F86C10D0F85011C0F8541161
:10D87800FAF7B8F92046BDE81040F9F74DBFBDE802
:10D88800104000F079B8BDE81040FCF747BE2046CC
:10D89800BDE81040F9F776BF0120F3F79DFDBDE81C
:10D8A8001040FEF7B5BD94F82C01042801D0C02122
:10D8B80007E02046FFF739FFBDE81040FBF7BABD87
:10D8C800C9213020F6F7FEF9CD21FAE710B500F0AE
:10D8D80087FF4DF6417108444FF47A71B0FBF1F0BF
:10D8E80000F5BA7010BDF401FA00960064004B0010
:10D8F80032001E0014000A0005000200010000EBBF
:10D90800D10001F007030278012199408A4302708F
:10D91800704710B50446D0F894016168884209D16F
:10D92800B4F898112289914204D1B4F89A11628905
:10D93800914213D02188A4F8B411FEF7E1FDA4F8B0
:10D94800B601B4F89801A4F8B801B4F89A01A4F89B
:10D95800BA01012084F8B001FBF76CFD02212046D2
:10D96800F7F7C4FF002004F8760F0320E07010BD1D
:10D97800F6F748BD00207047F7F716BA002180F87F
:10D98800751080F8761080F8791090F8FB1009B1BE
:10D99800022100E00321F9F7C5BA90F87C00FE28BF
:10D9A80001D0012070470020704710B5012806D02B
:10D9B800022804D040F273210620F6F783F910BD3F
:10D9C800012802D0022805D102E0012904D001E093
:10D9D800022901D00020704701207047401A00B288
:10D9E80047F6FE71884201DC002801DC01207047FF
:10D9F8000020704700EBD10001F0070100780122F8
:10DA08008A401040C840704718B1022801D0012050
:10DA18007047002070472DE9FC41817804461A2997
:10DA280025D00EDC16292ED2DFE801F02D2D2D2D64
:10DA38002D212D2D2D2D2D2D2D2D2D2D2D2D2D2126
:10DA480021212A291FD00BDCA1F11E010C291AD291
:10DA5800DFE801F019191919191919191919190DE6
:10DA68003A3904290FD2DFE801F00E020E022088AD
:10DA7800B0F5706F07D201276946FEF730FD20B177
:10DA88000220BDE8FC811220FBE7019D68462E4676
:10DA980005F5B87506F2711600F039FD08B1287859
:10DAA80008B10C20EDE72F70A07830706846FFF7BA
:10DAB80051F80020E5E710B5044600F0A2FD08B1D2
:10DAC8000C2010BD207818B1012801D0122010BDFB
:10DAD800FFF79AFF611CF7F7B5FD08B1002010BDEC
:10DAE800072010BD10B500F08CFD08B10C2010BD4A
:10DAF800F7F7D0FD002010BD10B50B46012200F14C
:10DB08001001FEF7CEFC002010BD10B500880021E2
:10DB1800FEF7BBFB18B190F8731111B107E00220B2
:10DB280010BD90F87610142903D0152901D00C20C7
:10DB380010BD022180F87311002010BD38B50546CC
:10DB480000880021FEF7A1FB040003D094F87301BC
:10DB580010B110E0022038BD94F87600142801D0E6
:10DB6800152808D194F8C4018DF800000098009099
:10DB78009DF8000008B10C2038BD1022A91C04F53E
:10DB8800BA70FDF723FC012084F87301002038BD2A
:10DB980010B50821F6F72AF9002010BD10B5044683
:10DBA80000F0CCFCFFF718FA2070002010BD10B56B
:10DBB8000446D820207000F085FC6070002010BD5D
:10DBC800082101700020704710B5044600F019FDC7
:10DBD80008B10C2010BD207808B1012807D1FFF743
:10DBE80013FF611CFEF752FC08B1002010BD122083
:10DBF80010BD70B586B0054600F0A0FC0446694625
:10DC0800FFF702FA18B16946E06AFEF784FB0022C2
:10DC180004A8E16AF6F798FCDDE90401CDE9000102
:10DC280068B129786A46681C00F03DFB06000CD0F4
:10DC38006946E06AFEF76FFB304606B070BD69467C
:10DC4800E06AFEF768FB0720F7E769462046FFF71A
:10DC5800F2F9009803902878ADF80A0000208DF8B2
:10DC6800080002A800F0AAF9E7E77FB5054600F02A
:10DC780065FC06462878002460B18DF80040012034
:10DC88000DF10101F6F7C0FE20B1684600F094F8E6
:10DC9800002812D18DF80C403046FFF793F918B1DF
:10DCA8008020ADF80D0001E0ADF80D408DF80F4073
:10DCB8002878012803D038B1122004B070BD03A918
:10DCC8003046FBF779FCF8E7304600F04FFCF4E704
:10DCD80030B58BB0044600F031FC02466088B0F5E0
:10DCE800804F02D912200BB030BD00258DF80450AA
:10DCF800217900959DF80000052940F010008DF865
:10DD0800000054D2DFE801F0030805110B0040F0D1
:10DD1800010040F0020006E040F0090001E040F098
:10DD2800010040F004008DF80000BDF800000090EC
:10DD3800BDF80000ADF805002188DDF8060061F3A4
:10DD48001F20CDF806006188DDF8090061F31F2067
:10DD5800CDF80900607B8DF80D0060798DF80E0014
:10DD6800A0798DF80F00D4F807000490B4F80B00E0
:10DD7800ADF81400A07B8DF816007F208DF81700F1
:10DD880001208DF818008DF819508DF81A008DF8BB
:10DD98001B501046FFF732F98DF81C008DF81D5006
:10DDA8008DF81E5009A901A800F082F89BE741F2FE
:10DDB800A9013920F5F786FF70B5044600780121DE
:10DDC800FEF763FA050007D0FFF70DFB60B12846A0
:10DDD800FFF7FEF810B105E0422070BD2846FFF7B6
:10DDE800EDF808B10C2070BD611C2846FFF7FEF85D
:10DDF800002070BD10B50446012000F042FA28B199
:10DE080021460120F6F718FE002010BD0C2010BD99
:10DE180030B587B0054600F091FB04466946FFF728
:10DE280012F918B16946E06AFEF775FA002205A8EA
:10DE3800E16AF6F789FBDDE90501CDE900012978FA
:10DE48006A46681C00F02FFA050006D06946E06AA9
:10DE5800FEF761FA284607B030BD69462046FFF74D
:10DE680009F900208DF80C0000980490BDF8040012
:10DE7800ADF80E0003A800F0CAF8ECE710B5F6F705
:10DE8800FFFD002010BD7CB50C46054600F039FBAF
:10DE980060B169462846FEF722FB002805D100211B
:10DEA8002246019800F0B8FA00207CBD01207CBD14
:10DEB8002DE9FC410F460546067800F044FA002893
:10DEC8000AD1284600F023FA002805D10120F6F7E8
:10DED800DFF8864202D30720BDE8FC8101213046E5
:10DEE800FEF7D3F9040004D0FFF77DFA58B10C20EF
:10DEF800F2E7002201213046FEF7ABF9040010D00A
:10DF08003146FFF709F82046FFF766F83870E874DD
:10DF180029462046F8F7BAF80646687E60B32EB15F
:10DF28002AE041F22B213920F5F7CCFE694620463C
:10DF3800FFF76AF818B16946E06AFEF7ECF9694636
:10DF48002046FFF780F818B16946E06AFEF7E3F962
:10DF58000020ADF804000090ADF8060069462046A0
:10DF6800FFF769F869462046FFF784F82046FFF76F
:10DF780059F82046FFF775F83046ADE710B5044666
:10DF8800FFF74BFA20B12078F8F78CFF002010BD7E
:10DF98000C2010BD10B5007800F00100F8F788FFDC
:10DFA800002010BD10B5044600F0ABFA20B12046A1
:10DFB800BDE81040FBF7CEBB012010BD7CB505467F
:10DFC80000780121FEF761F906001ED00122698858
:10DFD80000F07EF9002817D13046FEF7BCFF044652
:10DFE8006888A04200D8044669463046FFF71EF804
:10DFF80068680090ADF8044069463046FFF71BF8A2
:10E008003046FFF70FF800207CBD42207CBD7CB570
:10E01800044600780121FEF738F905000BD00122EB
:10E02800618800F055F9002806D166882846FEF771
:10E03800CFFF10B102E042207CBD00266946284689
:10E04800FFF713F860680090ADF804606946284649
:10E05800FFF710F82846FFF704F800207CBD7CB5D0
:10E068000C46054600886946FEF739FA002806D1AD
:10E07800019829882180B0F89800608000207CBD34
:10E0880010B5044601460020F6F7BEFC10B9002082
:10E098002060A080002010BD7CB500886946FEF78E
:10E0A8001EFA58B9684600F032FA38B1019C94F863
:10E0B800AC1104F5D670683429B901E002207CBDA2
:10E0C80094F8451009B13A207CBD94F846104FF0F9
:10E0D8000105890703D105706846FEF73BFD84F802
:10E0E800455000207CBD7CB50C4605460088694635
:10E0F800FEF7F5F908B102207CBDA87830B100F030
:10E10800E1F9A0702888208000207CBD019890F853
:10E118006600F6E710B5FBF7BFFB002010BD2DE940
:10E12800FC41044640880D46B0B120886946FEF798
:10E13800D6F900280ED120882880019E351D683622
:10E148002F68628839463046FEF7FBFA2868B842DD
:10E15800F6D10020BDE8FC811220FBE7FBF7EAB905
:10E168002DE9F04786B08A460646008801A9FEF7E1
:10E17800B6F9002838D102984FF0000801468946C0
:10E1880090F8F4118DF80010009900919DF8005056
:10E1980090F876106830212900D13DB100244C3028
:10E1A80008210746FFF726FC10B107E00124F6E72F
:10E1B8000B213846FFF71EFC00B9A4B104A8009053
:10E1C8009DF8040003AB3246494600F05BF90700AE
:10E1D8000AD19DF80400029C48B104F5D3740120CB
:10E1E80060704DB906E01A2006B0BDE8F08704F566
:10E1F8009574F4E7207808B13A2712E084F800A073
:10E208009DF80C00A0709DF81010E1708DF80000CA
:10E218008DF80110B088ADF8020069464846FEF74F
:10E228001DFA84F801803846DEE74FF4A47188426D
:10E2380003D340F64801884200D308467047C10717
:10E2480001D001207047800701D5022070470020C7
:10E2580070470EB569460120FEF721F850B140F22B
:10E2680031113920F5F72EFD0298FFF7BCF808B1F7
:10E2780001200EBD6846F5F757FF0028F4D00020AE
:10E288000EBD10B5FFF7E5FF58B100F057F9044689
:10E29800FEF79EFE18B92046FEF790FE08B1002052
:10E2A80010BD012010BD70B50D461446014690887A
:10E2B800E38842199A4201D9072070BD22681044A8
:10E2C8002A46FDF783F8A0882844A080002070BD66
:10E2D80070B50C46054612B11F2907D811E0FF2C6E
:10E2E80004D8FEF773FE18B11F2C01D9122070BD97
:10E2F8002846FEF774FE30B121462846FEF737FE61
:10E3080018B1002070BD422070BD452070BD10B509
:10E3180004464078C10612D5C0070BD0FBF7FAFABD
:10E3280068B16078C10605D4000703D5207D0228AE
:10E3380005D106E0207D022803D0A07E08B1112077
:10E3480010BD002010BD38B504460078EF2847D826
:10E35800B4F80100ADF80000009800F02DF9C0B342
:10E36800617808070FD4D4F80220D4F80500130AFE
:10E37800B3EB102F34D82023B3EB122F30D85A0226
:10E38800B2EB102F2CD3607A18B3072828D8A07ABC
:10E3980028B1012803D0022801D0032820D14A0738
:10E3A80003D4022801D0032805D1E07A08B1012856
:10E3B80016D1480707D4A07C28B1012803D0022829
:10E3C80001D003280CD1C806207D03D5012807D128
:10E3D80002E005E0022803D0207E18B1012801D010
:10E3E800122038BD002038BDFB2803D840F648006D
:10E3F800814201D911207047002070471B38E1285D
:10E4080006D2B1F5A47F03D344F29020814201D90A
:10E4180012207047002070472DE9F0410646B0F8F9
:10E428004A70B0F84C4015462430F8F747FD80464E
:10E438000221FEF7E4F8874200D238460746022157
:10E448004046FEF7DCF8844200D220463188298015
:10E458001B2F13D9FB2F00D3FB276F801B280FD945
:10E46800FB2800D3FB20E8804046FFF7DEFEA880AB
:10E478004046FFF7DAFE2881BDE8F0811B27ECE76C
:10E488001B20F0E72DE9F0419078069E1D461446C2
:10E4980008B9FBF78FFAE478074614B9FBF78AFA4C
:10E4A80004466FB164B13846FFF7C9FE2046FFF74E
:10E4B800C6FE2FB124B12F7034700020BDE8F08162
:10E4C8000920FBE710B5FCF725FF28B9FCF758FF32
:10E4D80010B9FCF75FFF08B1082010BDFCF7EFFE8C
:10E4E80040B9FCF7F6FE28B9FCF70AFF10B9FCF7AB
:10E4F8001BFF08B1042010BD40F297513920F5F7F1
:10E50800E1FB10B5FBF750FAC0F3401010BD4068AE
:10E5180000F000B808B590F82C1190F88C008DF830
:10E528000000009800909DF80000401E084203D0AB
:10E53800042901D0012008BD002008BD10B5012123
:10E548000020FDF7A2FE040009D100220121104697
:10E55800FDF77FFE040004D00021FEF7DDFC204615
:10E5680010BD40F226213920F5F7ACFB70B5054601
:10E57800FEF735FD70B12846FEF735FF002808D0B4
:10E588002846FEF72DFF04462846FEF703FF18B17C
:10E598000C2070BD422070BD64B12088FDF7EEFEEE
:10E5A80020880021F5F710FE20B141F27A41392088
:10E5B800F5F788FB002070BDC0B2C1060CD48106F7
:10E5C8004FEAC07103D5D1B9810718D401E00029F9
:10E5D800FAD1000713D410E0410610D481060ED4F6
:10E5E800C1074FEA807104D0002902DB400704D438
:10E5F80005E0010703D4400701D40120704700203B
:10E6080070473EB569460120FDF749FE78B140F2F2
:10E618004F113920F5F756FB029C2046FEF7E3FE22
:10E6280028B12046FEF743FD08B101203EBD6846EB
:10E63800F5F77AFD0028EFD000203EBD026812B938
:10E64800016070470246506808B18A42FAD18A428E
:10E65800F7D05160704710B5FEF7C8FE08B1D82151
:10E6680003E0F7F7E1FD18B1DD210120F5F72AFBFA
:10E67800BDE810400120F5F7EFBC10B5044602E0F4
:10E68800206880476468002CFAD110BD10B50020BE
:10E69800F5F7E2FCF5F716FFF6F798F9F6F776FBCB
:10E6A800002803D0B5210120F5F70CFB10BD10B5EB
:10E6B800FFF7D1FFFFF75EF9002803D0F62101200C
:10E6C800F5F700FB10BD10B5FBF7F0FC00F050F8B3
:10E6D800FBF7C4F9BDE81040FBF7BABA10B5C82477
:10E6E800641EE4B2FBF7D8F9022803D0012800D051
:10E6F800002010BD002CF3D18F213B20F5F7E2FA62
:10E7080010B5F5F7BFF9002805D0401C03D05021FB
:10E718004020F5F7D7FA10BD10B5F5F7BFF9002876
:10E7280005D0401C03D049214020F5F7CBFA10BD95
:10E7380010B5F5F7A1F9002805D0401C03D05721E2
:10E748004020F5F7BFFA10BD10B500210846F5F7CF
:10E758009FF908B1002010BD012010BD08B568461A
:10E76800F5F7A8F99DF80000002800D0012008BDA1
:10E778004FF0E0214FF40040C1F88001BFF34F8F04
:10E78800BFF36F8FFBF7E6BA002809DB00F01F0222
:10E79800012191404009800000F1E020C0F880127A
:10E7A800704700280DDB00F01F020121914040094D
:10E7B800800000F1E020C0F88011BFF34F8FBFF355
:10E7C8006F8F704710B5012806D0022806D040F692
:10E7D800C5313E20F5F776FA282010BD182010BD67
:10E7E80010B5012806D0022807D040F6D9313E20BE
:10E7F800F5F768FA41F6146010BD41F2301010BD0B
:10E80800FCF7F4B910B50A4630B101280BD040F234
:10E818004F613E20F5F756FABDE8104002F1280195
:10E828001046FBF78DB9BDE8104002F129011046EA
:10E83800FBF770B970B5054614460846FFF7D0FFD8
:10E8480005EB4501C1EBC511C0EBC1052046FFF73B
:10E85800C7FF28444FF47A7100F6B730B0FBF1F5E2
:10E868002046FFF7AFFF2844401D70BD2DE9F04159
:10E8780007461D460E4614461046FFF7B1FF07EB44
:10E888004701C1EBC71100EBC1014FF47A70022EAA
:10E898000ED040F2DC52114401F6B731B1FBF0F66C
:10E8A8002046FFF78FFF30442844401DBDE8F08123
:10E8B8000246F0E710B504460846FFF791FF4FF40B
:10E8C8007A7100F2E730B0FBF1F0201A801E10BD1B
:10E8D80010B504460846FFF783FF4FF47A71B0FB82
:10E8E800F1F0201A10BD4FF47A72022908D040F2D4
:10E8F800DC5101F2E731B1FBF2F10844801E7047A8
:10E908001146F6E74FF47A72022907D040F2DC513B
:10E9180001F57A71B1FBF2F1084470471146F7E747
:10E928000C0802170D010102090901010602091864
:10E938001803010109090303050000000000000095
:10E9480073B5BB4DD5F83431996811F0010121D167
:10E9580001AA40F6034003F093FB0446002869D15E
:10E96800019B9B681B7893B9BFF35B8F2B4653F8C9
:10E97800942FBFF35B8F02F00502BFF35B8F53E860
:10E98800001F43E800200028F9D1BFF35B8F0198EE
:10E9980007F078FB01AA002141F2030003F070FBA5
:10E9A8000446002846D1019BA248996808220131F3
:10E9B8000DF016F9019807F065FB214601AA41F20E
:10E9C800010003F05DFB0446002833D101988368F9
:10E9D8005A7885F83420D9789A7842EA0122EA866A
:10E9E8001A7985F83520197ADA7942EA01222A87D4
:10E9F8005A799B7942EA03236B8707F043FB214648
:10EA080001AA41F2020003F03BFB044690B9019BC6
:10EA180089489968402201310DF0E2F886480DF0E6
:10EA280085F9019807F02EFB95F840305B0604D471
:10EA38006FF01204204602B070BD214601AA42F2CE
:10EA4800030003F01DFB04460028F3D1019B7B481B
:10EA58009968082201310DF0C3F8019807F012FBFC
:10EA6800214601AA42F2020003F00AFB04460028EC
:10EA7800E0D1019B9B68B3F80120A5F8C42091B2AE
:10EA880021B1DA786E48114610F0D7FE019807F0E8
:10EA9800F9FA95F8406016F0200600F0B88095F86D
:10EAA80060301E0711D501AA002142F21C0003F0B4
:10EAB800E7FA04460028BDD10198836853F8012F6E
:10EAC8005B68C5E9282307F0DDFA95F898305C06FD
:10EAD8000FD501AA002142F22A0003F0D1FA044618
:10EAE8000028A7D1019883685B7885F8E03007F0A3
:10EAF800C9FA082142F2010003F03EFA0446002850
:10EB080000F08C80082108440FF083FE95F89810D7
:10EB180011F0400F024640F2022308BF0323880782
:10EB28004CBF43F02C0043F00C0095F86630C90741
:10EB380003F0060348BF40F01000062B08BF40F45E
:10EB4800C07000210DF08DFA2146002242F201002A
:10EB580003F096FA044600287FF46CAF95F840302D
:10EB68009A061ED4B5F8C410D9B901AA41F2050015
:10EB780003F086FA044600287FF45CAFB5F8C43089
:10EB880063B9019B9B685A78997842EA0122A5F8F3
:10EB9800C4209A882A48114610F04FFE019807F0C1
:10EBA80071FA082140F6014003F0E6F90446A8B3DB
:10EBB800082108440FF02DFE95F89830DB0702462F
:10EBC80054D519A1D1E900010DF04BFA21460022D4
:10EBD80040F6014003F054FA044600287FF42AAFB7
:10EBE8000DF04CFC044600287FF424AF04F096FE98
:10EBF800044600287FF41EAFEB79002B3FF41AAFD0
:10EC0800042110480DF06BF903F0C2FB12E7022152
:10EC180040F66D4003F0B0F90446A8B96FF06804F7
:10EC280008E700BFAFF30080908800020080002052
:10EC3800B8020020F4020020FC020020500300204B
:10EC4800800300204C030020022108300FF0E1FD72
:10EC58000123037046702146324640F66D4003F0AA
:10EC68000FFA044600283FF41AAFE3E601484FF0D4
:10EC78000051A9E71088000270B503788AB00446ED
:10EC88000E4607AD032B20D8DFE803F002191B1D41
:10EC9800114928460CF04CFF63780493A37803933A
:10ECA800E378029323790193637900930B4AA3795C
:10ECB80005951E2130460AF02AFE0AB070BD0849A3
:10ECC800E7E70849E5E70849E3E7084A0A2128464B
:10ECD8000AF01DFEE0E700BF700902009909020072
:10ECE800770902007E0902008809020092090200E1
:10ECF80010B5044688B061B90DF07BFE6946FFF790
:10ED0800BBFF20460DF094FD034B1860012010F066
:10ED1800EBFA08B010BD00BFE824002010B50C4C79
:10ED280088B00DF066FE6946FFF7A6FF206818B1A7
:10ED38000DF099FD00232360064C206830B10DF0DA
:10ED480092FD00230120236010F0D1FA08B010BD15
:10ED5800E0240020E824002010B588B004460DF017
:10ED680067FD054B186020460DF043FE6946FFF726
:10ED780083FF08B010BD00BFE024002038B50C4860
:10ED88000C4D4FF0FF324FF0FF3309F059FD4FF0B3
:10ED9800FF334FF0FF32284609F0F8FC828D044615
:10EDA800011D002001F04CFF204611F014F9EEE798
:10EDB800B8060020300700202DE9F04F002489B064
:10EDC80005460F46164621461A2201A800940CF063
:10EDD80012FF28460DF00DFE6946FFF74DFFDFF8DC
:10EDE8007480DFF87490A64202D109B0BDE8F08FB4
:10EDF800302011F0F7F805460028F6D0331B272BF2
:10EE080094BF9AB2272200F1040A82853919504624
:10EE18000CF0E6FEAB8D1C44A4B2B44209D13A19F9
:10EE280012F8012C0D2A04D1EA180A2101331171B4
:10EE3800AB85D8F80000AA8D83685146D3F804B092
:10EE48004FF0FF33D8470028CDD02946484610F068
:10EE5800A3FCC8E7EC2400204807002010B53020A8
:10EE680011F0C0F8014660B100238385094B18688A
:10EE78008368DC682822A4463223BDE810400431A8
:10EE88006047BDE81040044840F26762002309F07B
:10EE9800C3BE00BFEC2400201814002070B50B7806
:10EEA8000C46052B00F28780DFE803F00386246711
:10EEB800774D8B68002B7ED0486800287BD0464A67
:10EEC8001368ABB1181F00231360444A136011F094
:10EED80082F843480022002309F058FC00286AD031
:10EEE800828D011D3F4BBDE8704018680AF011BCC7
:10EEF8000438ECE74868E268038D13449BB23A4A49
:10EF080003850025282B1570A0F10401154604D1AE
:10EF1800BDE87040354810F03FBC034413F8013C8D
:10EF28000A2B01D00D2B46D1304810F035FC304B60
:10EF380062681A6001232B702A4B18688368BDE841
:10EF480070405B691847302011F04CF8014660B1F9
:10EF580000238385234B18688368DC682822A4462D
:10EF68003223BDE8704004316047BDE87040214855
:10EF780040F26762002309F04FBE302011F032F8EA
:10EF88000146C0B100238385164B18688368BDE825
:10EF980070401B69282204311847134D2B7853B150
:10EFA800134C48682368984205D0043811F013F8C8
:10EFB80000232B70236070BD074A13680BB94B6898
:10EFC80013600648A36801680B44116803600A8D42
:10EFD8001944D21A86E700BFD8240020DC24002078
:10EFE80048070020EC240020682900203007002072
:10EFF800E42400201814002038B50D4C034620687E
:10F00800A0B103EA0105EA0706D504F05DFC206813
:10F018000DF029FC00232360AB0707D5206804F016
:10F0280061FC20680DF01FFC0023236038BD00BF81
:10F03800E0240020F0B53B4889B008F00BF807F051
:10F04800C7FF3948394E09F0D7F8306010B330207F
:10F0580010F0C8FF0546E8B10024354984853548D5
:10F0680010F082FC30683449836822461B68984750
:10F0780080B9302010F0B6FF044658B1071D2F4A5A
:10F088002821384602F02AFA2728024604D92046C1
:10F0980010F0A1FF0AF045FBA085394630680AF058
:10F0A80038FB0028F6D1306883682822DC68291DDF
:10F0B8003223A04704460028ECD1214804F06CFA1A
:10F0C800204804F0E5FB204603F074F90028E1D15C
:10F0D8001D4809F08FFB0BF01CFA1C4801F0A4FD39
:10F0E800E8B91B4D0FCD03AC0FC42B682360012377
:10F0F80000931849184B022203A803F03DFE04466A
:10F1080068B9013404F0010148BF4942002008F001
:10F1180033F800214FF4004009F094FFF1E709B0FB
:10F12800F0BD00BF01F00000BC090200EC24002083
:10F1380065EE000018140020A5EE0000C3090200C7
:10F1480014040020F0030020B8060020300400203A
:10F15800A0020200480302005803020030B50A4C1E
:10F168000A44914200D130BD11F8013B58400309CF
:10F17800E35C83EA0013DDB2C3F30313E05C80EAC7
:10F188000510C0B2EDE700BF120A020030B585B025
:10F19800CDE901010446002501A90548039500F0C1
:10F1A800EFF8DDE902309842B8BF255405B030BD0C
:10F1B800F19801002DE9F84FB0F8189019F00808F7
:10F1C800044693460DD001290CBF49F0100949F0B7
:10F1D8002009A0F818908BF31188BFF36F8FBDE852
:10F1E800F88F09F00709022907D120460AF09CFB8D
:10F1F8000028F0D00128238B50D16769218B002F7C
:10F2080015DA256821F00701C4E9008841F00101F9
:10F2180021830026218B01F0070ACA4502D0A36882
:10F22800002B5CD10DB9002E74D0002358E001F0FA
:10F2380007035A1F012A20D821F00701062B256849
:10F2480089B2C4E900880CD1002D2B4638BF0023B1
:10F258002BB1628B1B6801326283002BF8D141F01D
:10F268000201218320460AF05FFB06460028D1D020
:10F27800238B43F020032383CBE7042B0CD121F00D
:10F28800070189B2218320460AF04EFB0546002873
:10F29800BFD041F0200121830025BAE7032809D116
:10F2A800226923F00703166843F006032383002529
:10F2B8002F46AFE7042806D1226923F007035668D2
:10F2C80043F00403F2E7052806D1226923F0070377
:10F2D800966843F00503E9E700252E46E8E7012391
:10F2E80041F0080121838BF31188BFF36F8F03BBB3
:10F2F800002D33D116B121492046B0474FF04003C5
:10F30800EFF3118B83F31188BFF36F8F238B23F0F7
:10F3180008032383238BDA0628D523F010032383DD
:10F328000121B4F8189009F0070900297FF45BAFB0
:10F3380051E7A1680029DBD00B68D1F804B0002B95
:10F3480038BF0023994652463B462046D847B9F174
:10F35800000FCDD0D9F800304946EEE729463B46A4
:10F36800524620462D680AF0FBFAC1E713F0200147
:10F378001EBF23F0200323830221D2E795990100C1
:10F388002DE9F04F91B08B46029092461C4600251D
:10F398009AF8000008B928465EE325280AF1010713
:10F3A80007D0029B594698470028C0F2558301357B
:10F3B80010E2182200210AA80CF01DFC9AF801306E
:10F3C800252B78D000229446164696461046394694
:10F3D80017F8013B2B2B00F09D8000F29480202B26
:10F3E80000F09B80232B00F09A8028B19DF8300014
:10F3F80040F004008DF83000BEF1000F05D09DF8F4
:10F40800300040F008008DF830002EB19DF8300033
:10F4180040F010008DF83000BCF1000F05D09DF8C9
:10F42800300040F020008DF830002AB19DF83020DF
:10F4380042F040028DF830209DF8302002F0440060
:10F44800442803D16FF386128DF830209DF83020C0
:10F458002A2B42F080028DF830207BD19DF8312094
:10F4680042F001024B1C8DF831201A782E2A9DF8A3
:10F4780031200CBF0121002161F341028DF83120B8
:10F4880074D15A782A2A6AD0013300210A261846EC
:10F4980010F8012BA2F13007092F40F28E809DF859
:10F4A80030200E91C2F3400040EAD17161F341026D
:10F4B8008DF830205AE00AF102078DF833309DF8B4
:10F4C8003130D90740F1498154F8049BB9F1000F54
:10F4D80007DA9DF8302042F004028DF83020C9F197
:10F4E80000095A0740F1428154F8048BB8F1000F23
:10F4F80080F241819DF831306FF341038DF831304E
:10F508004FF0FF3837E12D2B0CD0302B7FF46DAF47
:10F5180001225CE74FF0010E59E7012657E74FF04B
:10F52800010C54E7012052E70CFB0202303A334643
:10F538001E4616F8010BA0F13007092FF4D999429D
:10F5480093D09DF830100D92D20F62F341018DF8DF
:10F5580030108AE70B4600224FF00A0CE8E79DF8C6
:10F56800312042F004028DF8312002331F4617F88B
:10F57800012B6C2A41D025D8682A2BD06A2A46D07C
:10F588004C2A4CD01F4617F8012B9DF831308DF8C6
:10F598003320782A00F2D980572A4DD8412A03D03F
:10F5A800453A022A00F2D1809DF83230042262F3F3
:10F5B80002038DF8323001239EE006FB0121303929
:10F5C800034664E7742A26D07A2ADBD19DF83130C5
:10F5D80006220DE05A78682A9DF8312006D10121CB
:10F5E80061F3C6028DF831209F1CCCE71346022236
:10F5F80062F3C6038DF83130C5E75A786C2A9DF856
:10F60800312001D10421EBE713460322F0E79DF8EE
:10F6180031300522ECE79DF831300722E8E7BDF8E4
:10F62800303023F4F04323F0020343F4804343F0E3
:10F638000203ADF83030A6E7A2F15801202900F204
:10F64800848001A050F821F015F7000053F700005E
:10F6580053F7000053F7000053F7000053F700007A
:10F6680053F7000053F7000053F70000B1F500000E
:10F6780053F7000015F70000D5F60000B1F50000BB
:10F68800B1F50000B1F5000053F70000D5F6000011
:10F6980053F7000053F7000053F7000053F700003A
:10F6A8001DF7000015F7000039F7000053F70000B8
:10F6B80053F7000039F7000053F7000015F7000072
:10F6C80053F7000053F7000015F700009DF83210BB
:10F6D800012003F0780360F30201402B8DF832100B
:10F6E80002BF9DF8301041F001018DF83010632AF7
:10F6F80031D1003B18BF01239DF83020C2F34001EF
:10F708000B4363F341028DF83020D8E69DF83210A0
:10F718000220DEE79DF8322003F07803A3F14000D1
:10F72800032161F3020243428DF832204341E3E7AB
:10F738009DF83220032113F0780F61F302028DF84F
:10F74800322014BF01230023D6E79DF8303043F060
:10F7580001038DF830300023CEE79DF93020002AD0
:10F76800B4BFDDF834904FF0FF39BAE69B077FF558
:10F77800C7AEDDF838809DF831200023CDE90D3380
:10F788009DF8323003F00703012BC2F3C30236D1D0
:10F79800D31E042B20D8DFE803F00307071F1F0040
:10F7A80054F8040BC11704E0073424F00704F4E804
:10F7B8000201CDE90A019DF8303013F0030654D058
:10F7C80002983B46524659460AF05AFC0028C0F2B5
:10F7D80043810544BA46DBE554F8040B012A4FEA95
:10F7E800E071CDE90A0105D19DF828300A9300237C
:10F7F8000B93E0E7022ADED1BDF92800D2E7022BFD
:10F8080023D1D31E042B13D8DFE803F0030A0A120E
:10F81800120020680A900021231D0B911C46CAE79C
:10F82800073424F00703F3E80201CDE90A01F5E7FC
:10F8380054F8043B0A93012A4FF000030B93D3D0EA
:10F84800022AB8D1BDF82830D0E7042B07D10734F5
:10F8580024F00704F4E80201CDE90A01ABE7032B21
:10F8680004BF54F8043B0A93A5E79DF833007828B1
:10F87800B0D8622822D825283FF493AD5828A9D1BA
:10F888000DF126030093DDE90A0104AB0CAA0AF086
:10F89800ACFB8246B8F1000F0DF126000CDB9DF899
:10F8A8003020A0EB0A036FF3861298458DF83020BC
:10F8B80002D9A8EB03030D9380463DE06338152871
:10F8C80088D801A151F820F051F90000B5F90000DD
:10F8D800DDF70000DDF70000DDF70000DDF70000D0
:10F8E800B5F90000DDF70000DDF70000DDF70000E6
:10F8F800DDF7000013FA0000E1F90000E5F9000067
:10F90800DDF70000DDF7000029F90000DDF7000051
:10F91800E1F90000DDF70000DDF70000E1F9000083
:10F92800B8F1000FDDF828A00ADB414650460CF07C
:10F9380023F90AEB00080026BAF1000F0CD149E7B9
:10F9480050460CF012F9F4E70A9B8DF810300026A7
:10F958000DF111080DF1100AA8EB0A0306B10133E5
:10F968009DF83220D0066BD5023352060D9948BF58
:10F978000E9A0B4448BF9B18B9F1000F79DD9DF82A
:10F988003020A9EB0309C2F380030393530770D413
:10F99800500664D546B1029B594630469847002820
:10F9A8005ADB039B01351E46302359E01E0711D44C
:10F9B80013F0100618BF2026DDE90A23002A73F188
:10F9C8000001BFF65DAF524263EB4303CDE90A2362
:10F9D8002D2655E72B26EFE7002651E70A9848B36E
:10F9E8000DF1260300930CAA04AB00210AF0FDFADE
:10F9F800BDF8323003F0EF0343F4F04343F0100353
:10FA08008246ADF83230002644E70A9B072A3FF6C3
:10FA1800E1AEDFE802F00D04060D08080D0D1D70BB
:10FA2800D8E61D80D6E62846E917C3E90001D1E6E5
:10FA38001D60CFE6DFF8C4800646A8F1050A8BE70B
:10FA4800110748BF013390E7184603935946029BB4
:10FA580098470028039B04DA11B0BDE8F08F2023F3
:10FA68004D444A46002AA5EB090109F1FF39EBDCB0
:10FA78000D4636B1029B5946304698470028EBDBC5
:10FA880001359DF83230D90601D41A0706D5029BF4
:10FA98005946302098470028DEDB01359DF8323082
:10FAA800DB0607D59DF83300029B59469847002886
:10FAB800D2DB01350D9E2E44731B002B16DC0298F9
:10FAC8004346524659460AF0DBFA0028C4DB05448F
:10FAD800A944A9EB0503002B7FF77CAE029B59468E
:10FAE800202098470028B7DB0135F2E7029B5946EA
:10FAF800302098470028AFDB0135DDE7270A0200F0
:10FB08002DE9F7430F4606460821C06A0AF08BFB29
:10FB18003C68134B241A80463C6004EA0305994666
:10FB2800AC4203D8002003B0BDE8F08308236A463E
:10FB3800214630460AF0DAFA0028F4D16946304600
:10FB48000AF07BFB40B1BDF80230BDF804203C60F0
:10FB580005EA090513441D44A4EB0804E0E700BFC7
:10FB68000000FFFF2DE9F04F044695B0C06A082158
:10FB78000AF059FB63681B0C1B04054603A9E089BE
:10FB880003930AF074FB039BA18906AE1944491B31
:10FB980032460823204604910AF0A8FA021EC0F251
:10FBA800AB80E36A1A790023F15C914240F09280BD
:10FBB8000133082BF8D1A06863682844834280F099
:10FBC8008180039920460AF0EEFA024694E0049BED
:10FBD800BDF81A201B0C1B0413440493DFF820B152
:10FBE800DDF810A008AA04A920460AF0C4FB0246C2
:10FBF800002840F0818008A920460AF01EFB002852
:10FC080036D0636805930AAA05A92046059E0AF01E
:10FC1800B2FB024600286FD1BDF82820BDF820307D
:10FC28009A4228D06268059B9A42ECD156451FD16A
:10FC3800BDF82430E3B1BDF822300AEA0B071F44AF
:10FC480008A8A368ADF822300AF0E4FAE36ABDF820
:10FC580024801E68764206F020030193B8F1000F55
:10FC680010D108A920460AF060FB0246002843D1BB
:10FC7800CA45B5D19FE70AA920460AF0DEFA00284E
:10FC8800D0D0D3E7019B434528BF43460CAA394649
:10FC980020461E460AF02AFA024668BB36B10CAA6C
:10FCA800A168334620460AF00BFB02463146E06A5B
:10FCB8000AF0B9FAA1680144A160EAB9A8EB0608FC
:10FCC8003744CBE720460AF041FB024600283FF4C0
:10FCD80078AF11E0049B31462046A3EB05090AF0F2
:10FCE800D1FA00287FF473AF04A92046FFF708FF74
:10FCF800024600283FF472AF104615B0BDE8F08FF9
:10FD08000000FFFF2DE9F047044688B00D4600F1DA
:10FD1800140738460FF0BDFC284608F06DFAA062BB
:10FD2800002800F01E8183681B699847E06228B9A3
:10FD38006FF01505284608B0BDE8F087A06A83680B
:10FD48001B6998470368013B1F2BF1D8A06A2168FB
:10FD580005AA0EF060FE0028EAD1A389002BE7D09F
:10FD6800069AB3FBF2F502FB1535002DE0D1E389C5
:10FD7800012BDDD9E36A009593F804804FF0FF3238
:10FD88004FF0FF33384608F03DFCE06A08210AF0DE
:10FD98004AFAA9460646E3891FFA85FA534544D824
:10FDA800E3894B4500F0D28053450BD100990823D5
:10FDB8004246891B20460AF0D1F918B9E0896946FC
:10FDC8000AF055FA69462046FFF79AFE05460028CC
:10FDD80040F0BE80009B794A63601340A36091465F
:10FDE800D4E9011399420ED3082301AA20460AF048
:10FDF8007DF9C0B901AB13F8012B904540F0C180E3
:10FE080001300828F7D16368E0891B0C1B04694698
:10FE180000930AF02CFAA3890099424620460AF07A
:10FE28009DF9002825DA054692E0A1892B04891B53
:10FE380013FA81F142460823204600910AF08EF910
:10FE480078B1E08969460AF012FA09F101090099C6
:10FE58000823424620461FFA89F90AF07FF900284C
:10FE68009ED0013597E7002A00F0A3806FF01C05AB
:10FE78006EE046D06368334400934FF6FF780099EC
:10FE8800A3898AB29B1B9A4216D3616820460AF05E
:10FE98008AF90028C7D16268484902EA0103A289A1
:10FEA8001344A3EB460363600B40A3602046FFF7AF
:10FEB80059FE002840D0B6E7082303AA20460AF0D6
:10FEC80015F90028AFD103A920460AF0B6F938B1D0
:10FED800BDF80C30434503D1BDF81030002B43D09A
:10FEE800009B33440093CAE75B1A424620460AF057
:10FEF80035F9002897DB08D0E26AA3681268134432
:10FF0800A360D4E901318B42EED86168A38901EB83
:10FF180046029A42CDD1DFF8A480A36801EA08021C
:10FF28009342C6D020460AF03EF900287FF47BAF02
:10FF3800636803EA0803A360A089A388A0EB4606C8
:10FF4800B34205D120460AF001FA6CE76FF02C05A0
:10FF5800384608F0D5FB002D7FF4ECAE012323745E
:10FF6800E8E66FF00505E5E66368E0891B0C1B040D
:10FF7800694600930AF07BF9009920460AF013F9C4
:10FF880097E701A920460AF058F9D4F804A080B1EF
:10FF9800009BBDF80820BDF80610E06A03EA0903D3
:10FFA800A36011440AF03FF903445345A3603FF4AA
:10FFB8005AAFAAEB0603636012E700BF0000FFFF19
:10FFC8002DE9F04F1E46037C89B0044689469046C9
:10FFD800002B00F0BF80C36A082118460AF023F9F5
:10FFE8003146824618460AF01EF9A389A3EB8A0314
:08FFF8009E42074600F2B180B1
:020000021000EC
:1000000016B1002A00F0AD806368039304AA03A927
:100010002046DDF80CB00AF0B2F90546002866D19A
:10002000BDF810304B4505D06268039B9A42EDD174
:10003000E6B95CE004A920460AF003F90028F3D0F1
:10004000BDF8143086B19E4210D1BDF812004FEABF
:100050001B41090401443346424620460AF058F841
:10006000002803DC054642E0002B40D0002F42D19F
:1000700004F1140A4FF0FF324FF0FF335046DFF81F
:10008000ECB008F0C3FA0022E3899A4263D0D4E9C5
:1000900001317818834231D3FF2306A8ADF81890B8
:1000A000ADF81A10ADF81C608DF81E300AF0B6F8E5
:1000B00036B1A1683346424620460AF005F90546A6
:1000C000E06A31460AF0B3F8A3680344A360002D48
:1000D0004AD106A920460AF02CF90546002843D14A
:1000E00033460193504608F00FFB019B1D462846FE
:1000F00009B0BDE8F08F5744BFB2B9E7E06A01929A
:1001000008210AF094F84FF6FF71ADF8181000219D
:10011000ADF81C101918ADF81A10A18903EA0B03E9
:100120000B44181A606006A80AF078F806A9204661
:100130000AF0FFF8E089211D0AF09DF8636803EAE0
:100140000B03A3602046FFF711FD03460028C8D12A
:10015000019A013298E76FF01B03C2E76FF00C05BC
:10016000C5E76FF01505C2E72B46BAE70000FFFFB1
:10017000094B30B51D68094B02461C6800239D429F
:1001800001DC002030BD190104EB0310615C9142D9
:10019000F8D00133F3E700BFB00302003C040020B5
:1001A000084B1B6810B50C462BB1FFF7E1FF28B1D7
:1001B0002060002010BD6FF00C00FBE76FF0010025
:1001C000F8E700BF3C04002030B589B00C46154666
:1001D0000190FFF7CDFFB8B14368029383682268AE
:1001E000C068CDE903350023CDE9062305930AF065
:1001F00074F960B1074901AA0EF015FC079808B917
:10020000059B236009B030BD6FF01500FAE76FF071
:100210001200F7E7DFA40100104B2DE9F0411C6844
:1002200005460E461746ACB14FF0FF324FF0FF3394
:100230000B4808F0EBF963683246D3F8088029468A
:100240003B462046C0470446054808F05DFA204674
:10025000BDE8F0816FF00104F9E700BFF824002049
:10026000A406002000230360044B5A6812B9C3E9B6
:100270000000704710605860704700BFF0240020F5
:10028000014B1860704700BFF824002030B585B0DE
:1002900000230546CDE9023301904FF0FF330E48AD
:1002A0004FF0FF3208F0B2F90C4B1C68002C38BF3D
:1002B00000243CB1636820461B6801A99847246864
:1002C000002CF6D1284600F089F80446024808F0D0
:1002D0001BFA204605B030BDA4060020F024002003
:1002E0001FB5CDE9010103924FF0FF330C484FF0E9
:1002F000FF3208F08BF90B4B1C68002C38BF002430
:100300003CB1636820461B6801A998472468002C0B
:10031000F6D1034808F0F8F9002004B010BD00BF82
:10032000A4060020F0240020024B0022C3E9002292
:10033000704700BFF0240020024B0022C3E90022D6
:10034000FFF7F2BFFC2400202DE9F34107460E46DB
:1003500009B100230B601E4CDFF87C80002544456A
:1003600008D31C4B1C680CB1143CC4B9284602B01D
:10037000BDE8F081216801AA38460AF0D5F860B1DD
:1003800025B90EB1019B3360254606E02968206837
:1003900000220AF0C9F80028F3D11434DFE72168FD
:1003A00001AA38460AF0C0F860B125B90EB1019B28
:1003B0003360254606E02968206800220AF0B4F878
:1003C0000028F3D114F1140FD0D06469CBE700BF3B
:1003D00030020200FC2400206C020200F8B51A4C26
:1003E0001A4F06460025BC4206D3194B1C680CB1B7
:1003F000143C9CB92846F8BD1EB9E3684BB91434C7
:10040000F1E72068002231460AF08EF80028F4D186
:10041000F5E79847002D08BF0546F0E736B9E368D1
:1004200063B914F1140FE5D06469E0E72068002295
:1004300031460AF079F80028F1D1F2E79847002D0B
:1004400008BF0546EDE700BF300202006C02020063
:10045000FC24002010B5064C23783BB9FFF76CFF55
:1004600000F064F808B90123237010BD0020FCE7F8
:10047000692900202DE9F047048FDFF8ACA0013492
:1004800098B080468946A4B200F10806651EADB258
:10049000B5F5004F45D04A2305AA294630460AF053
:1004A00015F804F57F543F34A4B2074621460123D2
:1004B0000DF10B0230460AF009F8002F014603DC6B
:1004C000002803DC2C46E1E7002816DCB8F83830B9
:1004D000AB4209D142466B1E22F8383F4FF400412F
:1004E00002233046FFF770FD2946304609F093FF9E
:1004F0002146304609F08FFFE4E718AB1F44002384
:1005000007F84C3C5246CDF8009003AB05A8039683
:10051000ADF810400AF041F80028D3D018B0BDE87B
:10052000F0870020FAE700BF01A601007FB5012394
:10053000694604200193FFF733FE0446002836D1B4
:1005400002AA01A90420FFF73FFE10F1130F044691
:100550002DD038B10C3405D0404080F311884FF0D5
:10056000040002DF0399B1F5803F23D2009A0023F3
:1005700095681846084485429CB203D30133082B82
:10058000F8D11C460D4D5368AB602846D368EC8209
:10059000A982EB630AF0CBF8044640B9084E6E60BE
:1005A0002846FFF75FFE28466E60FFF769FE20468B
:1005B00004B070BD6FF02004F9E700BF04250020EF
:1005C00040040020F8B505464FF04003EFF31186D4
:1005D00083F31188BFF36F8F0B4B1C68002C38BF5F
:1005E00000245CB1094FD4E90132002D08BF134645
:1005F0000BB1387898472468002CF4D186F3118821
:10060000BFF36F8FF8BD00BF442500204C250020AC
:100610001FB50F4B1A68BAB901221A600D4A07CAF2
:1006200001AB83E807000C4A4AB193E807000BF0DE
:1006300022FB002005B05DF804EBFFF7C3BF82F397
:100640001188BFF36F8FF4E705B05DF804FB00BFBE
:10065000500400204C25002077BC0100F0B589B083
:100660006E460146054630460AF07DF896E80700DA
:10067000174C84E80700207840B3164B002119601E
:100680006B1C0ED0144817464FF400460021134A45
:100690000023E6FB0701EFF70FFD0121281A0FF0F9
:1006A000C5FA08F0D5FA0120FFF78CFF94E807009F
:1006B00005AB83E807000A4A1AB193E807000BF07C
:1006C000C7FAFFF7A5FF08F071FB207809B0F0BD6D
:1006D0004C250020500400203F420F0040420F00F4
:1006E00051BC01000E4A70B5841AA3100D4C5C4336
:1006F0000546E4B20C2000FB04200E4640210844CD
:100700000AF03FF8011E05DB074B03EBC4046368E6
:100710009847002128463346BDE87040184700BF7F
:100720006C250020B76DDBB6C80302002DE9F0414F
:10073000104E841BA310104C5C43E4B20C2565439F
:10074000804605F140000F46304440210AF032F85F
:10075000011E09DB094A7319C3E90E27084B53F838
:100760003430BDE8F041184740463B46BDE8F04113
:10077000184700BF6C250020B76DDBB617A8010035
:10078000C8030200002270B501210446104600F0A3
:1007900093FC002000F05EFC0F4807F0A7F90F4B18
:1007A000984215D10EF08EFE26690D49304609F0AB
:1007B0000EF900280BDB012535642469084904F192
:1007C0001C0009F004F9002801DBE564002070BD7D
:1007D0006FF00400FBE700BF190801000000AD0B3B
:1007E000D803020001460C2309484B4370B5C418D6
:1007F000D4E90E5600224033A263184409F0F8FFF2
:100800002DB132462B460348BDE87040184770BDF5
:100810006C2500207400020010B1012804D070473C
:10082000034B1B6C5B0701D1FFF7DCBF704700BFB8
:100830006C25002008B54FF04003EFF3118183F3DE
:100840001188BFF36F8F124A136843F0020013F050
:10085000010310600CD04FF08042D2F80C34D2F873
:100860000C2413F0010303D00A4809F0C1FF01234F
:1008700081F31188BFF36F8F23B1BDE808400020DA
:10088000FFF7B0BFBDE80840012007F01FB900BF67
:10089000BC250020AC250020094BBFF35B8F53E83B
:1008A000002F22F0020143E800100028F7D1BFF327
:1008B0005B8FD30702D401200EF0FFBD704700BF4D
:1008C000BC2500207FB500220123CDE9022304AB23
:1008D000CDE90433094ACDF800D06B46CDF804D0F9
:1008E00009F0BFFF002805DB4FF480420023684673
:1008F00007F0AAFF07B05DF804FB00BF35A80100B0
:100900002DE9F8433A49BFF35B8F0646012251E8CF
:10091000003F41E800200028F9D1BFF35B8F33B9D5
:10092000344935484B60CB608A6009F063F8731E28
:10093000012B32D8012E07D14FF08043D3F81C345D
:1009400003F00303012B28D00EF095FE044618B9DE
:100950002A4B1B78002B44D14FF04003EFF3118555
:1009600083F31188BFF36F8F0124254FDFF8948044
:10097000DFF894904FF08042D2F81834D2F818245F
:10098000D2030CD503F00303012B01D0012E06D1B5
:100990000CB385F31188BFF36F8FBDE8F883ACB15A
:1009A000284600F0F3FB4FF08042D2F81835002BB8
:1009B000E0D139680029DDD03B603B680123C2F8F3
:1009C0001835C8F88031C9F80030D3E7002121205C
:1009D00008F03CFBE7E74FF080430222C3F8042312
:1009E000DBE74FF080430222C3F808230546BCE74B
:1009F000C02500205C250020882500209635002099
:100A00000401004000E100E008000040044A1368CF
:100A1000C81A20F07F400344136008F08FBC00BF69
:100A2000D42500202DE9F047860006F1804600F12C
:100A3000500406F58836A400DFF87C80D6F84035EF
:100A4000A4B204F180444FF4803721F07F4504F5CF
:100A500088348740C146D8F804A5A3EB0A0323F0E5
:100A60007F432AF07F42012BC6F8402502D1132094
:100A70000FF0FAF80AF10202AB1A23F07F43B3F544
:100A8000000F88BF1546002323602368C9F844730C
:100A900025F07F43C6F84035D9F804359A4506D08D
:100AA000EB1A023B23F07F43B3F5000F01D8BDE8FA
:100AB000F0872B46CFE700BF00100140F8B5154C7A
:100AC000154F0026154B00201D689C4606B1F8BD49
:100AD000D4F80423D203FAD53A68002AF7D03E604E
:100AE0003A684FF48032C4F84823D4F84015D4F85B
:100AF0000465721A22F07F42B2F5000F88BF3146BA
:100B000001261DB15A681860A847DBE7CCF80050F1
:100B1000DDE700BF0010014040110140C825002062
:100B200038B5104D00244FF48033C5F80845C5F89A
:100B300004330D4B4FF40032C3F8802101212246CB
:100B4000112000F0B9FA112000F084FA074A0123BD
:100B50001360074A2B6002201360FFF7D1FE204686
:100B600038BD00BF0010014000E100E00810014066
:100B7000D0250020134BB0F1FF3F08BF18460138C5
:100B800000281CDD9842A8BF18460F4BD3F8042557
:100B90000E4B1968521A12F4000F22F07F4318BF4F
:100BA00000200B4A013303440A48106000205060C3
:100BB000044A934294BFC9188918FFF733BF002035
:100BC000E3E700BFFFFF7F0000100140D4250020B5
:100BD000C82500200D0A0100044BD3F80405044B7E
:100BE0001B68C01A20F07F40704700BF0010014012
:100BF000D4250020034B9B681BB1481E18BF012061
:100C000018477047D825002010B51C46034B1B68B9
:100C100011460BB122469847204610BDD82500202A
:100C2000024B5B6803B11847704700BFD82500200E
:100C300030B1044B02681A6042685A6082689A6058
:100C400000207047D825002070B586B00E461546A6
:100C500000210446182268460AF0D1FF0B490C4BCC
:100C6000ADF80C50CDE9011604932CB96946204625
:100C700003F0C8FE06B070BD012220460CF0DFFE76
:100C80000028F3D16FF01500F4E700BF0C04020058
:100C9000210C0100014B1868704700BF7C04002044
:100CA000F0B5082289B00C46064609F0B9FFCB6AB8
:100CB00003930B6B04934B6B05938B6B0693CB6B7E
:100CC0000793002708236A4669466846CDE90177FD
:100CD000009709F0A7FE082305466A4631463046CC
:100CE00009F0A0FE236B0393636B0493A36B05933E
:100CF000E36B0544CDE906376A4608236946684632
:100D000009F090FE3146054408236A46304609F052
:100D100089FE236A0093636A0193A36A0293A36B1B
:100D20000693E36B0793054408236A463046CDE9F2
:100D30000477039709F076FE636A0093A36AA26BB7
:100D40000193E36A02930492636BE26B0393CDE930
:100D50000523236A0793054408236A46304609F0B1
:100D600061FEE36A0093236B0193636B0293236A32
:100D70000693A36A0793054408236A463046CDE9E3
:100D80000477039709F082FF236B0093636B019351
:100D9000A36B0293E36B0393636A0693E36A07937F
:100DA0002D1A08236A463046CDE9047709F06EFF14
:100DB000636B0093A36B0193E36B0293236A03932A
:100DC000636A0493A36ACDE90537236B07932D1A51
:100DD00008236A46304609F059FFA36B0093E36B82
:100DE000CDE90137636A0393A36A0493E36ACDE90B
:100DF0000537636B07932D1A08236A46304609F0BE
:100E000045FF2D1A10D40D4C35B908223146204625
:100E100009F012FF01280FD0082322463146304640
:100E200009F034FF2D1AEFE7044A08233146304613
:100E300009F0F8FD2D18F8D409B0F0BD60040200E7
:100E4000F0B5264E07460C460FCE8DB001AD0FC54E
:100E50000FCE0FC596E8070085E807003846002F3B
:100E600038D0002C38D0381F2146024610344B7839
:100E70000D781B0443EA0563CD782B438D7804314C
:100E800043EA05238C4242F8043FF0D1144C04217C
:100E90008A07036916D1C3F30742A55C1A0EA25C48
:100EA00042EA0562C3F30725DBB2655DE35C42EA13
:100EB000054242EA03220CAD21F003032B4453F810
:100EC0002C3C534050F8042F013153402C2903612E
:100ED000DED101200DB0F0BD2046FBE7B4020200D8
:100EE0004B0A02002DE9F043154689B0064600285A
:100EF00058D0002959D0002A59D010230A466846F4
:100F0000194609F0CBFC294668462A4C0AF0D0FB6A
:100F100005F11007A146A035E8466A46102311786E
:100F2000013B615C02F8011BF9D168460AF005FC3F
:100F3000694604A80AF03AFC01A905A80AF036FCA3
:100F400002A906A80AF032FC03A907A80AF02EFCA1
:100F5000102319460DEB0302684609F09FFC394641
:100F6000684610370AF0A4FBAF42D5D1102498F898
:100F70000030013C19F8033008F8013BF7D168460E
:100F80000AF0DBFB294668460AF092FB102319465B
:100F90006A46304609F082FC68461022214609F074
:100FA0008AFC012009B0BDE8F0830846FAE7104644
:100FB000F8E700BF4B0A0200094A0A49936809682A
:100FC00019670949D8664B6843F080534B6000238A
:100FD00083F31188BFF36F8F9368186F704700BF5A
:100FE0002C2900206C09020000ED00E00F498A68FE
:100FF0004FF030001044EFF3098C80E8F01F4020E0
:1010000080F31188BFF36F8F094F4FF000660A6AB3
:101010008A603E60D06E0023D36680F3118802F1AF
:10102000300090E8F01F8CF3098870472C290020CD
:1010300004ED00E01EF0040F0CBFEFF30880EFF3A7
:101040000980816911F8021C0229FFD001B50AF05C
:10105000F2FC01BD43B2002B08DB012200F01F00AF
:1010600002FA00F05B09024A42F82300704700BF11
:1010700000E100E043B2002B0DDB01225B0900F030
:101080001F0002FA00F02033034A42F82300BFF3A6
:101090004F8FBFF36F8F704700E100E0054B4209AF
:1010A00000F01F0053F82220012303FA00F0104043
:1010B000704700BF00E100E0D30742B254BF0231E5
:1010C0000021002AACBF02F16042074A4FEA4113F7
:1010D000ACBF02F5614200F00F00DBB2B4BF1354A5
:1010E00082F80033704700BF14ED00E008B572B617
:1010F000044BD86918B10022DA610EF0C7FA62B663
:1011000008BD00BF2C29002042F8203C009B42F87B
:101110001C3C0A49019B42F8183C029B42F8143CD3
:1011200021F001014FF0807342F8043C42F8081CA2
:101130000023203A0265C366704700BF879A01000A
:10114000074B9860104681F30988002163B681F34C
:101150001188BFF36F8F0022002308F094FC00BFBA
:101160002C290020014910220A60704710ED00E090
:1011700072B6404080F31188BFF36F8FBFF34F8F7B
:1011800030BF62B6BFF36F8F704700BF72B6494081
:1011900081F3118820BF80F3118862B6704700BFC9
:1011A00030BFFFF7FDBF00BF08B5084B084A23F06A
:1011B0007F039360BFF34F8FBFF36F8F07F052F839
:1011C00007F0D8FF00F070F907F070F80000000099
:1011D00000ED00E001B572B60B4AD06900281EBFD1
:1011E0000021D1610EF052FA62B6EFF30580A0F152
:1011F00010004FEAC0000549014409C99847BDE8FD
:1012000001400349084700002C2900200401020086
:1012100009140100002080F31488BFF36F8F0EF0D3
:10122000EBFE00200D490860BFF34F8F0C4880F3A0
:10123000088800F007F9402080F3118809484FF42E
:101240008061401880F30988EFF31480022108437D
:1012500080F31488BFF36F8FFFF7A6FF94ED00E0D3
:10126000A048002020490020EFF30880EFF3098117
:1012700001B5724600F04CF801BD00BF0D4B9A6AF3
:101280009A6A9A6A920708D55A6B9A6A120604D526
:1012900018B19A6A22F080029A62064B9A6A9A6A98
:1012A000D20658BF9A6A9A6A002042F0FF029A62F8
:1012B0000870704700ED00E00B4B9A6A9A6A9A6AD0
:1012C000920507D59A6A120404D518B19A6A22F4D5
:1012D00000429A62044B9A6A9A6A9A6A002042F41F
:1012E0007F429A620870704700ED00E0074B9A6AEF
:1012F0009A6A9A6A9A6A9A6A9A6A9A6A6FEA024239
:101300006FEA12429A620020704700BF00ED00E0D1
:1013100070B5364B5B688AB00E46C3F308030025F0
:1013200085F31188BFF36F8F02F07F41B1F17F4FDA
:1013300011D102F00C0108290DD0110701D4064685
:1013400001250022033B8DF80720032B47D8DFE857
:1013500003F0043E423B2E46F3E7244BDA6A920741
:101360003DD4DC6A14F0804408D028331B78EBB1FC
:101370000DF107010120FFF781FF04469DF80730BA
:1013800093B92022314602A80AF02EFC099B45B3EE
:10139000C3F3080222B96FEA53236FEA4323099388
:1013A00002A920460AF045FB0AB070BD104B1B781D
:1013B0002BB10DF107010120FFF77EFFDDE70D4B9B
:1013C000188884B2002CD9D0FFF790FFD5E70DF133
:1013D00007010020CFE70DF107010020ECE7002412
:1013E000CCE723F4FF7323F00103D8E700ED00E01E
:1013F00029ED00E02AED00E0024A536943F01003B2
:101400005361704700ED00E0044B9968186A884208
:1014100003D003494FF080520A6070472C29002006
:1014200004ED00E0064A11680023C1F307211846C5
:101430008B4200D17047936010610133F8E700BF21
:1014400090ED00E008B572B6002383F31388FFF730
:10145000E9FF144B4FF0FF32C3F88020C3F884201B
:10146000C3F88820C3F88C20C3F89020C3F89420D8
:10147000C3F89820C3F89C20C3F88021C3F88421C6
:10148000C3F88821C3F88C21C3F89021C3F89421B4
:10149000C3F89821C3F89C2162B6BFF34F8FBFF306
:1014A0006F8F08BD00E100E0044800234021C2180E
:1014B00001331E2B82F80013F9D1704700E100E0E0
:1014C000064B9B68834207D1EFF3058323B1044A9F
:1014D000536843F08053536007F0E8BD2C29002087
:1014E00000ED00E00CB41FB509B90DF10300CDE922
:1014F000020107AB069A0648019302A9FDF744FFD3
:10150000029B00221A7005B05DF804EB02B0704730
:1015100011BC01004FF08043C0B2C3F81C05BFF3FB
:101520004F8F0549054BCA6802F4E0621343CB6054
:10153000BFF34F8F00BFFDE700ED00E00400FA05A8
:1015400020B1034B800143F001031847704700BFEF
:10155000400302002DE9F843604FDFF898813E46D2
:101560004FF0FF324FF0FF33404607F06DF9BFF305
:101570005B8F3C68BFF35B8F14F0010455D0DFF83C
:101580007091574C574D58484A46214609F09EF9EC
:1015900000283ED02022294620460AF015FB0028CC
:1015A000F1D04FF000094FF0FF324FF0FF33012030
:1015B00000F090FA00F108050221044628460DF0DB
:1015C0002CF93E23037042234370012128460DF07D
:1015D00024F908230370412128460DF01EF9054621
:1015E00000F8019BB9F1000F16D0402200210AF04B
:1015F00006FBBFF35B8F56E8003F23F0010346E88C
:101600000032002AF7D1BFF35B8F204600F08EFE38
:10161000A6E74FF01F09C6E733490AF081FB3349BB
:1016200005F121000AF07CFBE3E7BFF35B8F3B6829
:10163000BFF35B8F9B0793D52D492B480AF015F814
:10164000002811DBBFF35B8F3B6825492548BFF3BA
:101650005B8F13F0040F01F12002254B18BF0146E8
:10166000104609F082F904464FF0FF324FF0FF3385
:10167000012000F02FFA00F1080902210546484632
:101680000DF0CBF83E23037022234370012148461E
:101690000DF0C3F809230370212148460DF0BDF871
:1016A000034601309CB91F221A70FF2120220AF044
:1016B000A6FABFF35B8F56E8003F23F0020346E82B
:1016C0000032002AF7D1BFF35B8F28469EE7002245
:1016D00005491A700AF024FBEBE700BFE42500205F
:1016E0006A290020520B02008A290020AA29002022
:1016F0000C050200D006002070B5214CBFF35B8FB3
:101700002368BFF35B8FDA0706460D4601D50C2030
:1017100070BD012931D8BFF35B8F54E8003F43F01F
:10172000020244E800210029F7D1BFF35B8F9B0739
:10173000EDD4144831460AF0F3FA134806F12001BB
:101740000AF0EEFABFF35B8F75B154E8003F43F047
:10175000040344E80032002AF7D1BFF35B8F0B4843
:1017600007F04CF80020D3E754E8003F23F00403CF
:1017700044E80032002AF0D0F6E71220C8E700BFA4
:10178000E42500208A290020AA290020D006002074
:1017900070B5067D044676B983681D8842F226023C
:1017A000954245D00FD842F2010295424FD042F205
:1017B00025039D4213D02A4BD3F8343120461B69B0
:1017C000BDE87040184742F25E039D42F3D1032109
:1017D00008300DF041F8A06890F840102EE0032189
:1017E00008300DF039F8204604F050FCBFF35B8F51
:1017F0001C4B1A68BFF35B8F920707D50C26314646
:1018000042F225000AF068FA002070BDBFF35B8F3A
:1018100053E8002F42F0010143E800100028F7D1FF
:10182000BFF35B8FD307E9D40F4806F0E7FFE6E785
:10183000032108300DF010F8A0683146FFF75CFF77
:101840000646204604F022FC31462846DAE7DA78DC
:1018500002F07F02DA701A7922F001021A71AAE707
:10186000B8020020E4250020D006002010B588B082
:101870000C4C0D4900220023CDE9062300230A2247
:10188000CDE90323CDE9013300934FF48F62074B79
:10189000204606F01BFE0649204608B0BDE8104071
:1018A0000DF0EFBE481400209837002055150100B8
:1018B0004B0B020003490448CA79C2EBC202FEF78F
:1018C000ABBC00BFB8020020720B0200F7B5164691
:1018D0001F46044620B96FF00104204603B0F0BD56
:1018E00001A908F044FE1149024620460AF05DF9BC
:1018F00004460028EFD1BFF35B8F0D4D2B68BFF37B
:101900005B8F5B07E9D4943D072229463846B047F0
:10191000062806D80722214628460AF070F9EC71FD
:10192000DBE70723B0FBF3F0E871D6E78509020097
:101930004C0300202DE9F8430329DDF820900746E9
:10194000884614461D4646D927490AF0F5F821462F
:10195000A8F10302F81C0AF0F9F838460AF009F970
:10196000404538BF2F2304463CBF3B540134AE1DD5
:10197000A04503D8B9F1000F14D115E0A8EB04037A
:101980003A193046012107F021FF013EB5420444D7
:10199000EED1444524D22B7830333B550134B9F194
:1019A000000F15D0A04505D84744002307F8013C97
:1019B000BDE8F8832F233B5501343D19A8EB040201
:1019C000494628460AF0C2F828460AF0D2F80444EC
:1019D000A045EDD8E8E70029EAD000230370E7E747
:1019E000B9F1000FE0D1F3E7780B0200014807F0EE
:1019F00079B800BF8004002010B5154CE379E3B13D
:101A0000BFF35B8F134C2368BFF35B8F9B0701D43D
:101A100000F0C2FCBFF35B8F54E8000F20F480435A
:101A200044E80032002AF7D1BFF35B8F10F4804006
:101A30000CD0FFF7DBFF002008E000F063FFE37944
:101A4000002BDDD100F06EFF0028D9D010BD00BF03
:101A5000B80200204C030020F0B40278012A0446AA
:101A60000B4616D0022A2CD08AB9194A0D4602F12B
:101A70001007106851682E4603C60832BA42354630
:101A8000F7D11278327062885A73120A9A73F0BCD6
:101A900070470F4A0D4602F11007106851682E4634
:101AA00003C60832BA423546F7D1127832706268FE
:101AB0005A73C2F30721120CDA73120A99731A745B
:101AC000E5E70146F0BC112218460AF08DB800BFC8
:101AD0007F0B020038B5054605480CF048FE044669
:101AE00020B1002108300CF061FE2575204638BD7C
:101AF0001808002070B502460B464FF04001EFF386
:101B0000118581F31188BFF36F8F0C480021D0F845
:101B10000041C0F8001185F31188BFF36F8F24B91D
:101B2000BDE870400120FFF7D5BF012304F1080094
:101B30002375A1810CF03AFE204670BDB80200204A
:101B400070B504460F2C0D461046194605D80D2CCD
:101B500012D9BDE87040FFF7CDBF132C0CD10B4854
:101B60000CF005FE044628B1002108300CF01EFEE2
:101B700001232375204670BD02460B460DB1044873
:101B8000EEE7BDE870400120FFF7A4BF4008002049
:101B9000A007002038B583681A7872B9B3F80140FD
:101BA000204601F0B3FB054640B9084B1A8822B91C
:101BB0006FEA04506FEA1050188038BD012101F01F
:101BC000B1FB2846BDE838400AF051BE6429002028
:101BD00010B50121044608300CF046FE2146034AA8
:101BE0000078BDE8104008230AF050B9EC05020067
:101BF00038B58368B3F801001D7801F087FB04460F
